:020000040100F9
:1000000038480020E5000001ED000001EF0000018C
:1000100000000000000000000000000000000000E0
:10002000000000000000000000000000F1000001DE
:100030000000000000000000F3000001F5000001D6
:10004000F7000001F7000001F7000001F7000001D0
:10005000F7000001F7000001F7000001F7000001C0
:10006000F7000001F7000001F7000001F7000001B0
:10007000F7000001F7000001F7000001F7000001A0
:10008000F7000001F7000001F7000001F700000190
:10009000F7000001F7000001F7000001F700000180
:1000A000F7000001F7000001F7000001F700000170
:1000B000F7000001F7000001F7000001F700000160
:1000C0000348854600F056F80048004751050001F6
:1000D0003848002040BA7047C0BA70470138FDD197
:1000E000704700000448804704480047FEE7FEE7E9
:1000F000FEE7FEE7FEE7FEE795030001C100000111
:1001000030B50B46014600202022012409E00D46AF
:10011000D5409D4205D31D469540491B2546954037
:1001200040191546521E002DF1DC30BD03460B432D
:100130009B0703D009E008C9121F08C0042AFAD29D
:1001400003E00B780370401C491C521EF9D2704723
:10015000D2B201E00270401C491EFBD2704700225F
:10016000F6E710B513460A4604461946FFF7F0FFB6
:10017000204610BD064C0125064E05E0E36807CC7D
:100180002B430C3C98471034B442F7D3FFF79CFF45
:10019000C0070001D0070001F7B5D4B004460E46F1
:1001A00000205390052052900025002700BFEFF358
:1001B00010800090FF21453101A8FFF7D0FF00F02B
:1001C000F1F905462448854218D1012000038442F4
:1001D00002D1002053902AE001204003844202D142
:1001E0004011539023E003200003844203D10120F7
:1001F000400253901BE0529857B0F0BD174885421B
:1002000013D101200003844201D153900FE001205B
:100210004003844201D1539009E00320000384424B
:1002200001D1539003E05298E6E75298E4E705AF16
:100230000137FF2241320A4901A8FFF777FF012069
:1002400000F04FF93146569A5398B84752900098AB
:1002500000F047F95298CFE7C440130085601300BF
:10026000E8050001F1B58AB0002009907D20C000AA
:1002700008900125AD020027002007907F200690FE
:1002800040240026002005900390200102900020C9
:1002900001903E490A98884206D83D4800686102AC
:1002A00088433B49086006E0394800680121C903DA
:1002B0000843374908607D21C9000A98FFF720FFED
:1002C0007D21C9000090FFF71BFF450100BF3048AA
:1002D00000687F21090288430190200201990843A8
:1002E0002B4908600520FFF7F9FE10E00120FFF719
:1002F000F5FE2748406B02210840002800D007E0A7
:100300000598411C05910899884200D900E0EDE765
:1003100000BF1F48C06B86B2AE4201D9771B00E018
:10032000AF1B0298874203D2E0B20390B8B20290AA
:10033000AE4201D3069400E007940699079840184E
:10034000C005000E04900498A04200D103E0049C74
:1003500009988742BBD800BF0D4800687F21090279
:1003600088430190039800020199084308490860F6
:100370000846406840084000486000BF04484068A4
:10038000042108400028F9D10BB0F0BD0090D00343
:100390000010024010B53E48C0690121090708431A
:1003A0003B49C861812000063A4908633A484861E0
:1003B0003A4808623A48006803218903884338496B
:1003C00008603421374800F073F836480069401C53
:1003D000002803D033480069002817D12C48406812
:1003E0000121090408432A4948600846406807215A
:1003F00009028843264948600846406809150843B1
:10040000234948602848FFF72DFF3FE021488069D5
:100410004409640123480078C006C00E04431D4807
:1004200084611B4800680121C9038843184908609A
:10043000084600687F21090288430446194800697C
:10044000000220431249086008464068012109045F
:1004500008430F494860084640680721090288435D
:100460000B49486008464068091508430849486038
:100470000846006A0D490840054908620846006AB6
:100480000849C968090208430149086210BD000013
:1004900000100240007000400F0800001800020029
:1004A00000100140004000200090D003FF00F8FF42
:1004B00070B504460D462A46214601200003FFF789
:1004C0006BFE70BD02E008C8121F08C1002AFAD1F5
:1004D00070477047002001E001C1121F002AFBD1C4
:1004E000704780F31088704730B502460B460021F4
:1004F000C94312E01078521C414000240BE0480828
:10050000CD07ED0F002D01D0074D00E0002568401C
:100510000146601CC4B2082CF1DB18465B1E0028A3
:10052000E8D1C84330BD00002083B8ED0446012067
:10053000C007204305490863206880F3088800BF8E
:1005400062B66068804700BFFEE7000000700040B0
:10055000114C124D1249206888421AD12821204698
:10056000FFF7C2FFA16A884213D16168022902D154
:100570002146183101E0214608310846074A016842
:10058000914205D3412292040168914200D205684C
:1005900000BF2846FFF7CAFF0040000100800001AD
:1005A00011C011CA70B5D2B00024002500BFEFF30E
:1005B00010800646FF21453101A8FFF7D0FD01ACB0
:1005C00001349822074901A8FFF7B0FD0120FFF789
:1005D00088FFA04705463046FFF783FF284652B004
:1005E00070BD00002807000140BA7047C0BA7047CC
:1005F0000138FDD170470000F7B50325AD06286A24
:1006000082B016460C46400840002862286A022143
:1006100008432862286A8007FCD4662068600127A6
:100620002F61A86AC005FCD5992068602F61A86A6F
:10063000C005FCD5FF209130FFF7DAFFFF2301331F
:10064000AB626846EF60352169602F61A96AC90510
:10065000FCD5AB62A969EF60C9B205226A602F615F
:10066000AA6AD205FCD5AB62AA690902D2B21143CB
:100670000180C80702D0032005B0F0BDAB626869F5
:10068000FF210831884368616869C91E08436861B1
:1006900002980002483068600820A860EE602F6170
:1006A000A86AC005FCD5FF200130A8620023F61C13
:1006B000B0080ED0B2081148006899006054060ACC
:1006C00009194E70060C000E8E705B1CC8709A42A1
:1006D000F1D8FF200130A8626869FF210831884302
:1006E0006861686938436861286A80088000286208
:1006F000286A38432862002005B0F0BD8000000C55
:10070000032080064169FF2208329143416142691A
:1007100001210A434261026A920892000262026A5F
:100720000A43026270470000002003218906096A1B
:10073000490849000322920611621146096A022201
:10074000114303229206116200BF03218906096A40
:10075000022211400229F8D0D101032292069162AF
:100760000321D1609F2151600121116100BF03214C
:100770008906896AFF22013211409142F7D1032292
:1007800092069162114688694969FF2208329143B5
:100790000322920651611146496901221143032245
:1007A000920651611146096A890889001162114651
:1007B000096A012211430322920611627047000068
:1007C000D00700010040002038080000D4040001D8
:1040000011C011CA0100000000800001BCD30000F3
:1040100053A0D5081100010000400201E8D40000BF
:0C402000CBA8292211000100571C042B22
:106000007ADA12CA01000000F4010000000000006A
:106010000000000000000000000000000000000080
:106020000000000000000000000000000000000070
:04603000773E0CFCAF
:10800000D0B70020698100017181000141B00001F9
:108010000000000000000000000000000000000060
:1080200000000000000000000000000005B4000196
:1080300000000000000000002781000109B40001D9
:108040007B8100017B8100017B8100017B8100013C
:108050007B8100017B8100017B8100017B8100012C
:108060007B8100017B8100017B8100017B8100011C
:108070007B8100017B8100017B8100017B8100010C
:108080007B8100017B8100017B8100017B810001FC
:108090007B8100017B8100017B8100017B810001EC
:1080A0007B8100017B8100017B8100017B810001DC
:1080B00011B600017B8100017B8100017B81000101
:1080C0000348854601F076F80048004709F90001A9
:1080D000D0B7002040BA7047C0BA70470138FDD110
:1080E0007047000040BA7047C0BA7047704670478A
:1080F000084B19680868203080F30988022080F353
:108100001488BFF36F8F3FBCAE4608BC04BC62B698
:1081100018470000A4470020EFF3108072B67047A4
:1081200080F310887047EFF309800E4B1A682038EF
:108130001060F0C044464D4656465F46F0C008B554
:1081400072B60AF09BFF62B60CBC1168086810306A
:10815000F0C8A046A946B246BB4680F3098820383D
:10816000F0C81847A4470020044880470448004747
:10817000FEE7FEE7FEE7FEE7FEE7FEE761B400018B
:10818000C180000130B50B460146002020220124A9
:1081900009E00D46D5409D4205D31D469540491B3B
:1081A0002546954040191546521E002DF1DC30BD84
:1081B00070B500242546002801DA01244042002938
:1081C00001DA01254942FFF7DDFFAC4200D0404211
:1081D000002C00D0494270BDF0B51FB40646002007
:1081E00082B005464024019100901BE0019922468F
:1081F0000F46304600F02DFE049A059B801A9941E7
:1082000010D310461946224600F013FE361A8F414D
:108210000197224601200021009F00F00AFE381835
:108220004D4100902046641E0028DFDC019B009831
:108230002946324607B0F0BD01464139192900D818
:10824000203070470549064A08685043054A80189F
:10825000086040087047014908607047FC470020EB
:108260006D4EC6413930000003460B439B0703D0D7
:1082700009E008C9121F08C0042AFAD203E00B78EB
:108280000370401C491C521EF9D27047D2B201E063
:108290000270401C491EFBD270470022F6E710B561
:1082A00013460A4604461946FFF7F0FF204610BD64
:1082B000421C0178401C0029FBD1801A704710B580
:1082C000002200E0521C835C8C5CA34201D1002B95
:1082D000F8D1D8B2E1B2401A10BDC9B203E00378B8
:1082E0008B4203D0401C521EF9D20020704730B59B
:1082F00004460020034600E05B1C934203D2E05C8E
:10830000CD5C401BF8D030BD03460A780270401C9B
:10831000491C002AF9D11846704730B5054600209F
:10832000034600E05B1C934205D2EC5CC85C201A5B
:1083300001D1002CF6D130BD0FB400B58DB009903D
:108340000B9010A900200091C0430A9000200C90CF
:1083500006480690064807906A4609A80F9900F05B
:10836000B1FD0DB008BC04B018470000E58E000157
:10837000058F0001FFB5087889B01546FF2805D0A4
:10838000491C2D2804D00022002407E000240BE023
:108390000122F9E70A235C430419491C0878FF28E5
:1083A000F8D1002A00D06442002004902A780146C7
:1083B0002D2A01D02B2A0FD16D1C2D2A02D000228C
:1083C000049209E00122FBE700260A2233466D1CD5
:1083D00000F0F2FC381871412F78FF2FF4D10C9A7D
:1083E000A218069202460A4304D0FF23069A91334C
:1083F000DA4205DA002109980A4606C00DB0F0BD40
:108400000024B74AB54D2646079200F011FC0290B1
:1084100006980391002801DA474200E00746390533
:108420000020AF4A001C51410191009012E0F80772
:1084300007D022462B463046079900F0D9FA064667
:10844000079122462B461046194600F0D1FA044601
:108450000D467F10002FEAD10698019B0028009A54
:108460000399029806DA00F02BFB3246079B00F0D6
:1084700027FB05E000F0BCFA3246079B00F0B8FA93
:10848000049A002A02D00122D2075140099A03C25D
:10849000B4E7FFB591B0002009900025ED432E20F0
:1084A0009E685C681F460190B9696D1C12988847E8
:1084B0000090396A88470028F6D10098401C0AD0FD
:1084C0000D20C0018443002E12DD00982B2809D016
:1084D0002D280DD103E00020C04315B0F0BD0120D0
:1084E00080020443B9696D1C12988847761E00907B
:1084F00003A9600501D52D2000E02B206A461073EA
:10850000491C0CA80F9102900AE0B9696D1C1298E1
:10851000884700900120400204431398761E0560AE
:10852000002E02DD00983028EFD001990098884293
:1085300046D18020044308E00998401E099001209C
:10854000400204431399681C0860B9696D1C761ECB
:108550001298884700903028EED031E00199884287
:1085600005D1200603D480200443761E1EE0009827
:1085700003F05CFA002826D001204002044307A93A
:108580000F980331761E88420BD200980F9930382D
:1085900008700F98401C0F90200607D50998401EC0
:1085A00003E0200602D40998401C0990A00502D5DA
:1085B0001399681C0860B9696D1C1298884700906F
:1085C000002ECBDC59E0002E57DD0098652801D045
:1085D000452852D1A00550D5032000028443B96933
:1085E0006D1C761E129888470090002E0CDD2B28FB
:1085F00004D02D2808D1FF2001300443B9696D1C37
:1086000012988847761E0090E00501D52D2100E0E4
:108610002B21029801700298401C0290019025E0E5
:108620000120400204430EA902980131761E8842BF
:108630000ED20098029930380006000E087003D15F
:108640000299019881420AD90298401C029006E0E2
:10865000E00501D5234801E0224840420990B9696C
:108660006D1C12988847009013980560002E04DD59
:10867000009803F0DBF90028D2D1F96912988847F5
:108680000F99FF200870029903AA087000200A9031
:108690000B900CA90AA8099BFFF76CFEA00502D459
:1086A0000120C04319E72420044209D0E00713D178
:1086B00038680B9A0A99031D3B60006806C00BE0FE
:1086C0000B990A9800F05CFB0146E00704D138687A
:1086D000021D3A60006801602846FEE60000144072
:1086E0000000F03FF1D8FFFFF7B582B00F4600263B
:1086F000029C03F087F80090006801902578641CC4
:10870000002D05D000F0CAFB0068405DC007F5D120
:108710002B2D02D02D2D1CD0641E0098002101604D
:1087200039462046049A00F0FFFB0146002F04D092
:108730003868A04201D10298386000980068022889
:108740000BD00098019A0260700506D5484205B02A
:10875000F0BD012080020643DFE70846F7E7F8B5E1
:1087600002464A40D40F42004B0052085B089A422E
:1087700002D20246084611464A0023D0C30D4A00E1
:10878000DDB2120EAD1A202D35DA49020126490A52
:10879000F6058A19002C00D0524220214F1B1146A9
:1087A000B9402A411018C20D9A4221D0002C17D08E
:1087B000012D08DCDA05801AD20F8019D207DBB24E
:1087C00000F060FCF8BDDA05801A012340001B06AA
:1087D000C01880185A428018CA0F1043490007E099
:1087E0004908C2071143DA05801A80194008801829
:1087F00000F040FCF8BD61000122511A001BF7E7B0
:108800000122D2075140AAE70122D2075040A6E731
:10881000024670B54A40D30FDB0740002DD04A0016
:108820002AD0010E140E000212020919400A520A3F
:108830008418E50104465443000A120A2E045043EA
:10884000A4194219200CC543AA18120C0125AD0326
:10885000521C521912047F39240400D0521C1043B8
:1088600001D44000491EC2B20C06C0092018401CA9
:108870004008802A02D003E0002070BD400840007C
:10888000002900DA0020184370BD0000F0B507464B
:108890000846584087B0C00F049048000E46590063
:1088A00040084908BC1A884105D2384631461E4660
:1088B00017460B4602465800400810434CD0300D76
:1088C000039040055900400D490D0590401A029053
:1088D000402872DA18030121000B090508430190B2
:1088E00004980092002805D0019952420020884146
:1088F00000920190029840210A1A0199009800F014
:1089000098FA05460C466B4607CB00F0B3FAC0193F
:108910007141039A0E0D0023D71756401A467A402C
:10892000164344D0049A002A2DD0029A012A039AB1
:1089300015DC1205C01A914101263605001C714153
:10894000D20F059ED2070093019202962A46234633
:1089500000F0DEFB07B0F0BD38463146FAE71605F9
:10896000224A0F46B218C01AB74101210905001C5E
:108970004F4100187F41114618187941E20F10430A
:108980006D19644113E0E2076D0815436408C207DE
:108990001443039A01261205C01A91413605001CA2
:1089A0007141CE07400830434908C01851412A465A
:1089B000234600F0A0FBCDE7FFE70498012240002A
:1089C000C117121A00238B4104983146C417381A74
:1089D000A141EEE730B40124E407634030BC55E721
:1089E00030B40124E407614030BC4FE70000E0FFF1
:1089F000F0B51FB488B00B99099800244840099934
:108A0000C00F490049080991C0070B99009049001F
:108A100049080B9109990898A64608431CD00B9960
:108A20000A98084318D0099801244000420D4800D4
:108A3000410D099824050003000B204309900B9871
:108A40000003000B20430B9050181C4940180022D3
:108A500001901446104605E0002001460DB0F0BD1F
:108A6000032801DA034600E003239C46C11A0AAE3C
:108A70000AE05F0008ADED5B4F00F75B7D43002728
:108A8000AA187C41491C5B1E6145F2DD410004AB24
:108A90005A522104120C0A43240C401C0828DFDB24
:108AA000019802900099704601910090059B049AEC
:108AB0000799069800F02CFBD0E700000DFCFFFFA3
:108AC000F0B50C465C4085B0E40FE40703944C001D
:108AD000002664085900944649080246029622433B
:108AE00021D062460A431ED06200570D4A000E0391
:108AF0002303550D012402462C492405781B1B0B2A
:108B0000360B401823432643614600901C46501AFA
:108B1000B44103D30098401C009002E092180098E2
:108B20005B41002803DA0020014605B0F0BD0020BB
:108B3000012109050746864611E064461D46141BBF
:108B4000B54106D36546521BB341744607430C43F7
:108B5000A646CD0740084908284392185B410546C0
:108B60000D43EAD11046184313D0604619465040D1
:108B70007140084306D06046101AB34106D2012264
:108B8000002306E000220123DB0702E00122D2439A
:108B90005310009874460105381C6141029C039DE6
:108BA0000019694100F0A7FABFE70000FD030000CB
:108BB00070B54B005B0803430BD04B005C0D0026E7
:108BC00033466542B341D417AD1AA34102DB0020FE
:108BD000014670BD12053018514170BD10B500221C
:108BE0009623114600F04EFA10BD00000EB5C217D4
:108BF000C10F5040CA0740180021054B0293019253
:108C000000910A460B4600F083FA03B000BD000055
:108C1000330400000EB505490291002100910A4677
:108C20000B46019100F074FA03B000BD330400005C
:108C30000EB5054A0292002200921346019200F0FE
:108C400067FA03B000BD000033040000C20F41000A
:108C500040020123400ADB05D207090EC0187F2914
:108C600001DA00207047962903DC9623591AC84080
:108C700001E096398840002AF4D040427047000055
:108C800070B5CD0F4A0009030123090B1B051943D9
:108C90000B4BED070024520D9A4201DA002070BD03
:108CA000074B34339A4203DC9A1A00F0D2F802E000
:108CB0000449511888402C43F1D0404270BD000057
:108CC000FF030000CDFBFFFF4A0009030123090B4E
:108CD0001B0519430A4B10B5520D9A4202DA0020C7
:108CE000014610BD064B34339A4203DC9A1A00F059
:108CF000B0F810BD034BD21800F09BF810BD000077
:108D0000FF030000CDFBFFFFC20FD2074000400869
:108D10000BD0C10D0723DB01C91840020905400A29
:108D20001143C208400711437047002001467047B5
:108D300010B5002904DB0124E40740428C412146A0
:108D4000002B04DB1C460123DB075242A3418B426C
:108D500000D1824210BD000010B5002904DB0124BF
:108D6000E40740428C412146002B04DB1C460123D2
:108D7000DB075242A341994200D1904210BD00004E
:108D8000CB0FDB07490010B5490802460A4307D05C
:108D90000A0D07240903E401090B121B002A01DC58
:108DA000002010BDC900440F0C43C100E018D205DB
:108DB000801800F05FF910BDF0B51FB486B0002038
:108DC0000090019002900698069980B2049007984E
:108DD000090C02040014114307900027089D09980C
:108DE00006913E463C4603900398A9B20204000C4B
:108DF000039004982D0C154348430021224600F0AF
:108E000018F8C719714110340E46402CECDB384677
:108E1000029A00F00EF8009A019B801800905941C8
:108E200002980191103002904028CCDB00980BB0E2
:108E3000F0BD10B5202A04DB0146203A9140002005
:108E400010BD914020239C1A0346E34019439040F3
:108E500010BD10B5202A04DB0846203AD04000217E
:108E600010BD0B46D340D0402024A21A91400843A5
:108E7000194610BD10B5202A06DBCB170846203A4C
:108E80001041C1170B4306E00B461341D04020248C
:108E9000A21A91400843194610BD000000487047CF
:108EA0005849010110B50446FFF7F8FF0068005D5E
:108EB000C007C00F10BD0000026813785118016090
:108EC0001846704710B5D1600449516104491162D8
:108ED00000211161114600F08FF910BDB98E00011B
:108EE000A58E00014268002A08D001680B78491C51
:108EF000002B03D0521E06C0184670470121C160E6
:108F0000881E70474268002A0BD0C3680168002B96
:108F100007D183688B4204D0491E521C06C0002032
:108F200070470020C0437047F7B582B0029C00270D
:108F30002078641C15460197302802D0002D15D0EA
:108F400015E020780127641C782804D0582802D026
:108F5000002D09D00BE0002D01D0102D07D10027E6
:108F600010252078641C02E0082500E00A25002670
:108F7000009610E00099012769430818020C294661
:108F800080B2714300908E183804864201D30120CC
:108F900001902078641C294600F01EF90028E9DAC7
:108FA0000398002805D0002F01D0641E00E0029C29
:108FB00004600198002806D002F024FC0221016020
:108FC000C81E05B0F0BD009930040843F9E7000061
:108FD0000FB400B589B00CA900910B990023CB60A8
:108FE000204B214A06930792042201921F4A0292C3
:108FF0001F4A089202466B460020FFF74AFA09B062
:1090000008BC04B0184770B586B006460020C043BF
:109010000190002015460C460091029104903246C2
:10902000694604A8FFF7D4FF024604982118002DD2
:1090300005D0002801D0084600E0204628600498AA
:1090400000280DD0002A02DD0098884208D0081BB5
:109050000190009432466946029404A8FFF7B8FFD5
:1090600006B070BDE58E0001058F0001FFFFFF7F98
:10907000A58E0001002904DA401C490001D14008F6
:109080004000704770B40024050C05D11024000482
:1090900002D1002921D01124050E01D1000208348B
:1090A000050F01D10001241D850F01D18000A41CF2
:1090B000002801DB4000641C002908D020252E1B5D
:1090C0000D46F540A14000D0012129430843010687
:1090D0001B1B000ADB1D02D5002070BC7047DB059E
:1090E000181880180029F8DA401C4900F5D170BC26
:1090F00040084000704710B5002B08DA0024401CDF
:10910000614192185B411A4301D14008400010BDF3
:10911000F0B51FB482B005460C0003D0084602F03B
:1091200059FB02E002F056FB203002460090214637
:109130002846FFF77EFE049B059A04460F46184317
:109140001143084314D0184610431BD00098402107
:109150000A1A18460599FFF77CFE05460E46009A46
:1091600005990498FFF765FE084305D0012004E047
:109170002046394607B0F0BD0020C11705430E4315
:109180002C43374300990E986305401A7905E40A89
:1091900000220C43FD0A0A3002D500200146E9E70F
:1091A0000105101969410C9C0D9D00196941FFF7DB
:1091B000A2FFDFE7064C0125064E05E0E36807CC79
:1091C0002B430C3C98471034B442F7D3FEF77CFF96
:1091D000884D0101A84D01013A2800D230382023E2
:1091E00002469A43412A01D310463738884201D3B8
:1091F0000020C04370470000F3B58DB000200A90F6
:1092000001200B90002608460C300C46099062693C
:10921000012109989047051E2ED0252D2DD0216AB9
:109220008847002818D06269012109989047216A6F
:1092300088470028F7D1411E62690998904700E0ED
:10924000761CA1690D988847216A88470028F7D1C4
:10925000E1690D988847DAE7A1690D9888470746C4
:10926000A84201D1761CD2E7E1690D9888477F1C9E
:1092700002D10A98002877D049E1002762693D466B
:109280003946099890472A280CD16269012109982A
:109290009047012506E00A214F433F18303FEBD4A9
:1092A0001020054362690121099890470146303931
:1092B0000A2903D29B498F42DEDCECE7E90600D4A1
:1092C000994F6C280AD04C2810D0682824D06A28DE
:1092D0002ED074280CD07A280AD00DE062690121C2
:1092E000099890476C2823D004211CE020200543D6
:1092F0006269012109989047A760656065284FD091
:1093000026DC582839D01ADC452849D012DC25281B
:1093100034D04128B0D143E06269012109989047D7
:10932000682802D008210D43E6E70120C002DEE7ED
:109330000220DCE7462833D047282CD130E05B28D8
:1093400070D061282CD063286CD0642823D161E0D0
:109350006F284FD009DC662822D0672820D06928E2
:1093600026D06E2817D12EE0CDE070284DD073287E
:109370006FD075284ED078280DD154E0A1690D9892
:1093800088470546252800D16CE7E1690D98884794
:109390006D1C00D16DE7BAE00A224CE00A2252E0CF
:1093A000012023466A46C0430D99FFF772F8A3E0F7
:1093B0002846402108436060A807234601D50022C3
:1093C00039E000223FE0E80700D020E72068011DD7
:1093D00021600068290501D5067018E7290701D525
:1093E000068014E7A90703D5F117066041600EE770
:1093F00006600CE72846402108436060A807234622
:1094000001D5082217E008221DE0484928460840F7
:10941000606016E02846402108436060A8072346A4
:10942000BCD5B9E715E02846402108436060A8078D
:1094300007D5234610220120C0430D99C046C046DF
:109440005AE0234610220120C0430D99C046C04671
:1094500052E000210C910B460091632802D05B285A
:1094600007D043E0E80601D40120A060012000906D
:109470003CE062690121099890475E2805D10120EE
:109480000C9001466269099890472169002906D12C
:109490000B4601AA8F00491CD3510829FADB00288A
:1094A00035D0216900290ED1C117C90E09184A11FA
:1094B000930001AA9A1849094901411A0120136829
:1094C00088400343136062690121099890475D2831
:1094D000E5D10C98002808D0002001AB81005A5833
:1094E000401CD2435A500828F8DB01AB0120224629
:1094F000C0430D99C046C04600280ADA401C06D178
:109500000B98002803D00020C0430FB0F0BD0A988C
:10951000FBE7E90702D10A99491C0A913618002095
:109520000B9074E6CCCCCC0CFFFFFF7FF1F7FFFF74
:1095300070B58D180478401CA207920F01D10278F3
:10954000401C231106D10378401C03E006780E70FE
:10955000401C491C521EF9D1002B15D002780C2654
:109560008A1A3440401C0C2C03D0A401121B9B1CF3
:1095700008E004782402121B401CF8E714780C70F1
:10958000491C521C5B1EF9D5A942D3D3002070BDE3
:1095900003B40148019001BD232A000003B401482F
:1095A000019001BD6D56000003B40148019001BD5A
:1095B0006560000003B40148019001BDAF7F000069
:1095C00003B40148019001BDB551000003B4014846
:1095D000019001BDD37E000003B40148019001BD9C
:1095E000697E000003B40148019001BDC37F000003
:1095F00003B40148019001BDE954000003B40148DF
:10960000019001BD9957000003B40148019001BDCC
:10961000ED57000003B40148019001BD1D7C00001E
:1096200003B40148019001BD0D2A000003B40148B4
:10963000019001BDAB52000003B40148019001BD8F
:10964000F58F000003B40148019001BDE1FE000068
:1096500003B40148019001BD250E010003B4014887
:10966000019001BDB143000003B40148019001BD68
:1096700085290000C943416070470268702392B297
:109680009A430A430260704770B5044601F0A8FF90
:10969000002818D08069002815D0FFF79FFA0546EA
:1096A0002046FFF79BFA2946FFF7AEF8FFF72CFBA1
:1096B000064A074BFFF704FA0022064BFFF7E6F8CD
:1096C000FFF75EFB70BD044DEAE700001F85EB511C
:1096D000B81E01400000394000803B4470B50D4683
:1096E0000646002401F07CFF002816D0C16900293D
:1096F00013D0026A002A10D08BB290B289B292B213
:10970000102D0CD0202D0AD0302D17D0402D15D083
:10971000502D13D0602D11D022E0002070BD891A89
:10972000B01AAF2292005043FEF742FD0446963431
:109730000FD47D20C000844211DC11E0191AAF2241
:10974000301A12015043FEF733FD4B21C900441873
:1097500001D5002404E0E1200001844200DD04463C
:10976000204670BD70B5104CA0421BD1851401215C
:10977000284601F0E7FD0021284601F0E3FD012124
:10978000284601F0D3FD0948606100202060606038
:109790001F21A16006492161A06160622062A06270
:1097A0000448E06170BD000000080240080A0200A1
:1097B0000000FC0F2E6D00000029016802D001227C
:1097C000114301E049084900016070470422002963
:1097D000816902D0114381617047914381610848DA
:1097E0000649C1620749016307494163074981632B
:1097F0000749C1630849074808607047220078009C
:1098000000080240E700E1009F00BF04190C0516A4
:1098100070206E286E2B00004008024002220029B2
:10982000016801D0114300E0914301607047C068B6
:1098300080B270470246526800200A4200D00120E0
:1098400070470000044A9068C90640094001C90EEB
:1098500001439160704700000008024070B5054662
:1098600049480C464EC88CB0039602930192009171
:109870004EC8079606930592049142680168806875
:10988000099208910A90414A00996846914217D17D
:10989000282104F0BFF80A99884211D1022D1ADB61
:1098A0000020646802460B900BA92046FEF71CFFBF
:1098B00005460B98A04209D00078002806D101E0A7
:1098C00033A004E0012D0AD0022D08D03EA004F000
:1098D0009FF90CB070BD0198012809D001250198AD
:1098E000A84207D1294647A004F02CF90CB070BD5E
:1098F0000225F4E7012D6C4614D01834012D13D045
:1099000047482268824206D16068002803D00721B8
:10991000890388420AD9294642A0636804F012F9F3
:109920000CB070BD0834E9E74C48EAE74CA004F0FD
:109930006FF96168206804F06DF8A268824206D071
:1099400003462946544804F0FDF854A0BFE72946D1
:109950005FA06368E26804F0F5F86846019503F0DB
:1099600079FC002801D06AA0B1E76EA004F050F99C
:10997000C82009F079FABFF34F8F72497048C86068
:10998000BFF34F8FFEE700000040000111C011CA75
:1099900061707073773A20626F6F74736574746965
:1099A0006E67207265636F726420696E76616C69A0
:1099B000642C2072656675736520746F20737769F7
:1099C0007463680D0A00000075736167653A206171
:1099D00070707377205B317C325D20286E6F206160
:1099E0007267203D2073776974636820746F2074F8
:1099F0006865206F746865722062616E6B290D0A5C
:109A00000000000061707073773A20616C726561CC
:109A10006479206F6E20415050256C750D0A00004E
:109A20000040020161707073773A2062616E6B25AD
:109A30006C75207265636F726420696E76616C6903
:109A4000642028616464723D30782530386C582079
:109A500073697A653D256C75290D0A000080000147
:109A600061707073773A20766572696679696E679E
:109A70002074617267657420696D61676520637227
:109A8000632028666577207365636F6E6473292E83
:109A90002E2E0D0A00000000F44C01012020202091
:109AA00020202072756E20424C45204F5441207476
:109AB0006F20777269746520612076616C6964201B
:109AC000696D6167652066697273740D0A00000034
:109AD00061707073773A2062616E6B256C752069D6
:109AE0006D616765206F6B20287665722030782560
:109AF00030386C582C20256C752042292C20737727
:109B000069746368696E672E2E2E0D0A00000000CE
:109B100061707073773A20666C6173682066616962
:109B20006C0D0A0061707073773A20646F6E652C5B
:109B300020726573657474696E672E2E2E0D0A008F
:109B40000400FA0500ED00E010B50B488CB01EC80B
:109B500003940293019200911EC807940693059204
:109B600004914268016880680A90099208916846E9
:109B700003F09EFB0CB010BD00400001F0B58DB0AD
:109B80000E46032807DA54A004F042F85AA004F065
:109B90003FF85F480FE00024B76822460BA938461B
:109BA0000B94FEF7A1FD05460B98B84202D0007851
:109BB000002804D057A004F02BF80DB0F0BD5A4B8C
:109BC00087CB039702920191009087CB079706926B
:109BD000059104909A68596818680A920991534A45
:109BE000009908906846914205D1282103F012FFA0
:109BF0000A9988420DD0009401940294039404942D
:109C00000594069407940894099449A00A9403F0D3
:109C1000FFFF55A17068FEF752FB002804D0706862
:109C20000178622908D02BE0012D03D0022D01D04C
:109C30004FA0C0E701953AE04178312902D032299E
:109C400002D01DE002AC00E006AC51A1801CFEF782
:109C500036FB002816D070684FA1801CFEF72FFB42
:109C6000002819D070684EA1801CFEF728FB002840
:109C70001AD070684BA1801CFEF721FB002815D07C
:109C800049A098E74E48854204D04E48854201D00D
:109C90004DA090E725600AE007208003854201D9A6
:109CA00058A088E7656002E0A56000E0E5602A460C
:109CB0005DA0716803F046FF684603F0CBFA002808
:109CC00001D062A077E766A003F0A2FF684603F028
:109CD000EFFA0DB0F0BD000075736167653A206260
:109CE00073736574203C6669656C643E203C7661E4
:109CF0006C3E0D0A0000000020206669656C643A25
:109D000020616374697665203C317C323E0D0A0027
:109D10003C4D010162737365743A20626164207680
:109D2000616C75650D0A00000040000111C011CA88
:109D300062737365743A206578697374696E67201D
:109D40007265636F726420696E76616C69642C2041
:109D500072656275696C642066726F6D20736372E0
:109D6000617463680D0A00006163746976650000C0
:109D700062737365743A20616374697665206D75EA
:109D800073742062652031206F7220320D0A00004A
:109D9000616464720000000073697A65000000006D
:109DA000637263007665720062737365743A20753E
:109DB0006E6B6E6F776E206669656C640D0A0000CD
:109DC000008000010040020162737365743A2061F3
:109DD000646472206D757374206265204341494943
:109DE000435F415050315F42415345206F722043E1
:109DF000414949435F415050325F424153450D0A4A
:109E00000000000062737365743A2073697A6520FC
:109E100065786365656473207468652062616E6B44
:109E20002073697A650D0A0062737365743A2025A0
:109E300073203D2030782530386C582C207772699B
:109E400074696E672E2E2E0D0A0000006273736512
:109E5000743A20666C617368206661696C0D0A0053
:109E600062737365743A206F6B2028766572696639
:109E7000696564290D0A000000B583B00021032044
:109E80000B46012201910090920203A1034809F0C0
:109E900061FC03B000BD0000434C4900A5A20001D5
:109EA00010B5022805DB48680DA1FEF708FA002866
:109EB00005D00D480078002804D00CA103E006F07E
:109EC000C3FF10BD0BA110A003F03CFE124C13A069
:109ED000218903F037FE1CA0E16803F033FE10BDBA
:109EE0006A736F6E000000008847002076616C691D
:109EF0006400000064656661756C7420286E6F7480
:109F00002073617665642900706172616D733A2017
:109F100025730D0A00000000AC5C002020206C6559
:109F200064203D2025752020286C65643120626CFA
:109F3000696E6B2068616C6620706572696F642C55
:109F4000206D73290D0A0000202070776D203D20C0
:109F5000256C7520202870776D20647574792C200D
:109F60002525290D0A000000F3B595B015980D467A
:109F7000032807DA6F4803F04BFE6FA003F048FE9A
:109F800079A023E07FA16868FEF799F9002810D036
:109F90000020AE680246009069463046FEF7A4FBFA
:109FA00004460098B04202D0007800287BD077A009
:109FB0000CE000240226B00014902858FEF778F92F
:109FC0000746E019801C502804D975A003F020FE34
:109FD00017B0F0BD002C03D0202069460855641C42
:109FE00014983A46295868460019FEF73DF9159825
:109FF000E419761C8642DEDB002069460855451EC2
:10A000006E462C4605F02EFB304603F059FC060048
:10A0100023D003F03AFC00281FD069A1304603F09A
:10A02000FDFB074603F028FC002800D07D6965A1F0
:10A03000304603F0F3FB074603F01EFC002800D077
:10A040007C69002D13DA002C22DA5FA003F0E0FD1A
:10A05000304603F0B9FB17B0F0BD65A003F0D8FDA2
:10A06000002EF8D0304603F0AFFB17B0F0BD294604
:10A0700066483239814209D3654A322165A003F02E
:10A0800061FD304603F0A0FB17B0F0BD002C0BDBE8
:10A09000642C09DD642164A003F054FD304603F014
:10A0A00093FB17B0F0BD14E0304603F08DFB002D9C
:10A0B00001DB62480581002C01DB6048C46006F0CA
:10A0C00017FF002801D05EA080E706F0BDFE17B0A4
:10A0D000F0BD3BA16868FEF7F2F8002807D039A16F
:10A0E0006868FEF7ECF800280DD05CA06EE720460B
:10A0F00046493238884203D3454A322145A015E00B
:10A100004E48048109E0642C05D9642146A003F07F
:10A1100019FD17B0F0BD4948C46006F0E9FE0028FB
:10A1200001D055A052E7224659A0696803F00AFD04
:10A1300017B0F0BDB04C010120206C6564203D20BB
:10A140006C65643120626C696E6B2068616C66209E
:10A15000706572696F642035302E2E3130303030AA
:10A16000206D730D0A000000202070776D203D20C7
:10A1700070776D206475747920302E2E3130302048
:10A18000250D0A006A736F6E000000006170707325
:10A1900065743A206261642076616C75650D0A0011
:10A1A000617070736574206A736F6E3A206C696EAB
:10A1B0006520746F6F206C6F6E670D0A00000000E1
:10A1C0006C65640070776D00617070736574206AEF
:10A1D000736F6E3A206E6F206B6E6F776E206B65BB
:10A1E0007920286C65642C2070776D290D0A000099
:10A1F000617070736574206A736F6E3A207061725B
:10A200007365206661696C0D0A000000DF2600009E
:10A21000102700006C65642072616E6765202575EB
:10A220002E2E25750D0A000070776D2072616E6705
:10A230006520302E2E25750D0A000000AC5C002034
:10A24000617070736574206A736F6E3A20666C611A
:10A250007368206661696C0D0A000000756E6B6E94
:10A260006F776E20706172616D20286C65642C20A0
:10A2700070776D290D0A00006170707365743A2063
:10A28000666C617368206661696C0D0A00000000ED
:10A290002573203D20256C752C2073617665640D37
:10A2A0000A000000002498B0F4A725461594661E05
:10A2B00038461294FDF7FCFF81B2384603F0C2F92C
:10A2C0000027FF433946684603F01CF90028F7D001
:10A2D0001598002805D0002115916946097881421A
:10A2E000EED0129801281FD0022826D068460078A8
:10A2F0001B287DD009287CD00D287BD00A287AD055
:10A30000082879D07F2877D0014620395F29D7D215
:10A310003F2C72D2E5490855641CA4B2012168465D
:10A3200003F090F92546CBE7684600785B2802D019
:10A3300000201290C4E70220FBE70020129068463C
:10A340000078412816D04228BAD1002EB8DB761EFC
:10A3500057D4D7484078801BC01DC117490F091832
:10A36000C908C900401A8101D24809184038FDF7D0
:10A37000CBFF49E0CE48711C02789142A0DA4078C8
:10A38000761C801BC01DC117490F0918C908C900D8
:10A39000401A8101C74809184038FDF7B5FFC34886
:10A3A0000290FDF785FF87B2C3A42046FDF780FF2A
:10A3B00081B2204603F046F90024002D0BD9C1A03C
:10A3C0000190FDF775FF81B2019803F03BF9641C21
:10A3D000A4B2AC42F3D3B8A42046FDF769FF81B222
:10A3E000204603F02FF9002F34D03946029805E0BB
:10A3F00036E038E0E2E0E3E029E136E103F022F97B
:10A4000028E0AA4900200870A8480290FDF750FFF4
:10A4100087B2A9A42046FDF74BFF81B2204603F086
:10A4200011F90024002D0BD9A6A00190FDF740FFE3
:10A4300081B2019803F006F9641CA4B2AC42F3D3D4
:10A440009DA42046FDF734FF81B2204603F0FAF8C0
:10A45000002FCAD13D469548FDF72AFF84B22FE769
:10A46000012012902CE703F0CBF8904800252F46EE
:10A47000019003F0FEFA1390224620210198FDF787
:10A480002CFF002860D101990855139914900029D8
:10A490005AD9149803F0F0FA224616900199FDF764
:10A4A0003CFF002819D1002F0AD102A81699FDF708
:10A4B0002BFF02A8FDF7FCFE85B20DE06D1EADB2CC
:10A4C000A54206D92A4602A81699FDF726FF0028BC
:10A4D000F4D1002002A948557F1C14981399401C00
:10A4E00014908842D5D3002F64D0012F1AD0A542F2
:10A4F0002BD902AF3F2C5DD2AC425BD2381901217F
:10A5000003F0A0F80198395D0155641CA4B2F1E78D
:10A510003819012103F096F80198395D0155641C42
:10A52000A4B200E002AF3F2C44D2AC42F0D3019879
:10A5300020210155641C63A5A4B22846FDF7B8FE8E
:10A5400081B2284603F07EF834E05FA52846FDF787
:10A55000AFFE81B2284603F075F813980025002855
:10A560001CD9284603F088FA074622460199FDF7D0
:10A57000D4FE00280ED13846FDF79AFE81B2384647
:10A5800003F060F851A73846FDF792FE81B23846D5
:10A5900003F058F813986D1C8542E2D34AA528466B
:10A5A000FDF786FE81B2284603F04CF8214601985B
:10A5B00003F0DEFA254603F033F881E60A2000E0D6
:10A5C0000D20159003F01CF83FA52846FDF770FEFE
:10A5D00081B2284603F036F83449002008550D466C
:10A5E000287800281FD0324C207800280AD06078C4
:10A5F000C01D4007C10D2F4808182946FDF75FFE12
:10A60000002810D0607881012A4808182946FDF7F3
:10A610007BFE6078401C4007400F6070207808285F
:10A6200001D2401C2070002003F0ECFA1F4803F018
:10A630002FFA1CA42046FDF73BFE81B2204603F012
:10A6400001F802F0EDFF002425463E4638E6002CD6
:10A65000B3D0641E1EA5A4B22846FDF729FE81B220
:10A66000284602F0EFFF25462AE61AA73846FDF7EE
:10A670001FFE81B2384602F0E5FF21E60D0A434C89
:10A68000492072656164792E2054797065202768AD
:10A69000656C702720666F7220636F6D6D616E64EC
:10A6A000732E0D0A63616969632D3E00C05000205E
:10A6B00044470020005100200D63616969632D3E0D
:10A6C00000000000200000000D0A00002020000013
:10A6D000082008000700000010B50C46022812DB15
:10A6E0000EA16068FDF7EBFD002809D00CA16068A1
:10A6F000FDF7E5FD002804D00AA003F089FA10BD9B
:10A70000012001F06BFF01F063FF002801D003A1DD
:10A7100000E003A10AA003F015FA10BD6F6E00005F
:10A720006F66660075736167653A20626C656C6F71
:10A7300067205B6F6E7C6F66665D0D0A000000002F
:10A74000626C65206C6F673A2025730D0A0000006B
:10A75000F8B502F0CFF9074602F0C8F90546254AD8
:10A7600025A128A003F0EEF902F0F2F901462CA091
:10A7700003F0E8F92F48874203D12FA003F048FAED
:10A7800015E000F02DFF044602F014FA06460A21F7
:10A790003846FDF70DFD0A460146002C01D0A069A0
:10A7A00000E00020009033462BA003F0CBF902F02C
:10A7B0001DFA014632A003F0C5F93548854203D1A0
:10A7C00034A003F025FA03E029463AA003F0BAF9D1
:10A7D00009F08CF87D21C900FDF7D4FC014639A0B1
:10A7E00003F0B0F908F07CFC01463AA003F0AAF9A6
:10A7F000F8BD00001100010056312E30302E3137E7
:10A80000000000006669726D776172653A202573F9
:10A81000202830782530386C58290D0A00000000B7
:10A820006375722062616E6B3A2041505025750D40
:10A830000A000000FF7F0000636869702074656D86
:10A84000703A2041444320726561642074696D65EB
:10A850006F75740D0A000000636869702074656D7F
:10A86000703A2025642E2564204320286164633DCE
:10A870002575207472696D3D256C75290D0A0000DF
:10A880007664643A202575206D560D0A000000009C
:10A89000FFFF000066616E2072706D3A206E2F61BE
:10A8A00020286E6F20746163686F6D65746572290E
:10A8B0000D0A000066616E2072706D3A2025750DDC
:10A8C0000A000000757074696D653A20256C75206A
:10A8D000730D0A006672656520686561703A20250F
:10A8E0007520420D0A00000002F0C6FA00280DD0C3
:10A8F00007A003F08DF9C82008F0B6FABFF34F8F18
:10A9000011491048C860BFF34F8FFEE70FA0F0E772
:10A91000666163746F72793A20666C617368207740
:10A9200072697465206661696C65642C2072657358
:10A93000657474696E6720616E797761792E2E2E49
:10A940000D0A00000400FA0500ED00E06661637482
:10A950006F72792064656661756C747320726573BB
:10A96000746F7265642C20726573657474696E67A8
:10A970002E2E2E0D0A00000070B5194D0E4602282D
:10A9800019DB00240C20604329587068FDF797FC00
:10A99000002807D0641C0F2CF4D312A0716803F0B8
:10A9A000D1F870BD0C20444360194268295916A0A3
:10A9B00003F0C8F870BD17A003F02AF90024204660
:10A9C0000C21484341194A6829580FA003F0BAF8EE
:10A9D000641C0F2CF3D312A003F01AF970BD000011
:10A9E0001C480101756E6B6E6F776E20636F6D6D25
:10A9F000616E643A20257320287472792027686577
:10AA00006C7027290D0A00002020252D3873202581
:10AA1000730D0A00636F6D6D616E64733A0D0A0009
:10AA20006B6579733A20544142203D20636F6D700D
:10AA30006C6574652C2055502F444F574E203D2097
:10AA4000686973746F72790D0A00000070B50C4666
:10AA5000032823DB60680178312902D0322906D02F
:10AA60001CE04078002819D1184E012504E04078F8
:10AA7000002813D1164E402516A1A068FDF71FFC33
:10AA800000280FD014A1A068FDF719FC00280ED0F3
:10AA900012A1A068FDF713FC00280DD011A003F04F
:10AAA000B7F870BD2946304600F050FB08E0294653
:10AAB000304600F047FB03E02946304600F018FB23
:10AAC00011A0A268616803F03DF870BD000C014060
:10AAD000000801406F6E00006F666600746F676764
:10AAE0006C65000075736167653A206C6564203C95
:10AAF000317C323E203C6F6E7C6F66667C746F6783
:10AB0000676C653E0D0A00006C6564202573202586
:10AB10007320646F6E650D0A0000000006A003F04C
:10AB200077F8C82008F0A0F9BFF34F8F074906480F
:10AB3000C860BFF34F8FFEE7726573657474696E0A
:10AB4000672E2E2E0D0A00000400FA0500ED00E02D
:10AB500010B508F0CBFE7D210446C900FDF712FBBD
:10AB60000246214610A002F0EDFF08F0AFF80146C2
:10AB700014A002F0E7FF08F0B9FA044608F0B0FAB2
:10AB8000024605212346090311A002F0DBFF1DA0A8
:10AB900003F03EF8274900200870084608F084F9C1
:10ABA000244803F035F810BD757074696D653A205E
:10ABB000256C75207469636B732028256C75207370
:10ABC000290D0A007461736B733A2025750D0A0014
:10ABD000686561703A20746F74616C20257520423D
:10ABE0002C206672656520257520422C206D696ECB
:10ABF0002065766572206672656520257520420D98
:10AC00000A0000006E616D65202020202020202099
:10AC10002020202020737461746520207072696F79
:10AC20002020737461636B28772920206E756D0D69
:10AC30000A000000E04E002010B506A002F0E8FF78
:10AC4000E12149020BA002F07DFF16A002F0E0FF17
:10AC500010BD00007573617274313A2054583D5034
:10AC600042362052583D5042372028414634290D63
:10AC70000A000000626175643A20256C752C20384A
:10AC8000206461746120626974732C206E6F20707F
:10AC900061726974792C20312073746F702062693D
:10ACA000740D0A00666C6F7720636F6E74726F6C40
:10ACB0003A206E6F6E653B2074783A20444D4120F7
:10ACC0004348312028706F6C6C6564293B20727892
:10ACD0003A205258444E452069727120717565754D
:10ACE000650D0A0010B5E1246402204602F050FC14
:10ACF000214602A002F026FF10BD000075736172AC
:10AD0000742072657365743A20256C7520384E3155
:10AD10002C20727820717565756520666C75736876
:10AD200065640D0A0000000010B506A108A002F03D
:10AD300009FF0DA002F06CFF1948016819A002F08C
:10AD400001FF10BD56312E30302E3137000000008B
:10AD50006669726D776172652076657273696F6E70
:10AD60003A2025730D0A00006D636D2D6464632D18
:10AD7000626C653A20424C452872647473732920D2
:10AD80002B204672656552544F53202B205541525B
:10AD90005428444D4129202B20434C490D0A0000E2
:10ADA0000040002053797374656D436F7265436C86
:10ADB0006F636B203D20256C7520487A0D0A0000DA
:10ADC0004860704701681A4A114001600021016023
:10ADD00041608160C160174A1749904204D14868B8
:10ADE0000F22104348607047144A904204D14868CB
:10ADF000F022104348607047114A904205D14868DC
:10AE00000F2212021043486070470E4A904205D14B
:10AE100048680F2212031043486070470A4A904264
:10AE2000FBD148680F2212041043486070470000AD
:10AE3000FEFF000008000240000002401C0002402B
:10AE400030000240440002405800024000290168DE
:10AE500002D00122114301E0014A11400160704714
:10AE6000FEFF0000024609680020114200D00120C8
:10AE70007047000030B403680D4A0C6A13408A68BA
:10AE80004D6922430C692C4322438C692243CC69CF
:10AE900022434C6A22438C6A22431A430260CA68E6
:10AEA00042600A6882604968C16030BC7047000037
:10AEB0000F80FFFF002B01D0106170470020106150
:10AEC00070470000014948617047000000040140DC
:10AED000054B002219685B690140034202D000293A
:10AEE00000D00122104670470004014010B483795D
:10AEF00019490268002B28D00B6893430B604A68FD
:10AF000003689A434A60027952181368046823431D
:10AF100013608A6803689A438A60CA6803689A4320
:10AF2000CA604279102A06D051180A6800680243A4
:10AF30000A6010BC70478A6803681A438A60CA684E
:10AF400000680243CA6010BC70470079401801686D
:10AF50009143016010BC7047000401400B6800225F
:10AF6000002B56D0F0B401240B68944023424AD001
:10AF70004B68022B01D0122B16D113070AD5456A54
:10AF80005307DB0E0F269E40B5434E699E402E436D
:10AF9000466209E0056A5307DB0E0F269E40B54363
:10AFA0004E699E402E4306624B68012B05D0112B43
:10AFB00003D0022B01D0122B06D14568DB06DB0F34
:10AFC000A54393402B4343600568530003279F40EC
:10AFD0000E79BD43B607B60F9E402E430660C56886
:10AFE0008E68BD439E402E43C66085680126A543FA
:10AFF000CC6894402C438460C46A9E400D69B4437D
:10B000009D402543C5620B68521CD340ABD1F0BCB8
:10B010007047704705490160002242600F2182603D
:10B02000416101210261C16070470000FF3F0000E3
:10B03000816270478161704742694A40426170474E
:10B0400082B0EFF30884FDF751F8400701D5EFF324
:10B0500009840AA000F084FBE06800900CA0A368BB
:10B060006268216800F07CFBE069009014A0A3698D
:10B070006269216900F074FBFEE700000A2A2A2AAF
:10B0800020486172644661756C74202A2A2A0A007D
:10B09000523020203D2530386C5820523120203D40
:10B0A0002530386C5820523220203D2530386C58DD
:10B0B00020523320203D2530386C580A0000000013
:10B0C000523132203D2530386C58204C5220203DE2
:10B0D0002530386C5820504320203D2530386C589E
:10B0E00020785053523D2530386C580A000000003B
:10B0F00010B5FFF7A1FF10BD30B505460E4887B06B
:10B100000C46854202D10121042004E00B4885420F
:10B1100010D10121082000F021F90948844209D802
:10B120006846FFF777FF01200190694600942846A2
:10B13000FFF714FF07B030BD00080140000C0140CC
:10B14000FF3F000010B5FFF773FF10BD10B5FFF70C
:10B1500071FF10BD10B400214156FF23CAB29207FF
:10B16000D40E4278A3409207120EA24000290BDAB7
:10B170000907090F08398C081049A4006118CC6927
:10B180009C431443CC6107E08C080D49A40061186E
:10B190000C689C4314430C60827801210078002ADB
:10B1A00004D0C006C00E8140064803E0C006C00EB1
:10B1B00081400548016010BC7047000000ED00E0D0
:10B1C00000E400E000E100E080E100E0F7B5FFB05E
:10B1D00004460025A5B00520EFF31087FF2100905D
:10B1E000453102A8FDF759F8EFF31086FF214531EC
:10B1F00053A8FDF752F853A8013001909822224934
:10B2000053A8FDF731F8012080F31088019880479A
:10B2100086F3108801221D491203032653003603CA
:10B2200088420AD194421AD09C4201D1151116E0ED
:10B23000B44210D101256D0211E0154988420AD1AE
:10B24000944201D115460AE09C4201D11D4606E018
:10B250003546AC4203D000987FB028B0F0BD06ACB4
:10B26000FF22013441320B4902A8FCF7FDFF012007
:10B2700080F310882846A69AA599A04787F31088DE
:10B280007FB028B0F0BD0000183D0101C44013009C
:10B2900085601300D83B010110B5EFF31084012144
:10B2A00081F31088FF21090640180349096888477F
:10B2B00084F3108810BD00000440002010B5084839
:10B2C000064901600749416007498160C92292002F
:10B2D00006490748FCF7C8FF10BD0000E148002000
:10B2E000044000207549002049480020BC3D010170
:10B2F0004048002010B5EFF31084012383F3108839
:10B30000FF231B06C018034B5B68984784F3108823
:10B3100010BD000004400020034AD16A1023994365
:10B320000143D1627047000000100240044A002926
:10B33000516901D0014300E0814351617047000031
:10B3400000100240044A0029916A01D0014300E044
:10B35000814391627047000000100240044A0029B6
:10B36000916901D0014300E0814391617047000081
:10B37000001002400122054912060128086802D087
:10B380009043086070471043FBE700000010024044
:10B3900030B4164A516804231940154B01D00429D2
:10B3A00001D0036001E0134901605168124B890626
:10B3B000890F5B5C0168D940416053680F4C5B05A5
:10B3C0005B0FE35C0D46DD40856053689B045B0FBB
:10B3D000E35CD940C160D16AC90601D5084901E0E2
:10B3E0007D21C903016130BC70470000001002409C
:10B3F0000090D0030048E801B03D0101B43D0101D7
:10B4000000093D007047000010B5FCF785FE0446BA
:10B4100008F072FA002803D00120034900074860B1
:10B420002046FCF77DFE10BD00ED00E010B50A4C93
:10B430002069411C01D000280AD10120064934228C
:10B440000003FFF7C3FE2069411C03D0002801D090
:10B45000024810BD002010BD0C48002035480020D7
:10B46000F0B5564C85B0E06921040843E0618120C5
:10B47000534D000628635348686153482862534877
:10B4800003220168920391430160514934228014E0
:10B49000FFF79CFE4E4B4F4E18694F4F411C29D071
:10B4A000002827D0A9691A7849094901D206D20E85
:10B4B0000A43AA612168EA139143216021687F222F
:10B4C00012029143000208432060606830436060CC
:10B4D0006068B84360606068211508436060206A56
:10B4E0003E4908402062206AD96809020843206268
:10B4F00005B0F0BD61682046314361606168B943C1
:10B50000616061680127BF023943616000210491D5
:10B510007D21C9000391002100917F214024002555
:10B5200002950191026861028A4302600E1123496B
:10B5300008687F2212029043220202430A6005201B
:10B54000FCF7CCFD0120FCF7C9FD1C48406B8007CF
:10B5500004D4284603996D1C8842F3D91748C06B60
:10B5600080B2B04201D9811B00E0311AB94202D247
:10B57000E2B28FB20292B04201D3019400E0009493
:10B58000019A00988018C005000EA04203D004461E
:10B5900004988142CBD8094801687F221202914366
:10B5A000029A12020A430260416849084900416058
:10B5B00041684907FCD405B0F0BD0000001002400E
:10B5C000007000400F080000180002000010014049
:10B5D0000C4800200000010000070000FF00F8FFF9
:10B5E00010B50A4C2069411C01D000280AD1012065
:10B5F000064934220003FFF7E9FD2069411C03D00E
:10B60000002801D0014810BD002010BD0C480020CA
:10B6100010B501F093FF10BD10B40B06CC065B0F04
:10B62000E40E0121A140012B07D0022B07D01430DA
:10B63000002A026805D00A4304E00C30F8E7103015
:10B64000F6E78A43026010BC704700000029818938
:10B6500003D001225203114301E0024A11408181CB
:10B6600070470000FFDF0000002A828A01D00A43F1
:10B6700000E08A43828270470246128800200A4214
:10B6800000D00120704770B40A06530FCE06012582
:10B69000F60E2A460024B240012B0FD0022B10D008
:10B6A000838A1340090A00888D402840002B02D06D
:10B6B000002800D00124204670BC704783891340C5
:10B6C000F0E7038AEDE7000070B50446008A86B013
:10B6D0000D461B490840E98801432182A089194988
:10B6E0002A890840A98811436A8902431143A1812C
:10B6F000A08A15490840A9890143A1826846FFF73D
:10B7000047FE1248844201D1039800E0029829685C
:10B71000192289005043FCF735FD06466421FCF7E9
:10B7200031FD0501280964214843301A00013230F7
:10B73000FCF728FD0007000F2843208106B070BDEC
:10B74000FFCF0000F3E90000FFFC000000380140DB
:10B750008088C005C00D7047C905C90D818070473C
:10B760000FB410B503A9044B044A029800F066F91F
:10B7700010BC08BC04B0184705E10001C40100205A
:10B780000FB410B504A9074B02AA039800F056F9AC
:10B79000044602A9002000F0F8FC204610BC08BCBA
:10B7A00004B018478BC100017CB515460246002045
:10B7B0001C4600290BD0491E00920191044B6A4699
:10B7C0002146284600F03AF9009A002111707CBD0C
:10B7D00075C100012021020C01D010211046020A7F
:10B7E00001D010460839020901D01046091F82080D
:10B7F00001D01046891E420801D0881E7047081AE1
:10B8000070470000004870470848002030B5002805
:10B8100005D0164C021F20680023014605E00846AB
:10B8200030BD904203D8034640680028F9D1002B70
:10B8300000D05968002B0AD01C68D51AA54204D143
:10B840001268A4181A461C6002E05A6000E02260E8
:10B85000002807D01468851AA54203D10568641929
:10B86000146040685060184630BD00000048002059
:10B87000F1B50E4C0F480C4E001B0D4FC508ED00E6
:10B8800000221146009803F005FF002803D130681C
:10B89000002801D00020F8BD3C60002025606060D9
:10B8A00001203060ECE7000004480020D4AD002007
:10B8B00000480020D0AF0020F0B51FB486B0099832
:10B8C000089A030D0021024314D05148514A181818
:10B8D000504305141198012810981AD0281A401CBA
:10B8E00000264D4F4D49009601910490002812DA30
:10B8F000444211E01198012449A3012801D1109874
:10B90000C1430698119A84600360C26041600BB025
:10B91000F0BD4042E4E70446210500203F4A001CF8
:10B9200051410391029012E0E00707D032463B46B6
:10B9300001990098FDF75CF80191009032463B4672
:10B9400010461946FDF754F806460F466410002CC1
:10B95000EAD10498039B0028029A0999089806DA0C
:10B96000FDF746F8019B009AFDF742F805E0FDF768
:10B97000A7F8019B009AFDF7A3F804460E460022A3
:10B98000284BFDF7E9F903D80020C043014607E042
:10B990000022254B20463146FCF778FFFDF794F94D
:10B9A000102409E0002C0ADB0A220023FCF714FC17
:10B9B000079B30321A55641E02460A43F2D1112207
:10B9C000641C079B121B1C19119B012B03D0012324
:10B9D00008430ED10AE0084304D011201090002043
:10B9E000119077E71098151A6D1E0BE0109882429F
:10B9F00002DD00236D1C03E0824201DA00236D1E8C
:10BA0000002BEED0069811998260C16030C07EE7AD
:10BA100001FCFFFF104D0000000014400000F03F4B
:10BA2000300000000000F0430000E03F30380A28FA
:10BA300001D201207047002070470000FFB597B089
:10BA40000646002518E2252877D100242746FD491F
:10BA5000049400E00443761C32780120203A9040A0
:10BA60000842F7D130782A280ED0022230780146D9
:10BA70003039092916D804990A2359433039401816
:10BA80001443761C0490F1E7189802C804911890AA
:10BA9000002904DA012040030443484204900220B4
:10BAA0000443761C30782E2814D104200443707887
:10BAB000761C2A2809D11898761C80C8189009E0AD
:10BAC0000A214F43303FC719761C30780146303980
:10BAD0000929F5D930786C2810D006DC4C281AD00A
:10BAE00068280ED06A2817D104E0742813D07A2869
:10BAF00012D110E00120400504430CE001210905AA
:10BB000001E0032109050C437178814203D1012032
:10BB100000052418761C761C3078119066280BD00E
:10BB200013DC58287DD009DC00287BD04528F6D0CE
:10BB30004628F4D047281AD1A5E118E0632835D06B
:10BB4000642870D0652812D19DE170286CD008DC83
:10BB50006728F1D069287BD06E280DD06F2806D1D8
:10BB6000BAE073282ED0752871D0782859D01A9A47
:10BB7000199990476D1C7EE16002400F022809D0A0
:10BB800003280DD00428189801680DD00D60001D01
:10BB9000189070E11898EA1701680D604A60F6E79E
:10BBA000189801680D80F2E70D70F0E718986A4662
:10BBB00001781172001D18900020507202A80090A8
:10BBC000012005E0189802C8189000200091C04399
:10BBD00061070DD5002101E00199491C0191B9428D
:10BBE00012DA8142F8DB009A515C0029F4D10BE0B3
:10BBF000002101E00199491C01918142FADB019A7F
:10BC00000099895C0029F5D1019904981A9B471A7B
:10BC100021463846199A00F097FA019940194518BB
:10BC20000BE04FE02CE113E04EE000980099007823
:10BC3000491C00911A9A199990470198401E019049
:10BC4000401CF2D1214638461A9B199A10E137E080
:10BC50000A200021009001916002410F022907D0C3
:10BC6000189A01CA1892C2179446032908D00AE00C
:10BC70001898C01DC108C90005C91891944607E06D
:10BC800000B2C2179446042902D140B2C1178C46B3
:10BC900000226146944506DA0A460021404291415D
:10BCA0008C462D2102E0210504D52B216A46117313
:10BCB000012103E0E10701D02021F7E7029155E0DF
:10BCC0000A200AE0102008E0102000900021042043
:10BCD00004430191082703E008200021019100900E
:10BCE0006002410F022907D0189A01CA1892002257
:10BCF0009446032908D008E01898C01DC108C9005F
:10BD000005C91891944603E080B2042900D1C0B25D
:10BD100000210291210729D51199702906D0009A96
:10BD20001021019B4A401A4305D00EE040216A468B
:10BD30001173012108E06146014306D030216A46B3
:10BD400011731199517302210291009A0821019BEC
:10BD50004A401A430AD16146014301D1610705D522
:10BD600030216A46117301217F1E029111995829D1
:10BD700004D035A10E910DA90D910DE037A1F9E781
:10BD80006146019B009AFCF727FA0E9B8C469B5C50
:10BD90000D9A521E0D92137061460143F0D10D9819
:10BDA00005A9081A20300190600703D5012000047E
:10BDB000844300E001270198874201DD381A00E042
:10BDC0000020019900904118029809180498401A1F
:10BDD0000490E00306D421461A9B199A049800F0B7
:10BDE000B3F94519002706E003A81A9AC05D19990E
:10BDF00090476D1C7F1C02988742F5DBE0030CD551
:10BE000021461A9B199A049800F09EF9451904E0FE
:10BE10001A9A3020199990476D1C0099481E00907D
:10BE20000029F5DC08E00D980D990078491C0D916A
:10BE30001A9A199990476D1C0199481E0190002982
:10BE4000F1DC63E109280100303132333435363713
:10BE50003839616263646566000000003031323356
:10BE600034353637383941424344454600000000F6
:10BE700000F05AF94519761C3078002800D0E2E528
:10BE800028461BB0F0BD600700D406271898C01DD7
:10BE9000C108C90048680A680831C30FDB07189158
:10BEA000190001D09CA108E0210501D59BA104E067
:10BEB000E10701D09AA100E09AA1430011985B0824
:10BEC000109165280CD006DC452809D046281DD0E5
:10BED000472841D141E0662818D067283CD13CE092
:10BEE0000021112F01DB112000E0781C019100904E
:10BEF00008A911A8FFF7E0FC139905910021119AF8
:10BF000015927F1C12980197009150E00120C00704
:10BF100003900120019008A9009711A8FFF7CCFC1D
:10BF2000139A149905920022119B0092129815936E
:10BF3000059A0192002901D0104602E0791C4018B0
:10BF40000190381A01D5019804E04042401E00904B
:10BF5000781C0190C01B029043E0012F00DA0127FA
:10BF60000021112F01DD112000E0384601910090E1
:10BF700008A911A8FFF7A0FC13990591119A0021B7
:10BF8000129815920091019721070CD40599B94296
:10BF900001DB019900E00191012904DD159A491E98
:10BFA000515C302906D0B84201DA011D05DA0121C1
:10BFB000029115E00199491EEDE7002805DC009982
:10BFC000411800910199091A03E0019A411C91421C
:10BFD00000DD01910099401A401C02900120C00729
:10BFE0000390200706D402990198814202DB0020C9
:10BFF000C043029000206946C87707AF012103982B
:10C000000337C907884224D0022011902B201290B8
:10C01000039800280CDA404203902D20129007E08C
:10C020000A210398FCF7AEF830317F1E0390397077
:10C030001199481E11900029F2DC03980028EFD1D5
:10C04000791E129808703078202108404530BF1EB4
:10C05000387006A8C01BC01D0390109800780028F7
:10C0600000D00120019941180298C01709180398BF
:10C0700009180498401A401E0490E00306D4214693
:10C080001A9B199A049800F05FF8451910980078E7
:10C09000002803D01A9A199990476D1CE00324D503
:10C0A00021461A9B199A049800F04EF845191CE095
:10C0B0000098002807DB00990598884203DD159851
:10C0C000405C199901E0199930201A9A904700981C
:10C0D0006D1C401C00900298401E0290002804D164
:10C0E0001A9A2E20199990476D1C0199481E0190AB
:10C0F0000029DDDC05E038781A9A7F1C19999047F1
:10C100006D1C0399481E03900029F4DC21461A9BFC
:10C11000199A0498ACE600002D0000002B000000E6
:10C120002000000000000000F8B5044600251E466F
:10C130001746880404D405E039462020B0476D1C1A
:10C14000641EF9D52846F8BDFFB50446002581B028
:10C150001E46C80301D5302700E02027880404D5F7
:10C1600005E038460399B0476D1C641EF9D5284692
:10C1700005B0F0BD4A68002A06D00A68531C0B605F
:10C1800010704868401E486070470A68531C0B6076
:10C1900010707047002903D0002801D0884201D1D7
:10C1A000002070478268002A08D05268002A03D015
:10C1B00011604A6080684160012070478160496079
:10C1C00000200860F8E7FFB581B007000A98144620
:10C1D0000D4605D0002D03D0002C01D0A74202D17E
:10C1E000002005B0F0BD01267602002802D0E068EC
:10C1F000304307E02846049901F0F8FB051EF0D013
:10C20000E068B0430646A089800505D4206A00286E
:10C2100002D0049949688847E6602146384625627D
:10C22000FFF7B8FF05B0F0BD00B599B060216846D2
:10C23000FCF733F8042008AAD07012A0006801901F
:10C240000B2010AAD070024610A109A8FCF70CF828
:10C25000002010AA107101215171D0719171907359
:10C260001175D082A02010839176B420908319207C
:10C27000C001D08308480090684603F0EBFC19B079
:10C2800000BD000003160A18000000000AFFFFFFAF
:10C290004E6174696F6E73009DC2000170470000AB
:10C2A00010B540210848FEF751FF084900200870EA
:10C2B00000F08EF9002802D005A0FFF751FAF72010
:10C2C00003F03CFE10BD000000080140374700208D
:10C2D0005B424C455D20636F6E6E65637465640DF3
:10C2E0000A00000010B503F0D9FC00F07FF94021EE
:10C2F0000648FEF727FF06490020087000F068F99D
:10C30000002802D003A0FFF72BFA10BD000801405F
:10C31000374700205B424C455D20646973636F6E54
:10C320006E65637465642C206164766572746973EC
:10C33000696E67207265737461727465640D0A00BA
:10C3400010B58CB0002400940194029403940494DA
:10C35000059406940794089409940A94FFF766F8E4
:10C36000002804D0014601A8FDF712F907E012A049
:10C3700001886A4691804188D18080881081694611
:10C38000CC704C810A20887012220A7303A80CA179
:10C390000130FBF769FF0C206946088418204884A7
:10C3A000FF208C84F530C8840A480885684603F06D
:10C3B00013FD0CB010BD00000102030405060000CF
:10C3C00043414949432D4D434D2D323032363039AA
:10C3D000303200008813000000B583B00D49009191
:10C3E0000D4900200191029069460872684603F0E9
:10C3F000F7FDFFF7A5FF00F033FAFFF715FF074839
:10C4000003F094FB064803F091FB03F047FC03B0F4
:10C4100000BD000025C40001BDD000018DC9000190
:10C42000A5CE00010178012928D070B50025144E51
:10C43000144C022912D003290FD103F02FFC00F075
:10C44000D5F840213046FEF77DFE257000F0C0F89B
:10C45000002802D00C48FFF783F970BD4021304618
:10C46000FEF774FE257000F0B3F8002802D00748EC
:10C47000FFF776F9F72003F061FD70BD704700000B
:10C48000000801403747002014C30001D0C200015A
:10C49000F8B50646244F0020388178810124481ED3
:10C4A0000D463E2814D80A4631462048FBF7DCFEEC
:10C4B0001E49002048551E4801F0A4FB1B4801F00E
:10C4C000E7FA0446002001F09DFB388900280CD1D2
:10C4D000002C12D017A00090FBF7EAFE84B222468F
:10C4E00019480099FBF7C0FE3C81B878002819D0A4
:10C4F00016A0FFF735F900240CE019A0EBE7315D39
:10C50000084620385F2800D32E2117A0FFF728F90E
:10C51000641CA4B2AC4201D23F2CF0D3398913A0E1
:10C52000FFF71EF9F8BD00004C4700200055002021
:10C53000D9DB0001756E6B6E6F776E20636F6D6D6A
:10C54000616E640D0A0000007B5800205B424C4580
:10C550005D20636C6920657865633A2022000000E5
:10C560006F6B0D0A000000002563000022202D3EA5
:10C5700020257542207273700D0A000030B40C49FA
:10C58000098E182902D3891E8AB200E01422094CB0
:10C59000094D63892189ED18C91A89B2914200D9E0
:10C5A00011465A1862810180284630BC704700004D
:10C5B000B04D00204C4700207B580020034800214C
:10C5C00001708180C1804170704700004C4700209D
:10C5D00001488078704700004C470020002800D0B8
:10C5E00001200149887070474C47002010B505496B
:10C5F000002008708880488100F000FE00F06AFB8F
:10C6000010BD00004C470020F3B583B0049800240F
:10C6100000287AD95B4802905B4A03981178005D44
:10C62000002904D001290BD002291AD122E0CA28FE
:10C630006CD156490870012090800521D18017E007
:10C64000524B91885854491C88B2908005285DD17E
:10C650000298417803780802FF211843E1318842AB
:10C6600003D900201070908084E0C01DD08002208B
:10C6700010707FE0444A454B91885854491C88B259
:10C680009080D188884275D1029800224178007844
:10C690000D0205433E488446E81C86B23D48002E04
:10C6A00014D93D4F6146895C0902484000210304CA
:10C6B00002D54000784000E04000491CC9B280B279
:10C6C0000829F4D3521C92B2B242EBD32F4E711907
:10C6D0008A794B7911021943884247D17778B0782B
:10C6E00001902948761D8078002806D033460095B1
:10C6F00039462AA0019A05F087FB112F2AD006DCC3
:10C70000012F09D0102F31D124E039E032E0122F6F
:10C7100020D0202F2AD124E001273F2D11D82A46EE
:10C7200031461F48FBF7A0FD1D49002048551D4814
:10C7300001F068FA1A4801F0ABF90746002001F051
:10C7400061FA6846077001236A460320019900F0E8
:10C750002BF80BE02B4632463846019900F0CAFA16
:10C7600004E02A463146019800F0FEF9064800210F
:10C7700001708180641C0498A4B2844200D24BE70B
:10C7800005B0F0BD835500204C47002080550020A7
:10C7900081550020FFFF00002110000052580000CA
:10C7A00040550020D11D0101FFB5D81D80B283B0D6
:10C7B0001D460190FB2803D90020C04307B0F0BDFF
:10C7C000214CCA202070039860700498A070280A39
:10C7D000E5702071002D04D02A46601D0599FBF7F5
:10C7E00043FDE81C83B2194F19480024002B13D9CC
:10C7F000184E395D090248400021020402D540006C
:10C80000704000E04000491CC9B280B20829F4D34E
:10C81000641CA4B29C42ECD30B4949194871000A2C
:10C8200088710D488078002806D000950BA0059BE4
:10C83000049A039905F0E8FA0348019900F0E6FC30
:10C84000002007B0F0BD0000805700208157002075
:10C85000FFFF0000211000004C470020545800004A
:10C8600000B587B0002001900090039004906A46C4
:10C87000069010730C4902910521917003231370E7
:10C880001023D37050701071012353719071507345
:10C89000064805907D20917300011082104604F037
:10C8A00065F807B000BD000040E2010000B00301E0
:10C8B00010B5024803F002FE002010BD544E0020C7
:10C8C0002F48007900285AD1F8B56D202C23032277
:10C8D000072140010BF430D1A02104460170294802
:10C8E0000027C178617027710321E18067720126FA
:10C8F00066710721244D2177A9796177687B00282B
:10C9000003D0E780032060710EE0E87900280BD0A7
:10C91000A879022800D166772671E6802046A97999
:10C92000203041708670077015488079022804D045
:10C93000032815D004281BD116E004F009F80028BC
:10C940000BD00520E0806771688A6061688AA06109
:10C9500020460A3003F02AFE0AE0094903208871C4
:10C96000288B6061288B02E0E88B6061E88BA06116
:10C9700003480671467120460BF41AD1F8BD704782
:10C98000B04D0020344E0020A04E002010B584B0E1
:10C990000A230322072110480BF4CED01B2101707B
:10C9A000002141701424448003228280C1800B4AFC
:10C9B00002810BF4FDD06846048009480190684666
:10C9C00003F0D6FA684604810648039002A804F0F2
:10C9D00071FE04B010BD00001B0D0000FF0100003F
:10C9E000F0460101D1DD0001FFB585B0054602A882
:10C9F00000901C462846069904F002F86846007A22
:10CA0000002866D006980090280A334A01940390C3
:10CA10000E2826D0314800240178002951D92F480A
:10CA2000E1000818828803998A4240D1009A8168FF
:10CA30009646019A284694460A791206120E36D076
:10CA40000968254BD700083FCE1937887668BFB2F2
:10CA5000874201D09F4226D1634603227146B047E8
:10CA600025E01F49681809282BD800981D498446DD
:10CA700008792E4600062346000E1ED0C4000F681B
:10CA8000083C3C1927886468BFB2B74201D097427E
:10CA900004D1032261462846A0470EE0401E00064E
:10CAA000000EEBD109E0521E1206120ECAD10B483D
:10CAB000641C0078E4B2A042B1D86846007A00282D
:10CAC00007D00948426C002A02D0284606999047B0
:10CAD000002009B0F0BD0000FFFF00005C4D002009
:10CAE000EEF1FFFF40420101B04D002000487047C9
:10CAF000FFFF000070B5124D01212846FCF78EFEA5
:10CB0000142006F0B1F9702002F0BCFC702002F095
:10CB1000B9FC044600212846FCF780FE0948448001
:10CB20000948844201D1401070BD2046FCF7ACFD9D
:10CB30000649FBF76DFEFCF789F800B270BD0000F6
:10CB40000008024084470020FFFF00000000204151
:10CB500010B500F0CBF80349884201D1022010BD86
:10CB6000012010BD00400201F0B5074600208DB045
:10CB700015460E46002A04D0012D04D13178FF2934
:10CB800001D10B4E07250024002D08D90146325D46
:10CB9000684602F0ADFC641CA4B2AC42F6D3034676
:10CBA0006A4639462120FFF7FFFD0DB0F0BD0000B9
:10CBB000D0480101014840887047000084470020A8
:10CBC00070B506460020074D044601462A5D06481A
:10CBD00002F08EFC641CA4B2072CF6D3308002480D
:10CBE00070BD0000D04801017B5C002010B56020C2
:10CBF00002F048FC0449884201D1002010BD6021A8
:10CC0000FCF76CFD80B210BDFFFF000010B503F013
:10CC10001BFC04480169002901D00420884700203A
:10CC200010BD0000C04E002070B5224C606B224D3C
:10CC3000C00722D0A06B21497E2209685143401AC7
:10CC40002988491E29804B21C90040181C49884267
:10CC500013D300202880206A400840002062194930
:10CC600008680204930F184A01D0904300E0104373
:10CC700008601648407F03F01FF929880120002929
:10CC8000216B07D0014321630522032110480BF4D7
:10CC900015D20DE0FF22120291432163216B052280
:10CCA000920211432163216B0143216303F09EFE35
:10CCB000002070BD00100240344700208C0000208E
:10CCC000B10400000010014000C00000104E002020
:10CCD000010F000004480021017041618161C161C0
:10CCE0000162816270470000584700200048704789
:10CCF00000800001F8B514460D46102809D011280F
:10CD000077D0122804D11A462146284603F088FF1E
:10CD1000F8BD00910C2B04D00023012210212846DD
:10CD200063E02278E1781046627809061202104327
:10CD3000A2781204104308430502E0782D0A000689
:10CD40002279054310466279E17912021043A279F3
:10CD500009061204104308430602E079360A000669
:10CD60000643082021180A7810464A781202104318
:10CD70008A78C97812041043090608430702E07A4A
:10CD80003F0A000607431E481E491F4C884202D036
:10CD9000A0420BD10C461D49281F88420DD3002309
:10CDA00003221021009804F03AF8F8BD0023022273
:10CDB0001021009804F033F8F8BD15484078002899
:10CDC00004D1FEF77BFA1249012048701048012176
:10CDD0000170002141618161C16101628162001DB8
:10CDE000F0C00B460A461021009804F018F8F8BD70
:10CDF000FFE71A462146284603F066FEF8BD00000C
:10CE0000008000010080000100400201FDBF010020
:10CE10005847002000487047AC5C0020F8B5342229
:10CE200011491248FBF720FA104C114F20680125D8
:10CE3000104EB8420BD16068012808D1204630213D
:10CE400000F0E8FD216B884201D13570F8BD342136
:10CE50000648FBF722FAFF202760F5306560208145
:10CE60000020E0603070F8BD00600001AC5C002084
:10CE70007ADA12CA8847002010B534210748FBF738
:10CE80000CFA06480649016001214160FF21F53195
:10CE900001810021C16004F02BF810BDAC5C0020C2
:10CEA0007ADA12CA10B584B014230322072112487B
:10CEB0000AF442D61B2101700021417047244480AE
:10CEC00003228280C1800D4AC2600D4A02610B229A
:10CED00002720AF46DD6684604800A4801906846DA
:10CEE00003F046F8684604810748039002A804F05E
:10CEF000E1FB04B010BD00001B0D00001047010154
:10CF000000470101F8460101BD25010100207047DD
:10CF1000F8B5184D184FE879002801D02E7B00E0B5
:10CF2000FE780322331D072114480AF405D6A921EF
:10CF3000044601701248C178617000216180E8796F
:10CF40001049002803D02A7B896C201D02E0FA7862
:10CF5000201D091DFBF788F9608802218019608077
:10CF600007480279062A00D00171417120460AF46F
:10CF70001FD6F8BDA04E0020804E0020A60D000058
:10CF8000B04D0020604E0020F8B51F262323032259
:10CF9000072128480AF4D0D50446AA20264F20703D
:10CFA000F878264D6070E8786080EA782449201D82
:10CFB000FBF75AF96288B01AC1B2201D1018214A35
:10CFC0000326032910D92B79002B0DD006701923C5
:10CFD00043705389091F1B0AC370937A8370638857
:10CFE000C9B21B1D6380001D02291AD96B79002B61
:10CFF00017D0137B891E8B4200D21946CDB2691C13
:10D000000170117BA94201D1092100E00821417082
:10D010002A460D49801CFBF727F96088AD1C401992
:10D0200060803879062800D03E717E7120460AF46F
:10D03000BFD5F8BDA60D0000B04D0020A04E0020C9
:10D04000844E0020344E0020414E002070B53A231B
:10D050000322072116480AF46FD5A421154D044672
:10D060000170E8786070A97913480022022910D075
:10D07000032913D0042916D062802271807902F02E
:10D080004BFB052028710420687120460AF490D5D6
:10D0900070BD018A642359436180EEE7C18A64232D
:10D0A00059436180E9E7818B642359436180E4E758
:10D0B000A10D0000B04D0020A04E002070470000E0
:10D0C000FFB50F4683B000210091019116466946D5
:10D0D000FCF764FA040030D10521C9026846FCF768
:10D0E00063FA002828D121496846FCF75DFA002838
:10D0F00022D11F496846FCF757FA00281CD11D4968
:10D100006846FCF751FA002816D129210902684621
:10D11000FCF74AFA00280FD117496846FCF744FA91
:10D12000002809D115496846FCF73EFA002803D1CA
:10D1300000988088C10B03D00624204607B0F0BDBC
:10D1400000050099000D0D186888B04200D2072430
:10D150002988B819884201D90D24EEE7A8193A4662
:10D16000001D0699FBF780F86F80E6E701280000B4
:10D170000328000002280000022900000329000003
:10D180001EF40ED100F00EF8012005F06DFEF7E759
:10D1900010B503490020087000F004F810BD00002D
:10D1A0004647002012480021007800281FD070B5A3
:10D1B000104D86B02878002817D1A8886C88A04226
:10D1C00013D00D4E6A4680B2A04209D0335C53544E
:10D1D000401CC005491CC00D89B2A8801429F2D397
:10D1E00001202870104605F0EDF906B070BD7047BB
:10D1F0003747002046470020005300200249002006
:10D20000488088800870704746470020F0B4844604
:10D210000D480078002814D00022002911D90B48AD
:10D220000B4D878843881C465B1CDB05DB0DBB422E
:10D2300007D06646B65C521C2E5592B243808A4295
:10D24000F0D3F0BC7047000037470020464700206D
:10D250000053002070B5134D04462878002803D1F0
:10D26000FEF72CF8012028700F4820602821204666
:10D2700000F0D0FB0D4DA0622846FEF70DF8002807
:10D280000DD12C2221462846FEF734F8002806D17D
:10D290002C2229462046FBF72AF8002800D001203E
:10D2A00070BD00008A47002011C011CA0040000173
:10D2B00010B5044600681949884208D12046282143
:10D2C00000F0A8FBA16A884201D115A200E016A2D5
:10D2D0001B491CA000F036FC21A0216800F032FCA4
:10D2E00026A0616800F02EFC2AA02369E268A168EC
:10D2F00000F028FC33A0616900F024FC37A0236A09
:10D30000E269A16900F01EFC2EA0616A00F01AFC1F
:10D310003EA0A16A00F016FC10BD000011C011CAA9
:10D3200076616C6964000000494E56414C494420C6
:10D3300028626164206D616769632F6372632900ED
:10D3400000400001626F6F7473657474696E6720CA
:10D35000402030782530386C583A2025730D0A006B
:10D3600020206D61676963202020202020203D203F
:10D3700030782530386C580D0A0000002020616399
:10D38000746976655F62616E6B203D20256C750D5A
:10D390000A000000202062616E6B313A20616464F3
:10D3A000723D30782530386C582073697A653D2598
:10D3B0006C75206372633D30782530386C580D0AE7
:10D3C00000000000202020202020202020766572F0
:10D3D0003D30782530386C580D0A000020206261FD
:10D3E0006E6B323A20616464723D30782530386C5F
:10D3F000582073697A653D256C75206372633D30F2
:10D40000782530386C580D0A000000002020637227
:10D41000633332202020202020203D20307825300A
:10D42000386C580D0A00000030B58DB0012108207D
:10D43000FDF794FF01218803FDF790FF02A8FDF797
:10D44000E9FD402002900220284D0424039002A907
:10D4500007942846FDF782FD80210794029102A9D6
:10D460002846FDF77BFDE120400208900020694638
:10D470008884C884088588850C2048851C4D08A9A7
:10D480002846FEF721F901210846FDF74FFF194C08
:10D490002046FDF797FC0123224617490220FDF79D
:10D4A00009FD012280212846FEF7DEF80022012135
:10D4B000402005F05BFE114C2060012005F044FE89
:10D4C000606001220E492846FEF7A6F81C20694636
:10D4D000087003204870012088706846FDF73AFE06
:10D4E00001212846FEF7B2F80DB030BD000C014016
:10D4F0000038014008000240000002403847002088
:10D500002505000070B505460B480468002C0ED0B8
:10D51000481C0ED008467D21C9004843FAF732FE68
:10D5200002462946204605F088FF012800D0002049
:10D5300070BD0020C043F3E73847002010B582B02B
:10D540000020104C00900E492046FEF79CF8002861
:10D5500014D02046FEF7FCF8694608710A480068B6
:10D56000002804D00A46002301A905F01FFF0098F7
:10D57000002803D0012005490007486002B010BD13
:10D5800025050000003801403847002000ED00E08C
:10D5900030B5184D85B0044640212846FEF76CF89A
:10D5A0000028F9D000212846FEF750F800206946EF
:10D5B00000948880C880088188810C204881284692
:10D5C000FEF782F80C4C2068002807D006F07EF9A0
:10D5D000022803D10021206805F0EAFD0122074955
:10D5E0002846FEF719F801212846FEF72FF805B066
:10D5F00030BD0000003801403847002025050000FC
:10D6000010B5064C6068002807D006F05FF90228C4
:10D6100003D1C11E606805F0B1FF10BD384700207E
:10D6200010B5074C6068002809D006F04FF90228B1
:10D6300005D100231A461946606805F0F0FD10BDBB
:10D640003847002000283FD000293DD0F0B51F4EBC
:10D650000C4605468BB000213046FDF7F7FB1C4F0A
:10D6600002203946FDF7ACFB1A48009010200290CA
:10D670000020802105910490032101950394090362
:10D6800006900790089009910A9069463046FDF788
:10D69000F1FB01213046FDF7D9FB39460220FDF7A9
:10D6A000E1FB0028F9D000213046FDF7CFFB3946D9
:10D6B0000220FDF785FB084C40212046FDF7DCFFEA
:10D6C0000028F9D00BB0F0BD704700000800024000
:10D6D00000000240043801400038014010B4002826
:10D6E00007D00368002B04D042688168914201D2C0
:10D6F00006E0002010BC7047491C8160002804D05F
:10D70000914202D25C5C202CF6D99142F2D1491EA2
:10D71000816010BC70470000F8B50C460546104605
:10D72000194600F013F8064600200090064B3246DA
:10D7300021462846FEF747FD0028304602D100F07A
:10D7400043F80020F8BD00009447002070B505465E
:10D750000E46124800F0A2F804001CD0E661082032
:10D76000A561E0600E4A0F4B28463146FBF7F4FAFC
:10D7700002D80D4860610EE000220C4B284631466D
:10D78000FBF7D6FA02D80120C00703E0284631464D
:10D79000FBF776FA6061204670BD000094470020D8
:10D7A0000000C0FFFFFFDF41FFFFFF7F0000E0C17F
:10D7B00010B5044800F072F8002801D04021C16083
:10D7C00010BD000094470020002824D0F8B5124E68
:10D7D00004460027A0892568C0050DD4A06800284C
:10D7E00004D0FFF7F1FFA089C00505D42069002807
:10D7F00002D0716888472761A089800505D4206A16
:10D80000002802D0716888472762716820468847DF
:10D810002C00DFD1F8BD70479447002010B50022DE
:10D8200001F088FD10BD000030B4124A0E4D0F4BC0
:10D830000F4C0028136013D00168002900D011603C
:10D8400054604068002800D050600020906010684C
:10D85000984203D15068A04200D1956030BC704717
:10D860009560546030BC7047012A010171B8000115
:10D870000DB8000194470020002803D0007B082841
:10D8800001D00020704701207047002803D0007BA2
:10D89000402801D0002070470120704710B5016872
:10D8A0002820884700280AD000210160416081605B
:10D8B000C160016141618161C1610162416210BD6C
:10D8C00070B5002604463546002808D0FAF7F0FC6B
:10D8D000411C2B463246204600F004F870BD002063
:10D8E00070BD0000FFB5002489B006460094019485
:10D8F00034480294039404940594069404601546F5
:10D900004460002E5AD000293FD002460096019173
:10D91000D168906812690490069205912A48FFF731
:10D92000BDFF0790002830D000986F46002802D035
:10D930000298002801D000200DE00198042809D9A0
:10D94000032222A10098FAF7E8FC002802D10298ED
:10D95000C01C02903846FFF7C1FE0146079803F04D
:10D960002DFC00280ED00C98002814D06846FFF734
:10D97000B5FE02990198814204D202990098405C58
:10D98000002808D00798FFF71FFF019902988842E6
:10D990000AD204460BE0002D03D0029900984018EB
:10D9A000286007980DB0F0BD081E00D0441E002D61
:10D9B00001D03019286003480660446000200DB093
:10D9C000F0BD00008C47002094470020EFBBBF0053
:10D9D00010B5024A002103F00FFF10BD944700204C
:10D9E000014949680847000094470020002810D0EA
:10D9F00070B50E460446FAF75BFC401C33680546DA
:10DA00009847061E04D02A462146FAF72DFC3046D8
:10DA100070BD7047002230B4D243491E0FD3094C69
:10DA200003785A400023401C5508D20700D02246F4
:10DA30005B1C6A40DBB2082BF6D3491EF0D230BC27
:10DA4000D04370472083B8ED02468B880020022B1C
:10DA500001D00D207047C988002A05D00029F9D0CF
:10DA60000129F7D0812070470029FCD00229F9D183
:10DA700070470F20704700000F2804D20C21484344
:10DA80000249085870470020704700001C480101F7
:10DA900070B588B000246A46234616E0401C017821
:10DAA0002029FBD00929F9D00906090E12D0A100BE
:10DAB0005050641C00E0401C017800290AD0202945
:10DAC00001D00929F7D10370401C0178002901D049
:10DAD000082CE4DB002C14D0104E002528460C2125
:10DAE000484331580098FAF7EAFB00280CD06D1C27
:10DAF0000F2DF3D30AA0009900F024F8012008B0FC
:10DB000070BD002008B070BD0C204543A819826884
:10DB1000694620469047002008B070BD1C480101AE
:10DB2000756E6B6E6F776E20636F6D6D616E643AAC
:10DB30002025732028747279202768656C70272946
:10DB40000D0A00000FB410B503AB60210648029A1D
:10DB5000FDF72AFE05490020C877034800F058F871
:10DB600010BC08BC04B0184760500020A050002032
:10DB7000F3B581B00D460198FAF79AFB144C86B2C2
:10DB80002046FAF795FB81B22046FFF75BFD0024A3
:10DB9000002D0BD90F4F3846FAF78AFB81B2384671
:10DBA000FFF750FD641CA4B2AC42F3D3084C2046EE
:10DBB000FAF77EFB81B22046FFF744FD002E03D02A
:10DBC00031460198FFF73EFD304603B0F0BD00003E
:10DBD000B8A60001C4A6000130B40125074B084CCB
:10DBE000AD0203E06254491C1981401C0278002AEE
:10DBF00002D01989A942F5D330BC70474C470020A8
:10DC00007B58002001490860704700004047002011
:10DC100010B507490968002901D0884710BD04469E
:10DC2000FAF746FB81B22046FFF70CFD10BD00005D
:10DC300040470020F0B51FB405460398144646003F
:10DC40000198760847007F08334628463946FBF797
:10DC500083F802D22846394601E020463146332275
:10DC6000D243FAF7A5FF06460F4622462846039BF5
:10DC70000199FAF7AFFE490049083B463246FBF7E7
:10DC800057F802D8012005B0F0BD002005B0F0BD66
:10DC900002460020802901D98D207047062A06D02F
:10DCA000072A07D0082AF8D10729F5D17047082993
:10DCB000F2D170470629EFD370477047704770B5AF
:10DCC000C46805466068002803D00020002802D000
:10DCD0000CE00120FAE7201DFBF76CFC09F41CD6D0
:10DCE0006068002808D000200028F4D00020E860F8
:10DCF000204609F411D670BD0120F5E730B4044682
:10DD0000A2890920521C93B2E48900222546D540FD
:10DD1000ED0707D05D1C8D4202D130BC1046704724
:10DD20009B1C9BB2521CD2B2092AEFD330BC704765
:10DD3000FFB585B00E9D04462F8801201E460021A8
:10DD40003A46CA40D20704D04B0003225B1C9A40DB
:10DD50001043491CC9B20929F2D3049030461E2150
:10DD60000840218A184A00230191009302920390EF
:10DD7000132304AA15490698FBF722FC00900028FB
:10DD80001FD10121142009F451D60746E0600698FE
:10DD90000188B9812988F981F00701D00120C003E9
:10DDA000079908433880208A7880142060822046B2
:10DDB00000F060F8381DFBF709FC208A002109F407
:10DDC0008BD7009809B0F0BD004101010A1800008E
:10DDD0000048704798410101FFB5087881B00C46B2
:10DDE000092836D2142003F031FC0746217800F0D0
:10DDF000EFF800282BD061782078FFF749FF060064
:10DE000028D17D68002D0ED020782979814207D154
:10DE10002946381DFBF7E0FB284609F47DD502E0D2
:10DE20002D68002DF1D160780121083009F4FED56C
:10DE3000054620782871607868716278A11CA81D59
:10DE4000FAF712FA2946381DFBF7CCFB02E08226CE
:10DE500000E0812602230648039A049909F46CD64F
:10DE600021780170467009F4A3D6002005B0F0BDFA
:10DE70000114000010B50446142003F0E7FB044928
:10DE8000216003216181123060600120208110BD7A
:10DE9000A8410101F8B517460C46104609F40AD707
:10DEA000012831D1142003F0D1FB0546017C00F09C
:10DEB0008FF80646297C22781448914214D1697C57
:10DEC000637809023A46891D9B1D09F435D605463B
:10DED000068000202871607868806278A11C681D27
:10DEE000FAF7C2F9284609E0697C062309023A4696
:10DEF000891D09F421D606808021017109F458D6C4
:10DF00000021384609F4E8D60020F8BD140C0000C2
:10DF1000F8B50F46002409781846254609291DD270
:10DF20000B007B441B79DB189F4404071013131369
:10DF30000A160D00052414A510E00A2414A50DE00E
:10DF4000082416A50AE0072417A507E00A2418A547
:10DF500004E0052419A501E006241AA50146A31C26
:10DF60001A4809F4E9D50646387830707470002CE8
:10DF700004D022462946B01CFAF776F9304609F457
:10DF800017D60020F8BD00004E53494E4700000050
:10DF90004E532D424C452D312E300000123456FF89
:10DFA000FE9ABCDE00000000025E04400000030098
:10DFB000312E302E302E302D4C450000312E302E9B
:10DFC00030000000FFEEDDCCBBAA0000031400000F
:10DFD00010B48289C489521C93B200222046D040DA
:10DFE000C00706D0914202D15B1C9BB205E09B1C8E
:10DFF0009BB2521C52B2092AF0DB092A02D010BC93
:10E000001846704710BC00207047000070B505002E
:10E0100005D0134E3068854203D1002070BD72B622
:10E02000FEE704F0D9FE6C6904F0E2FE70688442F9
:10E0300002D0B068844201D1022070BD09488442F8
:10E0400004D1A86A0028F7D1032070BD0648844295
:10E0500003D0002C01D0012070BD042070BD000051
:10E06000A4470020BC5D0020A85D0020002802D04D
:10E070000368002B01D100207047F8B50D464168B8
:10E080000446002902D0A068884211D21B4EB54236
:10E090000ED8A2686D1C5019814201D39818F8BDA2
:10E0A0002169002904D11649884203D9B04202D916
:10E0B0000020F8BD4600226A0027002A05D031461C
:10E0C00018469047050012D00CE0A16930468847F9
:10E0D00005000CD0A2682168521CFAF7C5F8E16966
:10E0E0002068884766602560A0684019F8BDE1692E
:10E0F00020688847676000202760F8BDFFFFFF7F2A
:10E10000FFFFFF3F70B50D4D04460A2809D10D21D0
:10E110002846FDF721FB80212846FDF7ADFA0028AF
:10E12000F9D0E1B22846FDF717FB80212846FDF71C
:10E13000A3FA0028F9D0204670BD00000038014045
:10E14000F0B50878324F334D334E801E83B00C4605
:10E15000062859D201007944097949188F440225CB
:10E160005434543A01203070A0786876A078C00703
:10E1700005D02A492A48FBF70BFA387AA874B28AE4
:10E18000002A06D0FF20F53070800321254809F4CD
:10E1900095D7F169002937D0002000900190052023
:10E1A0006A461070684688472EE000246C7601F0BD
:10E1B000FDFDF169002927D0009406206A460194EC
:10E1C0001070684688471FE01722A11C1648FAF70E
:10E1D0004BF819E0B8780001C0194030807D002864
:10E1E00012D11C22A11C1148FAF73EF80F48A18A4F
:10E1F0000182E18A4182218B8182618BC1820B493C
:10E20000608A0883207F6874002003B0F0BD00009E
:10E21000B04D0020F44C0020104D0020B94D0020DE
:10E22000074D0020040F0000EE4C0020D44C0020CD
:10E23000F0B518460D46014685B0222303227448E6
:10E2400009F47AD401210446417028780B286ED253
:10E2500001007944097949188F4405CDCDCD6F6A05
:10E26000BB23CDCD6C00012020706070694881799E
:10E2700021710179A170C17961714179E170017AEF
:10E28000A171417AE171817A2172C16900294ED070
:10E290000020009002206A4610706846019488476A
:10E2A000A9E0072020700120607068461DF4D6D1D7
:10E2B000019F009EF9F7C6FF801960820025F9F7DB
:10E2C000C1FF8119601900908170F9F7BBFFC11976
:10E2D00000986D1CEDB20175082DF0D30825F9F7F3
:10E2E000B1FFB919401861196D1CEDB28870102D7D
:10E2F000F5D310202077484881780901081840306C
:10E30000807D012877D11C22A11C4448F9F7ACFF7D
:10E310004248A18A0182E18A4182218B8182618BFC
:10E32000C1823E49608A08833D48217F417462E092
:10E33000052000E00A2020705DE004222270687849
:10E34000012804D0002802D0022833D053E0012055
:10E35000304D6070287C002810D002A81DF47ED1BA
:10E36000F9F770FF2F49F9F70DFF2F4808180299A8
:10E3700040182E49F9F706FF009101E0E868009087
:10E38000E969002907D00020029003206A46107234
:10E3900002A8039288471021A01CF9F77EFF00987D
:10E3A000A0700098000AE0700098010C2171000E26
:10E3B000607120E01748C169002905D00020009055
:10E3C000019068460270884720460C3809F4E6D36D
:10E3D00014E00620164D2070E878012811D0102195
:10E3E000A01CF9F75AFFA9886182E988A1822989CE
:10E3F000E18200202076204609F4DAD3002005B01F
:10E40000F0BD10220B49A01CF9F72EFFEBE700002E
:10E41000140E0000104D0020B04D0020D44C002000
:10E42000F44C0020A0BB0D00A08601003F420F006D
:10E43000344E0020BF4D002000B5084883B0026C68
:10E44000002A08D000200090029005206B4618702A
:10E45000684601919047002003B000BDB04D0020F8
:10E4600010B584B0FF2B19D0144C226C002A08D0B0
:10E4700000200090029006206B46187068460191BB
:10E480009047032009F416D4032814D1A26F002A60
:10E4900011D003210A4809F411D60CE009480123E0
:10E4A000007F032201020848083109F445D30721FF
:10E4B000017009F47DD3002004B010BDB04D0020E0
:10E4C000090E0000104E0020050E0000FFB5180ACE
:10E4D0004C4E83B00C46B070FF287DD0010234232F
:10E4E00003224948083109F427D30546B0780027AC
:10E4F0000101891940318872B078218800018019A2
:10E5000040300181B078617A000180194030C172D9
:10E51000B07862890001811940318A81A289CA815B
:10E52000E0890882207C012802D0002807D00BE077
:10E53000B1780120090189194031887504E0B0786B
:10E54000000180194030877520883080607A3072F1
:10E5500021460A312D48FBF71BF802F0F9F9002893
:10E560001BD0607A012804D103221146284809F4FF
:10E5700033D302F0F5F905280FD201007944097967
:10E5800049188F4406060602060001202821485536
:10E5900005E005212820415501E0282047550321A9
:10E5A000059809F499D317203086B17809018919A3
:10E5B000403148821748C068002803D0032116481C
:10E5C00009F4DCD41548028D002A03D00321144835
:10E5D00009F474D5306C00E00EE0002808D0022069
:10E5E00069460097087002950194316C6846884727
:10E5F000284609F4DDD201E001F050FB002007B00D
:10E60000F0BD0000B04D0020020E0000B94D00200A
:10E61000150D0000C04E0020030F0000344E0020F6
:10E62000020F000030B5180A144D00010C464019C5
:10E6300083B0FF214030817201F004FC002803D137
:10E640000221032009F448D32A6C002A08D00020B4
:10E650000090029003206946087068460194904734
:10E6600010210748F9F719FE06480068002802D073
:10E67000092009F41BD1002003B030BDB04D0020AB
:10E68000CF4D0020100C002000B5084883B0C169B0
:10E69000002907D000200090019009206A461070E0
:10E6A00068468847002003B000BD0000104D0020E0
:10E6B000FFB591B00D46122303224348149909F483
:10E6C0003BD200210446017040480078002862D007
:10E6D0003E48407C002833D03C216846F9F7DDFDF8
:10E6E00001F028FF002841D004A90F913749461EA8
:10E6F000F0B23A228969504341186846091DF9F77A
:10E70000B3FD6846008B2988884206D10822A91CDF
:10E710000F98F9F7ECFD00280BD0207800280BD0DB
:10E7200008A8407C607410226946601CF9F79CFDC3
:10E730001CE001202070F3E73006000ED6D12AE05D
:10E7400023482988008B884225D10822A91C21480A
:10E75000F9F7CDFD002809D1012020701E481022B4
:10E76000407C60741A49601CF9F77EFD207800280F
:10E7700011D01648C169002907D0002000900190EF
:10E7800007206A46107068468847204609F410D270
:10E79000002015B0F0BD0D48C169002907D0002048
:10E7A0000090019008206A4610706846884702234E
:10E7B00003220A48149909F4BFD1012101700621EE
:10E7C000417009F4F5D1E0E7180E0000104D00206B
:10E7D000D44C0020E44C0020F44C0020040E000037
:10E7E00070B50C4609781B481B4D1E46002904D005
:10E7F000012912D002292BD11AE01C23314609F439
:10E800009BD1064620783070287B70802A7B134984
:10E81000301DF9F729FD304607E00A23314609F497
:10E820008BD1217801706989418009F4C1D10FE051
:10E830000A23314609F480D121780170298C418066
:10E84000698C8180A98CC180E98C018109F4B0D1E7
:10E85000002070BD0B0E0000344E0020414E002001
:10E8600010B5087800F058FF002010BD05480A8850
:10E8700042861A0A1201101809884030818200204D
:10E8800070470000B04D002030B5180AC0430006A4
:10E8900083B00D46000E21D0190A0902E12006239B
:10E8A00003220001083109F447D1044601202070F9
:10E8B00002206080FF204130A0800B48026C002ABB
:10E8C00008D0002000900420694608706846019531
:10E8D00002949047204609F46BD101E001F0DEF983
:10E8E000002003B030BD0000B04D002000B5084846
:10E8F00083B0026C002A08D000200090029008200B
:10E900006B461870684601919047002003B000BD27
:10E91000B04D002070B518460C46014602230A4847
:10E9200009F40AD105460949A07808736288211DB7
:10E930000748F9F799FC002068702078287028466D
:10E9400009F436D1002070BD0D0E0000344E0020B9
:10E95000414E00204A780B48002A05D02030012A79
:10E9600008D0022A09D00AE00279012A07D10978E1
:10E97000C17004E00978017501E009784175002053
:10E9800070470000B04D002070B54878002806D0D0
:10E99000FF25124C01280BD0022816D01BE010488E
:10E9A0000179062917D10721017101F0E5F812E07C
:10E9B000207DFF280FD001F0DDF90A482575016997
:10E9C000002908D00020884705E0607DFF2802D09C
:10E9D00001F0B2F96575002070BD0000D04D002037
:10E9E000B04D0020C04E002010B5032B06D01022E1
:10E9F0000548891DF9F738FC002010BD0348017A4D
:10EA0000034801F04DFEF7E7CF4D0020B04D002048
:10EA1000B94D0020F0B50D460878E34EE149344683
:10EA20004978002720348DB0A1287AD012DCDF4944
:10EA30000C911B2876D006DC012819D003287CD045
:10EA400017286DD14FE128286ED091286DD0A028CD
:10EA500066D152E10246A23A092A61D213007B44F0
:10EA60001B79DB189F44FE5CFDFD5CFDFCFDFD0099
:10EA70006878002854D1012002F04CFE01F04EFECF
:10EA8000342303220721CA4809F456D00321017018
:10EA9000C84904468A7842700122C276FB22428429
:10EAA000C54AC284C54A82840A88028487768A88D5
:10EAB0008280CA88C2800A892281487A8009032814
:10EAC00005D188780522104201D10120A076A07ED0
:10EAD00004221043A076BA486080C878012825D067
:10EAE000204610210A30F9F7D8FB316C002907D0F5
:10EAF00001206A4600971070684601950294884785
:10EB0000012000F009FE204609F452D0012303221F
:10EB10000721AC4809F410D01A21017009F448D03B
:10EB200033E11EE1CAE008E069E049E02046102236
:10EB30000A300C99F9F798FBD7E7009701970297ED
:10EB400003970497059706970797089709970A97D9
:10EB50000B9701F0FDFE002805D0684601F03EFD50
:10EB60000AA801F00BFD01F0F3FE00280CD0684666
:10EB70008079002808D108A8807B002804D00121D2
:10EB8000684601F071F900E18A4C6946A088088066
:10EB9000E0884880208988808F71102202A80C9913
:10EBA000F9F762FBE078012804D0069707970897E9
:10EBB0000997E4E7102206A80C99F9F755FBDEE760
:10EBC000E07B002813D11123032207217E4808F49B
:10EBD000B3D70546282028707648C078012808D089
:10EBE0001021681CF9F759FB284608F4E1D7E773B0
:10EBF000CBE01022681C0C99F9F736FBF4E70120F2
:10EC000002F088FD0121032009F466D06F48012439
:10EC100044841F20049067480178490601D57F216C
:10EC2000049181780522114204D0FF220499813297
:10EC3000114304910088C00504D5032104984902BA
:10EC400008430490082162480191029003210B239C
:10EC500004AA00970394C9025E48FAF7B1FC02E0E7
:10EC600079E04AE089E0002846D15B4806218786A2
:10EC7000FF200590594801910290082305AA0097AA
:10EC8000039457495748FAF79BFC00287DD100F0C0
:10EC90005DFF002879D10221032009F41DD0B0794D
:10ECA000012808D001F022F83E484078C0076CD017
:10ECB00001F064FB69E000F0F1FF66E001F048FE5E
:10ECC000E77300F043FF00285FD10221032009F41D
:10ECD00003D0B0790128EED001F008F8314840782F
:10ECE000C007E5D151E0687800284ED0F179481E80
:10ECF000F0713D4801F0A4FC47E07179491E0529F7
:10ED000006D8A72802D13079002806D100F034FFB8
:10ED10002878A42801D0A72837D17079042806D0F4
:10ED2000062804D0082808D00C282ED10CE02F4843
:10ED30000168002929D0B07904E01A480169002946
:10ED400023D00120884720E01648016900291CD003
:10ED50000320884719E03771FF20F0702075607537
:10ED600013E0207DFF2802D06878002802D001F04F
:10ED700001F80AE0C8079BD107E0607DFF2802D0B8
:10ED80006878002804D000F0D7FF00200DB0F0BD57
:10ED9000A07D0028F9D08807F7D5E17D144801F05F
:10EDA0005BFAF2E7C04E0020B04D0020BF4D0020BE
:10EDB000040D0000344E0020050200004808000049
:10EDC000A08C0000190D0000230D0000B00B0020E6
:10EDD0007C450101D20B0020680B0020D4450101C5
:10EDE000011800009C0B0020B94D0020604E00204F
:10EDF000E84D002070B500250C462846401C06282A
:10EE0000FCDB254E2246307E31461A32C96906287F
:10EE10002AD203007B441B79DB189F44240209108B
:10EE2000171E0622A01CF9F762FA00281BD01BE06F
:10EE3000237E092001F0B0F8002814D114E0237ECD
:10EE4000212001F0A9F800280DD10DE0237E162025
:10EE500001F0A2F8002806D106E0237E192001F077
:10EE60009BF8002800D001250C48807D002811D196
:10EE70007169002901D020468847002D0AD03169E8
:10EE8000002901D00220884701F0FAFA217AA01C5B
:10EE900001F0E2F9002070BDC04E0020D04D0020EE
:10EEA00010B50A78000A000210434A78FF231B02BB
:10EEB000120298431A4010438A781B0212049843A6
:10EEC0001A401043C9780002000A09060843F9F7FE
:10EED000C2F9002010BD10B5104608F4EBD6002092
:10EEE00010BD0020401C0628FCDB002070470000FD
:10EEF000F8B51C4617460D46104608F4DBD6002828
:10EF000011D1472002F0A2FB064604233A46032112
:10EF1000064808F411D6210A01702988B288891A96
:10EF2000418008F445D60020F8BD00000D470000E0
:10EF3000F8B517460C46472002F088FB21780646B4
:10EF4000122901D013291BD1B06805460C351229AE
:10EF5000C288018916D006230F4808F4EDD56988C8
:10EF600041806178017108F423D6B068002803D08D
:10EF700008F4D2D40020B0600021384608F4ACD6A2
:10EF80000020F8BD0423054808F4D6D5698801801F
:10EF900061788170E7E7000009470000074700003B
:10EFA00000B5084883B0026C002A08D00020009009
:10EFB000029009206B461870684601919047002026
:10EFC00003B000BDB04D002030B5104D83B00888AF
:10EFD00028861C0A200140190A88403042822A6C87
:10EFE0000025002A07D0009507206B46029518706F
:10EFF0006846019190470648A1004058002801D07A
:10F000004030C574002003B030BD0000B04D00207A
:10F01000580B0020FFB581B0002000900E460398E9
:10F0200008F448D6002802D001284CD04DE0142026
:10F0300002F00CFB07463188FEF760FE05462448C7
:10F04000092D36D27C68002C1ED02179A94203D02C
:10F050002468002CF9D117E0002C15D06379039AAD
:10F060009B1D049908F468D5054630882880002047
:10F070002871607968806279A11D681DF9F7F4F83C
:10F08000284608F495D520E03D740498010A797467
:10F09000384602F0D3FA014601230E48039A08F4D9
:10F0A0004BD5057008F484D50121039808F414D6D3
:10F0B0000BE00623039A049908F43ED531880180B9
:10F0C00080210171DDE702200090009805B0F0BDBD
:10F0D000140C000002140000FFB585B00E4607981E
:10F0E00008F4E8D5002802D0022009B0F0BD47207E
:10F0F00002F0ACFA02900020694608700898070AEE
:10F10000308803F0A8F90024694605468C80002861
:10F110001ED102981622016A6846007803465043C1
:10F12000024610328A5A5204920F1FD10A5C401CC8
:10F13000085C1E4900021018884217D102AA03A9D0
:10F14000184603F09BF802986946C05D8880022447
:10F15000A31D1748079A089908F4EED4074630888B
:10F1600038803D717C80002D15D019E03946029819
:10F1700002F064FA014604230E48079A08F4DCD42E
:10F18000077069460978418008F412D50121079873
:10F1900008F4A2D507E0224601A9781DF9F764F822
:10F1A000384608F405D5002009B0F0BD022900005A
:10F1B000140C000004470000FFB58BB00C4647203C
:10F1C00002F044FA0025694605900D740E9804A9D2
:10F1D000070A208803F03FF9060061D1059816223E
:10F1E000016A6846007C5043024610328A5A520433
:10F1F000920F3AD10A5C401C085C3049000210189A
:10F20000884232D102950395208800F0DFF802A9E8
:10F21000002300911A4608A9FAF7EAF96846008C1B
:10F22000012109030840C043C004C0172146401C07
:10F23000FEF70AFC0606360E32D168460997007CB6
:10F240000190A57907AA694603F018F86846028874
:10F2500006A80799F9F708F806A909980A460D546F
:10F2600068460188019803F047F83946059802F08E
:10F27000E5F9A1880D9A891D8BB20146104808F462
:10F280005BD40546A288A11D801DF8F7EDFF2F7005
:10F290006846007C6880A088A880284608F488D446
:10F2A000042308480D9A0E9908F446D42188018059
:10F2B000867008F47DD400200FB0F0BD0229000054
:10F2C0000A470000160C0000F0B589B00446FAF7B2
:10F2D00095F905460026154F1BE006A92046FAF7CA
:10F2E0005DF9002302AA01A906A80096FAF78CF995
:10F2F00068460089B84203D169460979022911D0CC
:10F300000B49884203D168460079022807D0641C63
:10F31000A4B2A888A04202D8E888A042DDD200208A
:10F3200009B0F0BD204609B0F0BD00000229000080
:10F3300003280000F7B5002845D00199002942D0E4
:10F340008668002A01D10CE03668002E3BD0316A75
:10F35000002938D00198F8F7B2FF0028F4D12CE04A
:10F360003668002E2FD0019C356A002CF8D0002D75
:10F37000F6D0AC4224D02078F8F75EFF0746287814
:10F38000F8F75AFF87420DD12078002813D0607813
:10F39000641C6D1CF8F750FF07462878F8F74CFFFF
:10F3A0008742F1D02078F8F747FF04462878F8F72D
:10F3B00043FF8442D4D1002E05D0306A002802D009
:10F3C000304603B0F0BD002003B0F0BDF0B589B009
:10F3D0000446FAF713F905460026104F14E006A973
:10F3E0002046FAF7DBF8002302AA01A906A8009636
:10F3F000FAF70AF968460089B84203D1641CA0B242
:10F4000009B0F0BD641EA4B2A888A04202D8E88862
:10F41000A042E4D2002009B0F0BD000003280000A3
:10F4200070B5164C2078002827D101210803FBF77E
:10F430007DFF0020FBF770FF0120FBF79BFF104DC5
:10F440002846FAF78FF903212846FAF7FBF901213C
:10F450002846FAF7BBF9012121702846FAF7DEF9B0
:10F46000142003F001FD702000F00CF8702000F073
:10F4700009F800212846FAF7D1F970BD8447002029
:10F480000008024070B50546164CFFF7C9FF294633
:10F49000154D2846FAF7F1F801212846FAF78CF9BC
:10F4A00001212846FAF7C6F9002807D1641E13D0B7
:10F4B00001212846FAF7BEF90028F7D00121284695
:10F4C000FAF7D8F82846FAF7B2F904460021284698
:10F4D000FAF772F9204670BD00212846FAF76CF958
:10F4E000024870BDA086010000080240FFFF000036
:10F4F000F7B504270225494E86B01446082A74D26F
:10F500001000784400790018874484030D3A3D5375
:10F5100063704348019001AB00970799069800F08B
:10F520008BF809B0F0BD3F4F01213846FAF776F964
:10F53000142003F099FC7020FFF7A4FF7020FFF760
:10F54000A1FF044600213846FAF768F93648B4426C
:10F55000448001D1354808E02046FAF795F834494F
:10F56000F9F756F9F9F772FB00B2694688812A4625
:10F5700003AB00950799069800F05EF809B0F0BD5E
:10F58000FDF7B4FA0AE06020FFF77CFFB04201D13A
:10F59000002003E06021FAF7A1F880B269460881F3
:10F5A00002AB224600950799069800F045F809B08D
:10F5B000F0BD04F09BF97D21C900F8F7E3FD01904F
:10F5C00001AB224600970799069800F035F809B07C
:10F5D000F0BD03F085FD019001AB2246009707992D
:10F5E000069800F029F809B0F0BD13E0FDF77EFBA6
:10F5F0001049884201D1022000E0012069460874C8
:10F600000120009004AB22460799069800F014F8F8
:10F6100009B0F0BD079809B0F0BD0000FFFF000081
:10F62000110001000008024084470020FF7F000015
:10F63000000020410040020130B4029C42540546C3
:10F64000491C88B22C54401C002180B2002C07D9E0
:10F650005A5C2A54401C491CC9B280B2A142F7D35B
:10F6600030BC704710B5084C82B02078002808D113
:10F6700006480090064801906846FEF7D5F801203C
:10F68000207002B010BD0000A04700204D210101F4
:10F690000D2E0101F8B50B30C608F600104D19E02B
:10F6A0002068B04215D3B0420BD96368871B201D78
:10F6B0000093F8F7D9FDA019009B0760436028600C
:10F6C00004E060682860201DF8F7CEFD201D26604C
:10F6D000F8BD251D2C68002CE2D10020F8BD0000EB
:10F6E00000480020FF25F5350A4E6F00FDF792FB1C
:10F6F0000489322C00D22C4601213046FBF7F8FC5D
:10F700007D212046C90048433946F8F73BFD03F008
:10F71000ABFBEBE7000C014010B5A0230949022820
:10F7200009D0002203280AD0042808D00B704A70A0
:10F7300000F0A2F810BD0B7080204870F8E7E020C0
:10F740000870F4E711400020F8B52A4920204860ED
:10F7500029480121C163294905228A610021C16329
:10F7600027490B20086100F087F82748254A0263E3
:10F7700026494163264B8363264CC4632748264DA4
:10F780000560274E4660274981602749C1602749A7
:10F79000016127494161274981612749016328485F
:10F7A00026494160274FC760274F07610262274AF9
:10F7B00042628362C46205634663254A8263254AC6
:10F7C000C2632648244A0260184A4260244A826082
:10F7D0000163244981632448244A41688918244AE2
:10F7E000914206D2234982680A63C2684A6300696B
:10F7F0008863F8BD00100140C02702404025024048
:10F80000402702400259F80040280240025B850070
:10F81000025A8000025D8500025F8050802802400D
:10F8200002000878020A0800026EAC500259FC007F
:10F830000200C8001270131402700314026E280034
:10F84000C0280240025D0500125B0500025B8400D7
:10F85000020A0600026E2C5002C3BF0000290240BB
:10F860001200AC00125D0500104000206F2895FFCB
:10F87000AF590F00C026024030B415481549037D2A
:10F88000154AFF2B06D1407DFF2803D1134840784D
:10F89000C0070CD01248134B04789C604078D861A4
:10F8A00011480861114B8B62106030BC7047104BDF
:10F8B0000B6110484861104C8C61104D8D62C8621C
:10F8C0000F48086313600F485060946030BC704765
:10F8D000D04D00200028024040280240C04E0020A9
:10F8E0001140002000270240127E0200127E030019
:10F8F000027E020002C2A00012C70000027E0300C6
:10F9000012C7800002C2E00082B02249204808638A
:10F91000FDF78AFD20A0FBF723FF2AA0FBF720FFBD
:10F9200031A134A0FBF71CFF3848016838A0FBF771
:10F9300017FF3EA142A0FBF713FF4AA0FBF710FF01
:10F94000FCF74AFDFCF73AFE01215148FBF7D4FBD6
:10F9500040215048FBF7D0FBFDF760FA01F03AF880
:10F96000022000240202009023464BA101944B4840
:10F9700003F0F0FE012000900023802248A10194B2
:10F98000484803F0E7FEFAF777FA03F047FBFEE793
:10F9900000800081007000400A3D3D3D3D3D3D3D01
:10F9A0003D3D3D3D3D3D3D3D3D3D3D3D3D3D3D3D87
:10F9B0003D3D3D3D3D3D3D3D3D3D3D3D3D3D3D3D77
:10F9C0003D0A0000206D636D2D6464632D626C65DB
:10F9D0003A20424C45202B204672656552544F53C5
:10F9E000202B20434C490A0056312E30302E31371F
:10F9F00000000000204669726D77617265207665AF
:10FA00007273696F6E2025730A00000000400020A9
:10FA10002053797374656D436F7265436C6F636BCC
:10FA2000203D20256C7520487A0A00004341494951
:10FA3000432D4D434D2D32303236303930320000B7
:10FA400020424C4520656E61626C65642C206164C7
:10FA5000766572746973696E6720617320222573FD
:10FA6000220A00003D3D3D3D3D3D3D3D3D3D3D3D8E
:10FA70003D3D3D3D3D3D3D3D3D3D3D3D3D3D3D3DB6
:10FA80003D3D3D3D3D3D3D3D3D3D3D3D0A00000090
:10FA9000000C014000080140424C450081D10001AA
:10FAA0004C454400E5F6000110B50124E40220466F
:10FAB000FBF70EFA002805D02046FBF703FA0D49A4
:10FAC00002200870012424032046FBF701FA0028D5
:10FAD0000AD02046FBF7F6F9BFF34F8F07490648D7
:10FAE000C860BFF34F8FFEE705484068002800D08C
:10FAF000804710BD800000200400FA0500ED00E002
:10FB00004040002006480068002800D08047BFF32E
:10FB10004F8F05490348C860BFF34F8FFEE70000D1
:10FB2000404000200400FA0500ED00E0064A11788C
:10FB30000A2907D28900891848601078401C107083
:10FB40000120704700207047304D002010B5084C50
:10FB5000084AE17913780020994207D2880080187A
:10FB600040688047E079401CE071012010BD000032
:10FB7000B04D0020304D0020F8B5324D05262979D2
:10FB800028468079304C08290CD20A007A44127930
:10FB90009218974403080D1313191C2A052801D045
:10FBA000FCF78EFEF8BD022808D0FDF7B1F9F8BDCC
:10FBB000607B002802D1E079002802D0FDF746FAE8
:10FBC000F8BDFDF7E1F9F8BD06202871F8BD022364
:10FBD000032207211D4807F4AFD7A5210170E9785A
:10FBE0004170072129716E7128E002230322072149
:10FBF000174807F4A1D70746A7203870E97879702D
:10FC00000620687100202871032008F453D00328CF
:10FC100012D0A879012804D0022802D003280BD1E1
:10FC200004E0207D002801D0032003E0A07E00280E
:10FC300002D00420A87100E0AE71384607F4B8D7AE
:10FC4000F8BD0000B04D0020A04E0020A20D000025
:10FC5000A30D000010B5002804D0014660220C4816
:10FC6000F8F702FB0B490C48CA781C2A04D9427BDE
:10FC7000002A01D11C22CA70C1781F2901D91F2175
:10FC8000C170017BE22901D9E221017310BD00009E
:10FC9000604E0020804E0020A04E0020114901221D
:10FCA000087907280CD08879002809D0012801D0CC
:10FCB000052806D10C48827B002A03D002200CE0E4
:10FCC0008A717047027D002A01D0032005E0807E02
:10FCD000002801D0042000E00520887110B5FCF751
:10FCE000EFFD10BDB04D0020A04E002070B5104CAF
:10FCF0000525A079062809D2010079440979491817
:10FD00008F44020204040403A57170BDA57102238F
:10FD100003220721074807F40FD7A5210170E178D6
:10FD2000417007212171657107F442D770BD000051
:10FD3000B04D0020A20D000010B50B4C607DFF28D7
:10FD400010D0022303220721084807F4F5D6A72183
:10FD50000170617D4170064A00215171FF2161757A
:10FD600007F426D710BD0000D04D0020A30D0000E1
:10FD7000B04D002010B50A4C207DFF280ED0022384
:10FD800003220721074807F4D7D6A7210170217D58
:10FD90004170054A0021517107F40AD710BD0000D7
:10FDA000D04D0020A30D0000B04D002010B5084834
:10FDB00002238078032201020648083107F4BCD6EA
:10FDC000012101701321417007F4F2D610BD00002B
:10FDD000B04D0020040E000010B584B0002804D0FF
:10FDE00001462A220E48F8F73FFA0EA00FC86C46CB
:10FDF0000FC40B4B002069461C180A5C247922436F
:10FE00000A54401CC0B20628F6D310220A48F8F75C
:10FE10002BFA0A490A48F9F7BBFB04B010BD0000F1
:10FE2000344E0020501921901F04D5624FA489AB95
:10FE300090D0CF2300000000BF4D0020384E00209E
:10FE4000FC0000200020074B01460A01D218403276
:10FE5000927AFF2A01D0401CC0B2491CC9B20329C2
:10FE6000F3D37047B04D0020F8B507460B46282065
:10FE700043430D46032207210E489B1C07F45CD622
:10FE800091210170002406464570002D0ED92046B0
:10FE900028214843C1190022CA7180192822801CD8
:10FEA000F8F7E2F9641CE4B2AC42F0D3304607F450
:10FEB0007FD6F8BD910D0000F8B57D262025F6000F
:10FEC000184B194C1949032812D00A6A01273A43E2
:10FED0000A620A6A9207FCD50A6AAA430A620128E2
:10FEE0001AD002281AD01E60F9F794FB2060F8BDE2
:10FEF0000F480F2782683F023A438260086A042253
:10FF000010430862086A0007FCD5086A28430862A3
:10FF10003D2000011E60E9E7064800E00648186041
:10FF2000E2E700008C00002090000020001002405A
:10FF300000100140D10300005704000010B5044632
:10FF4000084804238078032201020748891D07F42A
:10FF5000F3D506494C80012101700021418007F44E
:10FF600027D610BDB04D0020010C0000F00B002082
:10FF7000084A11780A290AD2C9004368891800681A
:10FF80008B6048601078401C107001207047002082
:10FF9000704700005C4D0020FFB581B01C00064694
:10FFA00018D01078411CA14214D8032C12D3401E43
:10FFB000C5B25078971CB04206D12A4638460299FD
:10FFC000F8F795F9002808D07A19601B801E0406FE
:10FFD000240EE6D1002005B0F0BD012005B0F0BD33
:10FFE000F0B504466F4E704883B06D4FB168C16282
:10FFF0006E490163F16A8162F16B4163B16B8163A8
:020000040101F8
:1000000031467C2240313846F8F72EF900257D60D4
:10001000FD607D626648B8627D64BD64FD643D66D6
:100020006448B866644838626448654905700320CE
:1000300008706448F91401600904016089140160C2
:10004000F06861490746401E0088604B884200D036
:100050001F60366E701E0088884200D05E600120EE
:1000600000030090694601950D7108204871012731
:100070008F716846FAF73AFF84215548F8F70DF971
:100080002A215448F8F709F960215348F8F705F98F
:1000900052484F49056145618561C5610562456208
:1000A0008562C562FF264E48CE70067546750020F3
:1000B000020152184032401CC0B296720328F7D396
:1000C000206808646068486446486189C187217A6D
:1000D0004548032901D8417700E0457701212020D8
:1000E000FBF724F9414A4249042001F041FA424910
:1000F000404808600A464149052001F039FA404A63
:100100004049072001F034FA40493F4808600A4658
:100110003F49082001F02CFA3E4A3F49092001F0EE
:1001200027FA3E4805633E48414907703D4805703F
:100130003D4805703D48086001203E49C0020880E6
:100140003D494F2008703D49082008703C48072170
:10015000067046708670C170057145718571C571F4
:1001600011483849C161384901623849416200206B
:1001700002F080FC3649032007F4F2D50021032069
:1001800007F4AAD5002001F0C5FA012303220721B4
:10019000304807F4D1D4077007F40AD503B0F0BD96
:1001A000C009002000800001C000002005FB000104
:1001B0000D4700208D2B0101A9FA0001C600002087
:1001C000D800002000E100E0FEE7000040400020F1
:1001D000B04D0020344E0020604E0020B04E002074
:1001E000D04D0020F04D0020104E00208040002017
:1001F0008080010049420101C0400020C080010010
:100200000041002000DB010081410020404100202E
:1002100040DB0100C0460020C061020000700040C9
:1002200060000020C9000020610000200090D00381
:100230006C000020680000206300002064000020A3
:1002400008010020B5150101DD1601017D1601012F
:10025000DC460101020D0000F8B5404D0646687D00
:100260003F4C0F46FF281CD02046C268002A03D00E
:1002700003213C4807F422D73A23032207213A48B6
:1002800007F45AD4A4210170697D044641703748AF
:100290000022017800291ED00121A170A2800270E5
:1002A0001BE06D20022303220721400107F444D400
:1002B000A22101702E49C978417007F479D4EF75F5
:1002C00031462C48F9F764F90120A87560780221BD
:1002D00008436070F8BDA270A2800120E07019216F
:1002E0004901E18022482181038CE381438C2382F0
:1002F000838C6382C38CA382FF23E2824133184D37
:1003000023836D786D070DD50525E5706181A18189
:10031000018CE184418C2185818C6185C08CA08514
:10032000E285238638200755204631463230F9F7DA
:100330002FF9E078810703D50220FFF7EDF906E0F9
:10034000400701D5032000E00120FFF7E5F90A4945
:100350000C204871204607F42BD4F8BDD04D002066
:10036000C04E0020030F0000A10D0000304E002001
:10037000344E0020E84D0020B04D0020F8B52C4E42
:100380002C4D317D01276878FF2941D0C1073ED02F
:10039000B84368702849002008703A2303220721D7
:1003A000264807F4C9D30446A4202070307D60702D
:1003B0002878A07068788006800F20716888E080B7
:1003C000A8882081E888E08128892082E7700120C0
:1003D000FFF7A2F9687840070AD5E07802210843C0
:1003E000E07068886081A888A0810320FFF794F9F5
:1003F0006878000703D5E0780C210843E0701049C5
:10040000082048710020B075204607F4D1D3F8BD0C
:10041000384368706D20022303220721400107F44E
:100420008BD3A12101700749C9784170EDE7000025
:10043000D04D0020C04E0020304E0020A10D000005
:10044000B04D0020344E002010B50A4C607DFF28CE
:100450000ED0022303220721074807F46DD3A521FC
:100460000170617D4170054A0D21517107F4A0D3DF
:1004700010BD0000D04D0020A20D0000B04D0020A6
:1004800070B50B4C207DFF2811D00A4D68790928E2
:100490000DD0022303220721074807F44DD3A521DD
:1004A0000170217D41700921697107F481D370BD0C
:1004B000D04D0020B04D0020A20D000010B5044624
:1004C0004088A1880246491C19234A43DB019A420D
:1004D0000FDC06280DD3228890420AD3E2887D23C0
:1004E000DB009A4205D84B00C9184843D100884226
:1004F00001DD002010BD0D480E238078032201028B
:100500000B48083107F418D3092101702188418074
:1005100061888180A188C180E188018100214181B9
:10052000491E818107F444D3012010BDB04D002045
:100530000E0E000010B5084A084B906901888478B7
:10054000994206D1917CA14204D20024FAF7A4FE7C
:1005500000E00024204610BD104D002034120000A1
:100560000B4610B504493A22896950434118184690
:10057000091DF7F779FE10BD104D002010B590B0A1
:1005800004463C216846F7F788FEFFF7D3FF401E7C
:10059000C0B26946FFF7E4FF08A8807CA0710CA9EF
:1005A00020460331F8F7F4FF10B010BD10B590B03D
:1005B00004463C216846F7F770FEFFF7BBFF401E7C
:1005C000C0B26946FFF7CCFF08A8007CA0710AA959
:1005D00020460231F8F7DCFF10B010BD10B590B026
:1005E00004463C216846F7F758FEFFF7A3FF401E7C
:1005F000C0B26946FFF7B4FF0AA920460231F8F7F6
:10060000C7FF08A8007CA071204606A91022083068
:100610000231F7F729FE0848C17820461830012931
:1006200004D01021F7F739FE10B010BD1022034995
:10063000F7F71AFE10B010BD344E0020BF4D002059
:1006400070B590B00D460646FFF774FF002D23D01D
:10065000854221D8182303220721104807F46CD2C1
:10066000044617202070012060703146A01CF8F766
:100670008FFF3C216846F7F710FE6D1EE8B2694611
:10068000FFF76EFF204606A9102208300231F7F767
:10069000EBFD204607F48CD210B070BD140D0000A5
:1006A000F3B58FB00C463C216846F7F7F6FDFFF72F
:1006B00041FF012C1AD0002816D0154D0AAE023683
:1006C000441EE0B23A22A969504341186846091D08
:1006D000F7F7CAFD062231460F98F7F708FE002803
:1006E0000DD02006000EEBD111B0F0BD0949421E1D
:1006F000CA7101460F98FFF7A3FF11B0F0BD06A91C
:10070000102205480231F7F7AFFD11B0F0BD00002F
:10071000104D0020B04D0020CF4D002070B5284C6A
:1007200082B020688003FCD5264D687FFFF7C4FBAC
:10073000606A606A012630436062606AB04360624A
:100740002148C08F0A2811D9E16932071143E161BC
:100750001E494A6832434A601E491D4A0A60032204
:100760004A6088601C4808601C48086068461AF4A3
:1007700075D71B4900980860687FFF252D02032864
:1007800011D000F027F9206BA8432063206B3F2194
:10079000490208432063206B304320630122032178
:1007A000104807F48BD410480168A94301600F4931
:1007B0000868FF2212049043086002B070BD000078
:1007C00000100240104E0020F04D0020401002406A
:1007D0005555000000300040AAAA0000CCCC000013
:1007E00048400020010F000000E400E008E400E0C1
:1007F000F0B5D7B054A81AF431D74A490024886A12
:10080000C96A54990122411A09010909D206914283
:1008100004D95499081A000100094142424E402966
:100820000CDC7088002809D0401E7080142203213F
:100830003E4807F443D4002057B0F0BD3C48FF21A8
:10084000569029316846F7F728FD707CB569002875
:1008500032D0FFF76FFE69468870B17C6F468842E0
:100860000BD23A2148430246291D381DF7F7FCFCFC
:1008700069468878401C887008E03A21401E484349
:10088000024629463E31381DF7F7EEFC6946887866
:100890003A214843C0190A4636385699F7F7E4FC1E
:1008A000244869460880B069FAF7F6FCFF2227322F
:1008B0006946B069FAF71EFDFF20F53070804A9452
:1008C0004B944C944D944E944F9450945194529414
:1008D00017485394418D40AA1185818D5185C08D53
:1008E0009085154C48AA257C9573102213494CA875
:1008F000F7F7BAFC1248C078012804D11022114938
:1009000050A8F7F7B1FC01260F48002DC67306D199
:10091000A07C002803D001214AA8FFF7A5FA0B48C4
:10092000067088E7C0800240104D0020040F0000D0
:10093000D44C002034120000F44C0020EE4C002077
:10094000344E0020BF4D0020D04D0020304E0020FE
:1009500002480078002800D001207047104D002088
:100960000148007970470000104D002070B517490C
:100970003CC80E4684B040363CC643680268806876
:100980004B65134C0A658865607C002818D00025EB
:1009900069460D72FAF792FCFFF7CCFD69460872C2
:1009A000E1690126002906D068460095067002A874
:1009B0000190684688476846007A002802D0267071
:1009C00004B070BD257004B070BD0000D44C002090
:1009D000104D002004490868401C0860012801D01F
:1009E0000120704700207047244000200349086818
:1009F000002802D0401E08600120704724400020DB
:100A0000F8B50C462849294B4118294F294A002698
:100A1000069D002908D0012922D0274940180A281C
:100A20002FD301202870F8BD20780A2838D2214918
:100A300080000958214A914203D11E490E501E5090
:100A40002EE0B9422CD10322082311461C4807F49A
:100A500073D0217801706168416007F4A9D01FE06C
:100A600020780A281CD280001158B94218D1195890
:100A700011502078134962684018032107F41ED3EF
:100A80000EE0C0B20A280BD284001159002907D009
:100A9000B94205D0094FB94202D016511E518847BC
:100AA0002E700020F8BD0000FBF0FFFFAC4C0020D2
:100AB000A32C0101844C0020F9F0FFFFA12C0101BF
:100AC000060F0000070F0000F7B5534F38780028D5
:100AD00009D0042A09D2012211217B69009800F073
:100AE0009EF903B0F0BD002314E00C784E78204648
:100AF0008C783602CB783043240420431B061843FD
:100B0000CB780002000A1B0618437B690D1D141FD9
:100B1000984206D002221121009800F080F903B01B
:100B2000F0BDB8681E19864203D90322112100982E
:100B30006DE07E61F869B0420FD2F96978684018BB
:100B4000FAF7AAFB002801D0052207E00120F96985
:100B500000030818F861B042EFD30022002A3CD10C
:100B6000B86A002822D02D49042808D2002C1BD0B6
:100B70002B780B54401C641E6D1CB862F4E73E4693
:100B8000042811D1B1697068244B40180422194619
:100B9000FAF7B0FB002801D0052203E0B069001D80
:100BA0000022B0610020B062002A16D1042C1DD3AF
:100BB000BA697868A608B600801829463246FAF75E
:100BC00099FB002801D0052203E0B86980190022B2
:100BD000B861AD19A41B002A08D011217B690098C7
:100BE00000F01DF9FCF776F803B0F0BD002C05D03D
:100BF000224629460948F7F737FBBC62BB693A6AC7
:100C00000098190B9142EFD939620022112100F0AE
:100C100006F903B0F0BD0000584700207C470020D3
:100C2000F7B56F4D8CB028780B46002809D0042A00
:100C300009D0012212216B690C9800F0F0F80FB076
:100C4000F0BD002313E01A78D97810465A780906C7
:100C5000120210439A781204104308430402D87811
:100C6000240A000604436B69A868834206D0022266
:100C700012210C9800F0D3F80FB0F0BDA86A00263E
:100C8000002815D0042806D2564AFF211154401CD2
:100C9000A8620428FAD3AB69686852490422C018D4
:100CA000FAF728FB00287DD1A869AE62001DA86173
:100CB000A9686868FCF7AEFEA04202D1E9688842E4
:100CC00009D0042212216B690C9800F0A8F8FCF7F7
:100CD00001F80FB0F0BD6868001D00F08FF869687A
:100CE0000A460832904203D3AA688918814209D87B
:100CF000062212216B690C9800F091F8FBF7EAFFCD
:100D00000FB0F0BD384C6F460FCC0FC70FCC0FC7DC
:100D1000A268616820680A920890344F0098203CCD
:100D20000991B84206D128212046FCF773FE0A99A2
:100D300088420AD00096019602960396049605967C
:100D400006960796089609960A960097284A6968B3
:100D5000914201D1012000E00220019091426846B9
:100D600001D1083000E018300160A9684160E968ED
:100D700081602969C16028216846FCF74BFE0A9012
:100D80002046FAF789FA00280FD12C22694620461E
:100D9000FAF7B0FA002808D12C2221466846F7F766
:100DA000A6FA00E001E0002809D0052212216B69B3
:100DB0000C9800F034F8FBF78DFF0FB0F0BD002267
:100DC0001221AB680C9800F02AF8C82002F04CF809
:100DD000BFF34F8F08490748C860BFF34F8FFEE746
:100DE000584700207C4700200040000111C011CA74
:100DF000008000010400FA0500ED00E00378C278ED
:100E00001946437812061B0219438378C0781B04E5
:100E1000194311430902090A00060843704710B537
:100E200082B06C4621706270A370190AE170190CCF
:100E30002171190E6171014606236A461F20FBF7D6
:100E4000B3FC02B010BD000070B5FEF70BFCFCF760
:100E5000AFFC04002FD01A4D2889F7F7DBFE0246BD
:100E60000B4618A12046FCF757FCE868F7F7D2FEBE
:100E700002460B4614A12046FCF74EFC13480078AE
:100E8000F7F7C8FE02460B4611A12046FCF744FCCA
:100E90002046FCF79DFD05462046FCF795FC002DFD
:100EA00009D02846FCF7B4FE0BA0FCF7B1FE28469B
:100EB000FCF796FD70BD09A0FCF7AAFE70BD00000E
:100EC000AC5C00206C65640070776D008847002082
:100ED00076616C69640000000D0A00006A736F6E31
:100EE0003A20616C6C6F63206661696C0D0A0000CA
:100EF00070B5134C01256078002802D1FAF7DEF9AD
:100F0000657010483021FCF785FD0E490E4E0863D0
:100F10003046FAF7C1F900280DD13422094930468C
:100F2000FAF7E8F9002806D1342231460548F7F7E8
:100F3000DEF9002801D0012070BD2570002070BDB1
:100F400088470020AC5C002000600001F3B583B04E
:100F50000498002106688068009137187D1C305C79
:100F60002C4622287ED10498406807E05C2A04D1F0
:100F70005B1C834277D2491C641C641CA31B834204
:100F800002D22278222AF1D1A21B82426BD220788F
:100F9000222868D1E01B401A0499401C096988473F
:100FA000009000285ED0A54270D229785C2903D039
:100FB0000170401C6D1CD8E00223611B012952DB2B
:100FC0006A78662A15D008DC222A22D02F2A20D05F
:100FD0005C2A1ED0622A46D108E06E2A0DD0722A01
:100FE0000FD0742A11D0752A3DD115E00821017067
:100FF00010E00C210170401CB6E00A210170401C79
:10100000B2E00D210170401CAEE009210170401CCE
:10101000AAE00270401CA7E00022944606296FDB7C
:10102000AF1C1346F95C0E46303E092E02D8303A0A
:101030008A180BE00E46413E052E01D8373A04E0EF
:101040000E46613E052E1FD8573A8A18032B00D250
:1010500012015B1C042BE5D337218902531A554931
:101060008B4201E09CE094E07BD91B23DB02D31A86
:101070008B423FD80C23A91D9E46631A062B70DBBA
:101080000B785C2B6DD102E00022E5E770E04B7835
:10109000752B66D1891C019100210E46019B9B5D39
:1010A0001F46303F092F02D8303959180BE01F4630
:1010B000413F052F01D8373904E01F46613F052F16
:1010C00016D857395918032E00D20901761C042E60
:1010D000E4D337239B02CE1A01239B029E4240D2C7
:1010E00092058905120B890D0A439901521803E0F4
:1010F0000021EEE706218E46802A02D2012315E068
:101100002FE00121C9028A4203D20223C0218C466A
:101110000CE0012109048A4202D20323E02104E009
:1011200025498A421DD80423F0218C46591E090600
:10113000090E0AD0164680273E43BF273E4046543C
:10114000491E92090906090EF4D1012B03D9614603
:101150000A43027002E05106490E0170C01873463E
:1011600000E00023002B14D0ED18A54200D21CE7AC
:101170000021017003981021C16003990098086153
:10118000049804990068201A401C8860012005B06A
:10119000F0BD0098002803D0049841690098884762
:1011A000002D04D004980068291A0498816000205A
:1011B00005B0F0BDFF030000FFFF1000F0B591B0D7
:1011C0000C0006467ED0216800297BD0A0686368A9
:1011D000021D9A4206D808180422DBA1F7F79DF8F1
:1011E000002833D0A0686268411D914207D8216869
:1011F00005220818D6A1F7F790F800282ED0A0688D
:101200006268011D914207D8216804220818D2A102
:10121000F7F783F8002829D06268A168914203D2C9
:101220002068405C22282BD091427AD22068405C12
:101230002D2802D03038092873D80020014610909C
:1012400020682E22002807D06B464DE00420F06075
:10125000A068001DA060012011B0F0BD0120F06069
:10126000A068401DA060012011B0F0BD0220F06018
:1012700001207061A068001DA060012011B0F0BDC8
:1012800021463046FFF762FE11B0F0BD25682818F0
:10129000085C342820D00DDC05462B3D092D28D2D2
:1012A0002F007F443F79FF19BF44162316182316D9
:1012B0001616160038280FD008DC35280CD0362832
:1012C0000AD000E074E0372813D105E0392803D0B4
:1012D000452801D065280CD1585400E05A54491CC7
:1012E0003F2906D2002C04D0A06867684518BD428B
:1012F000CCD30020585410A9184601F0C3FC0F4667
:10130000054610996846884252D0F761944A954B39
:1013100028463946B561F7F71FFD03D8924870613A
:101320000FE019E00022914B28463946F7F700FDFF
:1013300002D80120C00703E028463946F7F7A0FC91
:1013400070610820F060109AA1686846101A0818A9
:10135000A060012011B0F0BD7D20C000914203D2F9
:1013600023685B5C5B2B06D0914279D22268515C8A
:101370007B2967D074E00027E1683D4681426FD247
:10138000491CE1602168A068095C5B2968D1401CA8
:10139000A0602046FCF7A2F96168A068884203D2E9
:1013A0002268125C5D2A38D0884202D3401EA060B9
:1013B00056E0401EA060204610300090FCF76EFA08
:1013C000002839D0002F23D0286045600546A0684A
:1013D000401CA0602046FCF781F921462846FFF713
:1013E000EDFE00282AD02046FCF778F9002C25D005
:1013F0006168A068884203D22168095C2C290AD060
:10140000626890421AD22168085C5D2816D104E017
:1014100007463D46DBE70098D0E7E068401EE06005
:10142000002F00D07D602020B760F060A068401CD5
:10143000A060012011B0F0BD002F11D03846FCF79C
:10144000C3F90DE00027E1683D46814208D2491CFE
:10145000E1606168A068884202D2115C7B2902D0F9
:10146000002011B0F0BD401CA0602046FCF736F90A
:101470006168A068884203D22268125C7D2A4CD041
:10148000884293D2401EA060204610300090FCF7A6
:1014900005FA002855D0002F4ED02860456005463B
:1014A000002CCBD0A0686168401C8842C6D2A060E6
:1014B0002046FCF713F921462846FFF747FD002890
:1014C000BCD02046FCF70AF9286928620020286170
:1014D0006168A0688842B1D22168095C3A29ADD11F
:1014E000401CA0602046FCF7F9F821462846FFF78B
:1014F00065FE0028A2D02046FCF7F0F86168A068DD
:10150000884203D22168095C2C2918D06268904275
:1015100094D22168085C7D2890D1E068401EE0608C
:10152000002F00D07D604020B760F060A068401CB4
:10153000A060012011B0F0BD07463D46B0E700981D
:10154000A5E7002F8CD079E76E756C6C0000000069
:1015500066616C73650000007472756500000000C0
:101560000000C0FFFFFFDF41FFFFFF7F0000E0C181
:10157000102819D230B40D4C83001B199D698903C2
:101580002D0B2D03090D0D439D619969084D92099D
:1015900092052940920A11439961012261698240B2
:1015A0001143616130BC7047704700000020024069
:1015B000FF0FC0FFF3B5054681B00026408800F05C
:1015C00003F901000AD01C4F6A880020142343430A
:1015D000DB195B8A934203D142262AE0402628E0A9
:1015E000401CC0B20A28F1D3002E22D100241420BE
:1015F0006043C019408AFF2806D0641CE4B20A2C5C
:10160000F5D30A2C14D014E028460830009014209A
:101610006043C0190E686B78AA880746A91DB047B9
:101620000600EED1688878820298398A0180E8E75E
:101630004B26304603B0F0BD684B002002885004B2
:10164000400CD20B01D009020843704710B40024AB
:10165000094A214614234B439B185B8A834204D1D9
:10166000142041438818C46803E0491CC9B20A2900
:10167000F0D3204610BC7047684B002030B4FF23E5
:10168000040AC5B20A490020142242435218128AA1
:10169000AA4204D1142250434018438A03E0401C5C
:1016A000C0B20A28F0D3200230BC184370470000B3
:1016B000684B0020084A11780A290AD2C9004368F9
:1016C000891800688B6048601078401C10700120F9
:1016D0007047002070470000304C002030B4FF23DA
:1016E000040AC5B20A490020142242435218528A01
:1016F000AA4204D1142250434018038A03E0401C3C
:10170000C0B20A28F0D3200230BC18437047000052
:10171000684B0020F1B582B00299294E00200029C3
:1017200000D1307000250298002804D0012834D060
:1017300002283ED10FE0294614225143214A28466F
:1017400009308C182082C0B206F424D3207C2146B4
:1017500006F406D32DE028461421484319490023F6
:101760004718B87C009030781C4600280DD9E0005E
:101770008019828800998A4202D180688047034696
:10178000641C3078E4B2A042F1D8002B02D0596832
:1017900038468847387C06F421D31422094B6A4323
:1017A0000021D018FF24C16044829950416001811A
:1017B00041816D1CEDB20A2DB5D303B0F0BD000020
:1017C000304C0020684B002070B50146094DCEB268
:1017D00000202978044600290BD9E10049198A889C
:1017E000B24201D188688047641C2978E4B2A142E2
:1017F000F3D870BD304C0020F7B500248AB00094B7
:101800000194029403940E4604940594069407945C
:101810000894FF2701371168154638468847059612
:1018200001970090AA686968286806900098089255
:10183000079100283CD069460A9800F0CDF80028AE
:1018400030D00098002806D002994018F6F730FDF5
:10185000029940180290AA68002A07D002990098BD
:10186000491C904706001DD0009418E00298296892
:10187000401C8847060015D002980199401C8142FF
:1018800001D20A4601E0029A521C30460099F6F74E
:10189000EBFC0298345469680098884700943046FD
:1018A0000DB0F0BD0098002802D069688847009408
:1018B00000200DB0F0BD0000F8B500240A46054632
:1018C000002910D0002D10D001460078002826D025
:1018D00008780C283BD015DC082838D0092836D0E9
:1018E0000A2815D133E00020F8BD03211046FCF78B
:1018F000BDFB0028F8D022210170417000218170C9
:101900000120F8BD0D2822D0222820D05C281ED02E
:10191000202800D2641D4878491C0028D8D1481BD3
:101920000719F91C1046FCF7A1FB061EE9D0002C94
:101930000FD0222030702878741C002834D0C0B218
:101940001F2813D9222811D05C2837D10EE0641C3F
:10195000E1E7222434703A462946701CF6F784FCED
:10196000F0194470002181700120F8BD5C202070C6
:101970002A78641C0C2A23D006DC082A1DD0092AE8
:1019800024D00A2A06D11DE00D2A1DD0222A12D009
:101990005C2A13D00EA12046F9F7F2FE241D6878C8
:1019A000641C6D1C0028CAD12221F019417000214D
:1019B00081700120F8BD222000E062202070EEE757
:1019C0006620FBE76E20F9E77220F7E77420F5E761
:1019D0007525303478000000002801D0002901D19D
:1019E00000207047F0B50546007B8BB00C461028F0
:1019F0007ED008DC012819D0022821D0042809D083
:101A0000082876D128E0202874D0402873D0802878
:101A10007DD19BE005212046FCF728FB002803D060
:101A2000DCA1F7F7FDFD01200BB0F0BD062120463B
:101A3000FCF71CFB0028F7D0D8A1F7F7A9FD08E0B8
:101A400005212046FCF712FB0028EDD0D5A1F7F7C1
:101A5000E7FD01200BB0F0BD07910024AF69EE69EE
:101A600000942E2001940394049405940294069407
:101A70000894314609940A90002F01D0012000E01B
:101A8000002001434800C9494008081AC00F14D17A
:101A9000012170004905C84201D1002F0DD06869AD
:101AA000F7F7A4F83A463346F7F742F90BD1C0A14D
:101AB00068466A69F9F764FE26E0BEA16846F9F750
:101AC0005FFE054621E03A463346BCA16846F9F779
:101AD00057FE054608AABBA16846F6F72DFC01286B
:101AE0000CD13A46334609990898FCF7A3F803E06D
:101AF0003EE00CE041E094E0002806D13A4633464F
:101B0000B1A16846F9F73CFE05461A2D02D3002024
:101B10000BB0F0BD691C0798FCF7A8FA0028F7D0B5
:101B2000002D0BD92E236A46115D0A9EB14201D1C8
:101B3000035500E00155641CAC42F5D3002101556A
:101B40000798806841190798816082E72869002812
:101B5000DED0F6F7ADFB401C064601462046FCF7FA
:101B600085FA0028D4D032462969F6F77DFB70E764
:101B70002869FFF7A1FE0BB0F0BDAD68012120463A
:101B8000FCF774FA0028F6D05B210170A068401CB5
:101B9000A060E068401CE060002D34D000262146A3
:101BA0002846FFF719FF002813D0002C09D0206821
:101BB000002806D0A1684018F6F77AFBA168411802
:101BC000A160286800281BD06069002804D0022783
:101BD00003E030460BB0F0BD0127791C2046FCF72E
:101BE00045FA0028F5D02C2101706169401C0029BC
:101BF00002D020210170401C0670A068C019A060AE
:101C00002D68002DCBD102212046FCF72FFA0028A9
:101C1000E0D05D21017000214170E068401EE0606D
:101C200017E76069AD68002801D0022700E00127AE
:101C3000791C2046FCF71AFA0028CBD07B210170D2
:101C4000E168401C491CE16062690A21002A00D059
:101C50000170A068C019A060002D78D000276069CD
:101C6000002814D02046E168FCF700FA002825D0AF
:101C7000E2680021002A06D909220270E368401CAC
:101C8000491C8B42F9D8E168A0684018A060214641
:101C9000286AFFF711FE002810D0002C09D0206818
:101CA000002806D0A1684018F6F702FBA168411889
:101CB000A1606069002804D0022603E038460BB01A
:101CC000F0BD012631462046FCF7D0F90028F5D0BA
:101CD0003A2101706169401C002901D0092101707D
:101CE000A06821468019A0602846FFF775FE0028ED
:101CF000E4D0002C09D02068002806D0A168401844
:101D0000F6F7D6FAA1684118A1606069002800D0F2
:101D100001202968002900D001214618711C2046A5
:101D2000FCF7A4F90028C9D02968002902D02C2189
:101D30000170401C6169002902D00A210170401C19
:101D40000770A0688019A0602D68002D87D1606998
:101D5000002802D0E168491C00E002212046FCF77F
:101D600085F90028ABD0616900290BD0E268002119
:101D7000012A07D009220270E368401C491C5B1E3F
:101D80008B42F8D87D21017000214170E068401E2F
:101D9000E0605EE66E756C6C0000000066616C735E
:101DA0006500000074727565000000000000F07F9F
:101DB000256400006E756C6C0000000025312E312A
:101DC00035670000256C670025312E31376700002C
:101DD00070B505460078002813D00A4E2846F6F75D
:101DE00067FA84B20D2C00D90D2471782346481C63
:101DF00070702A460220FAF7D7FC2D19287800289F
:101E0000ECD170BD4C470020F8B5069E1F46182E39
:101E100001D9182500E0354613460A4601460CA0B4
:101E20000096F9F79DFC0024002D07D9395D11A01B
:101E3000F9F796FC641CA4B2AC42F7D3AE4202D9C7
:101E40000EA0F9F78DFC0FA0F9F78AFCF8BD000091
:101E50005B424C452025735D20747970653D307878
:101E600025303258207365713D2575206C656E3DB7
:101E7000257500002025303258000000202E2E2E1F
:101E8000000000000D0A0000F8B5134E0F467569FA
:101E900004463068001D00F005FF601C07D1002FCC
:101EA00005D031680D48091D00F089FFF8BD306884
:101EB0002C1944603168AC4204D2B068091D00F0AE
:101EC00065FFF8BD7068091D00F060FF306B84424B
:101ED000F7D23463F8BD0000A4470020BC5D0020A9
:101EE000F8B5856B164604460027026C002A11D00F
:101EF000002E19D0E068F6F7B7F9216CE068401AB7
:101F0000E0602268904202D26068401AE060022ECF
:101F100017D019E02068002816D1606801F056FD3E
:101F20000746002060600FE0A068F6F79DF9216C7D
:101F3000A0684018A0606168884205D32068A0604E
:101F400002E0002D00D06D1E6D1CA5633846F8BD63
:101F5000114D124E124FE868002817D000F03CFFD8
:101F6000F068C468201D00F09DFE2869401E2861AD
:101F7000E868401EE86000F03BFF206B00F046FF81
:101F8000204600F043FFE8680028E7D138680128C0
:101F9000E1D900F05DFFDEE7A4470020A85D002046
:101FA000E05C002030B4124900E011460A68824229
:101FB000FBD34B685C18844203D140681818486012
:101FC000084643681C1894420CD10A4C2468A2426B
:101FD00006D052689A1842600A681268026002E0ED
:101FE000046000E00260814200D0086030BC7047AD
:101FF000F0470020E0470020F7B582B003980026A4
:102000000068002859D003984168024649680832A0
:1020100041600092914201D1496841604068C068C6
:1020200001900398416849684160009A914201D14A
:1020300049684160CF68242002997043441804988D
:102040003D46002F01D11E490D68256029463431D7
:102050006160E96A2161296BE161696CA16000231B
:10206000E96CA3616161052813D015490A6895429E
:1020700001D1237311E0207303280ED1886B401C1B
:102080008863A86A002801D00220207301F040FD77
:1020900003E02846FBF7BAFF2073286B0021027883
:1020A000A52A04D14278401C491CA52AFAD08808E8
:1020B00020840198761C8742B3D1304605B0F0BD2C
:1020C000A447002003480068401C72B600D0FEE719
:1020D000FEE70000F8470020F8B5054600F07CFE5A
:1020E0002E46403605243457002C0FDD2F4624376A
:1020F000686A00280AD0384601F0D8FC002801D0D0
:1021000000F03AFF641E64B2002CF1DC0027FF43AC
:10211000777100F06DFE00F05FFE04243457002C50
:1021200010DD284610300090286900280AD0009859
:1021300001F0BCFC002801D000F01EFF641E64B258
:10214000002CF1DC377100F053FEF8BDF8B5044601
:10215000002500F08BFF374E00273068364A0028F4
:1021600001D0F0681BE0052134480903430705D07E
:10217000C01DC008314BC000C31AC91A4118083924
:10218000C908C9005760106031604F600B1A0F60BA
:1021900043600160B3600120C0077360F0600442D7
:1021A0003FD1002C3DD020460830410708D04107E0
:1021B000490F0823591A0818410701D072B6FEE7E3
:1021C00000282ED0716888422BD81B49146801E082
:1021D000214614466268824202D22268002AF7D160
:1021E000326894421DD00D6822680A606168083523
:1021F0000A1A102A09D921184B0701D072B6FEE736
:102200004A6060600846FFF7CDFE61687068401A5A
:102210007060B268904200D2B060F06827600143FD
:10222000616001F075FC680701D072B6FEE72846D0
:10223000F8BD0000E0470020F0470020D05D0020FE
:1022400004490868002803D00868026D521C026522
:1022500008687047A447002010B40124031F240617
:102260001C601B1F1960191F034B0B6014390A6097
:1022700010BC403870470000C520010170B506460B
:1022800014460D464720FFF7E1F90369002B0DD0F6
:102290001879B04207D158792880981D2060002B0A
:1022A00004D0002070BD1B68002BF1D100202880D5
:1022B00020600A2070BD000070B516460C4610461E
:1022C00005F4F8D4002813D14720FFF7BFF90546DD
:1022D000062332461946074805F42ED4A988628899
:1022E00089180180A1884180A179017105F460D429
:1022F000002070BD180C0000F7B506460D464720BB
:10230000FFF7A4F904690746002C14D02079B042E5
:102310000BD16079A8420CD0384621461030F7F72F
:102320005BF9204605F4F8D205E02468002CEDD1D5
:1023300001E0002C0AD128460121083005F476D3AB
:102340000446014638461030F7F74CF9267165719E
:102350002A46A01D0299F5F787FF002003B0F0BDC3
:10236000F8B5C5680124287F0F4601281ADD0E4EF6
:102370002046162250430246296A10328A5A5204D5
:10238000920F0BD10A5C401C085C00021018B0428E
:1023900004D1E1B20022384600F03EF9287F641CE7
:1023A000A042E5DCF8BD000002290000F8B5C568D0
:1023B0000124287F0F4601281ADD0E4E20461622E2
:1023C00050430246296A10328A5A5204920F0BD1A6
:1023D0000A5C401C085C00021018B04204D1E1B253
:1023E0000022384600F018F9287F641CA042E5DC82
:1023F000F8BD00000229000070B5C46805462069D8
:10240000002803D00020002802D00EE00120FAE7C7
:10241000264610363046F7F7CDF805F47DD2206910
:10242000002808D000210029F4D00020E8602046D0
:1024300005F472D270BD0121F5E710B504464720BE
:10244000FFF704F982790021A24202D9808800199D
:1024500081B2084610BD70B504460D464720FFF70F
:10246000F5F8014680888022A04206D88979411873
:10247000A14202D9201A28700022104670BDFFB573
:1024800085B00E9D0646297801208840401E0490A4
:1024900018460E210840328A69681F464030019272
:1024A00000230390009302912B7804AAA968069850
:1024B000F7F7BCF8009000282AD10121282005F464
:1024C000B5D20446AA686968286862622162E06140
:1024D000F46006980188A180217FA171F80701D0DE
:1024E0000120C003079908432080308A608047207C
:1024F0007082304600F0AAF820461030F7F766F8F0
:10250000217F206A00F008F8308A002105F4E4D326
:10251000009809B0F0BD0000F3B583B00020019031
:1025200004980125012845DD1621039A694388187E
:10253000028A5204920F39D1039A4078515C00020A
:1025400009181D48814231D101A80290EFB204263A
:102550004720FFF77BF800900469002C14D0207905
:10256000B8420BD16079B0420CD0009821461030AF
:10257000F7F732F8204605F4CFD105E02468002CA7
:10258000EDD101E0002C0AD130460121083005F4DC
:102590004DD20446014600981030F7F723F8277112
:1025A00066713246A01D0299F5F75EFE04986D1C17
:1025B0008542B9DB05B0F0BD022900000048704734
:1025C000C041010170B5064610480D46007800284C
:1025D0001AD04720FFF782F8A91D8BB201460322CB
:1025E0000B4805F4A9D204460A482A468078207090
:1025F0000120607005206080A5803146A01DF5F7A0
:1026000033FE204605F4D4D270BD000037470020C9
:1026100006470000B04D002070B584B00E46144649
:10262000054601AA69463046FFF728FE684602883B
:1026300002A80199F5F718FE02A84455024668461B
:1026400001883046FFF758FE04B070BD10B504464F
:102650004720FEF7FBFF0449216009216181183002
:1026600060600120208110BDD0410101FFB583B021
:102670000C464720FEF7EAFF0546808861882678E9
:10268000401887B2059805F415D3012807D03846BD
:10269000FCF71AFE6946FFF7DEFE002802D0022092
:1026A00007B0F0BD0121059805F416D30C3C0020BD
:1026B000AC60287368460078687301AA02A9FFF726
:1026C000DDFDA86801990446895D0C34890720D591
:1026D000A188C28808318BB23102C1200001891D56
:1026E00005F42AD2064613203070A8886188401865
:1026F000B080A088F0803046A288A11D0830F5F790
:10270000B3FD304605F454D20121059805F4E4D216
:1027100001E005F401D1012007B0F0BD10B5FAF7D2
:1027200037FD002010BDFFB583B00C464720FEF7F3
:102730008DFF0546808861882678401887B2059805
:1027400005F4B8D2012807D03846FCF7BDFD69462C
:10275000FFF781FE002802D0022007B0F0BD0C3C3C
:10276000AC602E7368460078687301AA02A9FFF76F
:1027700085FDA86801990446895D0C34890720D03D
:10278000A188C28808318BB23102C1200001891DA5
:1027900005F4D2D1064612203070A888618840180E
:1027A000B080A088F0803046A288A11D0830F5F7DF
:1027B0005BFD304605F4FCD10121059805F48CD26F
:1027C00001E005F4A9D0012007B0F0BD10B50C461A
:1027D0004720FEF73BFF80886188A31D401880B228
:1027E000A1880022FAF76CFC002010BDF8B54888DB
:1027F00000900C468E88F9F7EBFE00281DD0182EAD
:1028000001D9182700E03746324623A00099F8F78F
:10281000A7FF0025002F08D96019817927A0F8F7B4
:102820009FFF6D1CADB2BD42F6D3BE4202D925A0BA
:10283000F8F796FF25A0F8F793FF009802281FD01D
:10284000062802D0082824D11FE0022E21D1E088DA
:102850001F49012802D0002808D01AE00120087082
:10286000F9F7B6FE002814D01AA006E00020087080
:10287000F9F7AEFE00280CD01CA0F8F771FF08E0B5
:10288000A188A01DF9F7C0FE03E0A188A01DF9F7FB
:10289000FFFD0020F8BD00005B424C455D207772D3
:1028A00069746520696E643A206174745F69647844
:1028B0003D2575206C656E3D257500002025303264
:1028C00058000000202E2E2E000000000D0A0000EF
:1028D000374700205B424C455D206E6F7469667916
:1028E00020656E61626C65640D0A00005B424C45B8
:1028F0005D206E6F746966792064697361626C65CE
:10290000640D0A00FFB581B000276846078048883B
:102910001C460D46082823D00A2825D005206946E4
:10292000088014A6684600882146083083B2134800
:10293000039A05F401D1877129780446017068462D
:102940000288A28069886180002A03D03146E01D98
:10295000F5F78AFC204605F42BD1002005B0F0BD28
:102960006846F9F70BFE02E06846FAF729F90646D1
:10297000D8E700004E53494E4700000005470000CD
:1029800070B516460C46104605F494D1012818D1AE
:10299000A1791A48002916D0217806230902324667
:1029A000891D05F4C9D00546A078FFF746FD2880AB
:1029B00080202871284605F4FBD00021304605F41C
:1029C0008BD1002070BDA1883246891D8BB2217841
:1029D0000902891D05F4B0D00546A078FFF72DFD4A
:1029E000288000202871A0886880A288E11D681DC9
:1029F000F5F73AFC284605F4DBD0DEE7140C0000BE
:102A0000F3B583B005001AD02868019028468038B5
:102A10000290C76F04983E1F864200D9064628469A
:102A2000F8F7F4FE04460091324629460498FCF774
:102A300031FE0199002806D0016005B0F0BD049870
:102A4000F8F716FFF9E729600299002CCF670AD042
:102A500021686218291F8A4202D9291B091F216097
:102A600000996160E9E7024A00991160E5E700001A
:102A70000048002010B5012400206407206004F401
:102A8000B1D72E4802882E480168002005F436D0C0
:102A90002C4802882C480168012005F42FD02B48CF
:102AA000008882B22A480168022005F427D029480C
:102AB000008882B228480168032005F41FD0274807
:102AC000416AF02211434162254818F409D0264892
:102AD0002449016025494161254981602549C1603A
:102AE000254981612549C161264925488863FCF74C
:102AF0002BFE2068C0B2F6F79FFD2348007800281F
:102B000006D0002018F432D301460020F6F79AFDD3
:102B10002068C0B2F6F79CFDF6F7A0FD2068C0B2B1
:102B200018F4B0D02068C0B218F4BAD02068C0B28F
:102B300018F478D20120206010BD00001C01002094
:102B40001801002024010020200100203401002071
:102B5000300100202C0100202801002040250240E7
:102B600074020020500250008080024000080F00D4
:102B700058086A00420500000F0505060F000F0304
:102B80004000D0004080024062000020F0B5314C8F
:102B900083B0E06980075AD502202062A56B082027
:102BA00018F488D3012018F493D32B49002708691F
:102BB00040194608B219801A086128480068F6F7DB
:102BC00029F80022264BF5F77BFF019100903E216A
:102BD0002846F6F749FD80197941F6F729F8019B57
:102BE000009AF5F705FFF6F76FF805461D4A002332
:102BF000F5F7F2FA06461B49F6F736FD1A49281A88
:102C0000081A81B222041948324342600160206BE5
:102C10000821884308432063A069072109078843E6
:102C2000A061A169012081430143A1612062FCF7F9
:102C30008BFD0F48104A0078410041180D480818D4
:102C40004178D1610D498078C8600D48077003B0A4
:102C5000F0BD000000800240A8020020900000208B
:102C600000408F407102000070020000408002406E
:102C700010400020E0400101402502408025024034
:102C80008000002000B50A4683B000210091019128
:102C900001466846F6F7B7F90199009803B000BD00
:102CA000704770474368826801699A608368426828
:102CB0005A604A68824201D182684A6000220261F9
:102CC0000868401E086008687047000001480069F5
:102CD00070470000A4470020F8B51746204A064672
:102CE0000024906B0725401C90631069814232D309
:102CF00014206D1E1B49684341182420604380192D
:102D00000122FFF779F90419002DF1D12420144D87
:102D10006043801902226968FFF76EF904192420C4
:102D2000604380190222A968FFF766F9041924207C
:102D30006043801904220C49FFF75EF9041924202E
:102D40006043801903220949FFF756F90419002F3F
:102D500001D00020386000F0DBFE2046F8BD000006
:102D6000A4470020E05C0020A85D0020BC5D00209E
:102D70000146083100224160D243C1608260016196
:102D800000210160704700210161704730B40C6878
:102D9000621C02D00246083202E0026904E01A46D0
:102DA00053681D68A542FAD953684B6099608A60E0
:102DB000516008610168491C016030BC704742687D
:102DC0004A6093688B6093685960916008610168FC
:102DD000491C01607047000072B604480168491C34
:102DE0000160BFF34F8FBFF36F8F7047F84700202C
:102DF00005490868002804D0401E086000D162B66A
:102E0000704772B6FEE70000F847002000281CD08B
:102E100070B504460D4D083C6068E968084201D170
:102E200072B6FEE72268002A01D072B6FEE7884338
:102E3000606000F01BF960686968401868602046AF
:102E4000FFF7B0F800F064FE70BD7047E047002067
:102E50000120044900074860BFF34F8FBFF36F8F15
:102E60007047000000ED00E010B500280FD00949C0
:102E70008A6B002A01D072B6FEE78A6B521C8A6305
:102E80000021FFF701F800F043FE002801D1FFF711
:102E9000DFFF10BDA447002002498A6A0260496929
:102EA00041607047A4470020F0B585B00027054673
:102EB00007702C4801690291006924214843FFF7FB
:102EC00045F906004CD000220299FFF705FF039751
:102ED0000290002841D90398242148438019017B9E
:102EE000052911D20A007A441279921897440204F3
:102EF00006080A00582408E0522406E0422404E0B0
:102F0000532402E0442400E0002441682846F5F7F9
:102F1000FBF92846F5F7CCF90F2804D220212954D3
:102F2000401C0F28FBD32F542D180398242148430D
:102F30008019018C826801920091036922460AA1DE
:102F40002846F8F71DFC2846F5F7B2F9451903980D
:102F50000299401C03908842BDD33046FFF756FFCC
:102F600005B0F0BDA4470020092563092575092592
:102F7000750925750D0A0000014901204862704756
:102F8000A447002010B50C46002809D0054909685F
:102F90001831FFF7FBFE01212046FEF775FF10BD3B
:102FA00072B6FEE7A447002070B50B4604002FD090
:102FB000226D002A0ED0E16C994200D21946E06AD7
:102FC000884225D0012A23D1124D2A68944203D188
:102FD00072B6FEE772B6FEE7E162A269002A02DB82
:102FE0000722511AA16114220B4E504361698019C6
:102FF00081420DD1201DFFF755FEE06AA969884284
:1030000000D9A861142148438019211DFFF7D7FE7C
:1030100070BD0000A4470020E05C002010B582B025
:103020000D4800240190234680220CA100940D48F5
:1030300000F090FB012803D0401C0BD172B6FEE7D4
:1030400072B600210848C94301630121C16144618E
:1030500000F052F802B010BDD847002049444C455A
:1030600000000000511F0101A44700200248816BAD
:10307000491C816370470000A4470020164B986BE1
:10308000002802D0012058627047002058629869D9
:10309000142102464A4311498A58002A0AD10028BD
:1030A00006D01422401E42438A58002AF7D001E07D
:1030B00072B6FEE7142210B4424351184A680C4617
:1030C000526808344A60A24201D152684A60D1680D
:1030D0001960986110BC7047A4470020E05C002094
:1030E0000148406870470000E047002001488068C0
:1030F00070470000E047002070B50F48016AFF22CA
:10310000120411430162016A1202114301620B4C65
:1031100000252561A5610A487D21C9000068F5F7F1
:1031200031F8401E60610720206106480560F4F711
:10313000DFFF002070BD000000ED00E000E000E0D7
:1031400000400020F847002010B502460021012071
:1031500000F00CF8041E07D00021416001600B460E
:103160000A46C16000F05BF8204610BDF8B517466E
:103170000E46050016D0002E16D070435030FEF7D4
:10318000E5FF04000CD020465030002E0ED0206009
:10319000266420460121E56300F00AF84C2007551B
:1031A0002046F8BD72B6FEE70020E7E72460EFE7AF
:1031B00070B50D46040026D0FFF70EFE216CE06BC3
:1031C00048432168411861600021A1632168A16022
:1031D000E06B216C401E48432168224641180020C4
:1031E000C0434032E1601071507120461030002D14
:1031F0000BD0FFF7BDFD20462430FFF7B9FDFFF7E8
:10320000F7FD012070BD72B6FEE721690029F6D0F6
:1032100000F04CFC0028F2D0FFF71AFEEFE7FFB5F4
:10322000002783B00446002803D00498002802D069
:1032300006E072B6FEE7206C002801D072B6FEE709
:103240000698022804D1E06B012801D072B6FEE78F
:1032500000F03CFB002804D10598002801D072B68C
:10326000FEE720462546103040350290FFF7B4FDBA
:10327000A06BE16B884208D30698022805D0059818
:1032800000284AD0002F4BD04EE0069E0499A56B33
:103290000027226C002A11D0002E19D0E068F4F724
:1032A000E3FFE168206C091AE1602268914202D2D2
:1032B0006168081AE060022E17D019E02068002823
:1032C00016D1606800F082FB0746002060600FE0C6
:1032D000A068F4F7C9FF216CA0684018A06061687D
:1032E000884205D32068A06002E0002D00D06D1E4A
:1032F0006D1CA563606A002806D02046243000F0CB
:10330000D5FB002802D103E0002F01D0FFF7A0FD7C
:10331000FFF76EFD012007B0F0BDFFF769FD20E06B
:103320006846FFF7B9FD0127FFF762FDFFF79EFE34
:10333000FFF752FD04202856401C00D128710520BB
:103340002856401C00D16871FFF752FD05A9684658
:1033500000F0CEF9002807D02046FEF7BDFE00F0B1
:10336000D7FB002007B0F0BDFFF736FDA06BE16B87
:10337000884201D1012600E00026FFF739FD002E2A
:103380000ED005990298FFF7FDFD2046FEF7A4FE3A
:1033900000F0BEFB002800D068E7FFF759FD65E7A5
:1033A0002046FEF799FE00F0B3FB5FE7FFB583B060
:1033B0001E461746040003D00498002802D006E0F9
:1033C00072B6FEE7206C002801D072B6FEE7022E2E
:1033D00004D1E06B012801D072B6FEE7F4F79CFE41
:1033E0000190A06BE16B884208D3022E06D0002426
:1033F0000198F4F795FE204607B0F0BD2046403016
:10340000052500904557324620460499FEF768FD91
:10341000681C04D000986D1C45710124E8E7606ABF
:103420000028FAD02046243000F040FB0028F4D0D9
:10343000002FF2D001203860EFE7F7B5002784B005
:103440000446002803D00598002802D006E072B692
:10345000FEE7206C002801D072B6FEE700F036FAD5
:10346000002804D10698002801D072B6FEE7204655
:103470002546243040350290FFF7AEFCA66B002EA7
:1034800021D0226C059B002A0BD0E0688018E060F8
:103490006168884201D32068E06001461846F4F76D
:1034A000E3FE761EA6632069002807D02046103070
:1034B00000F0FCFA002801D0FFF7CAFCFFF798FCE7
:1034C000012007B0F0BD0698002802D0002F05D0DB
:1034D00008E0FFF78DFC002007B0F0BD6846FFF75D
:1034E000DBFC0127FFF784FCFFF7C0FDFFF774FC4E
:1034F00004202856401C00D1287105202856401C65
:1035000000D16871FFF774FC06A9684600F0F0F876
:10351000002811D02046FEF7DFFD00F0F9FAFFF792
:103520005BFCA06B002827D00026FFF761FC002E73
:10353000A2D0002007B0F0BDFFF74EFCA06B002822
:1035400012D00026FFF754FC002E0FD006990298E7
:10355000FFF718FD2046FEF7BFFD00F0D9FA00285E
:103560008AD1FFF775FC87E70126EBE72046FEF7D7
:10357000B3FD00F0CDFA7FE70126D6E7F3B50027CB
:1035800085B004460097002804D0206C002803D0A2
:1035900072B6FEE772B6FEE700F098F9002804D193
:1035A0000698002801D072B6FEE720462546243052
:1035B00040350190FFF710FCA06B002817D0401E8B
:1035C000A0632068002802D1FEF73AFE60602069FF
:1035D000002807D02046103000F068FA002801D0FB
:1035E000FFF736FCFFF704FC012007B0F0BD06989A
:1035F000002802D0002F0AD00DE00098002801D04A
:1036000072B6FEE7FFF7F4FB002007B0F0BD02A89A
:10361000FFF742FC0127FFF7EBFBFFF727FDFFF762
:10362000DBFB04202856401C00D1287105202856B9
:10363000401C00D16871FFF7DBFB06A902A800F06F
:1036400057F800281BD02046FEF746FD00F060FA30
:10365000FFF7C2FBA06B00283ED00026FFF7C8FB97
:10366000002EA7D0009800283ED0FFF7B5FB606A77
:10367000002833D0206B07210068091A2FE0FFF7DC
:10368000ABFBA06B002808D00026FFF7B1FB002E93
:103690001CD02068002802D009E00126F5E7FFF7DA
:1036A0009BFB606800F0C6F90090FFF7A1FB06994C
:1036B0000198FFF767FC2046FEF70EFD00F028FAA0
:1036C000002800D076E7FFF7C3FB73E72046FEF73C
:1036D00003FD00F01DFA6DE70126BFE700216068D9
:1036E000FFF762FCFFF784FB002007B0F0BD00008D
:1036F000F8B50D46040012D0002D12D0FFF76CFB78
:10370000134E726963682868D11A471C0BD027686A
:10371000B66AB74209D0934207D8012413E072B6C3
:10372000FEE772B6FEE700240DE0884208D9401A91
:1037300028600748816A216040696060002402E0D7
:10374000002001242860FFF753FB2046F8BD00004D
:10375000A4470020FFB585B090000F9F0E9D0290FA
:10376000FEF7F4FC06001ED05C20FEF7EFFC040020
:1037700016D0266305990191089900913046029967
:10378000069EA5220391F4F781FD0399206B091F82
:103790004018C008C0000290400708D072B6FEE78B
:1037A0003046FFF733FB0020C04309B0F0BD2118BD
:1037B000325C20310A75315C002902D0401C10288F
:1037C000F5D3264600204036F070072D00D306259D
:1037D000E5620020E5642065201DFFF7D4FA20464D
:1037E0001830FFF7D0FA24610720411B6462A16101
:1037F000002161653176009A01990298FEF72CFD4F
:103800002060002F00D03C602546FFF7E5FA284EE7
:103810003069401C30613068264F002803D0F069C1
:10382000002821D026E035603069012822D100240B
:1038300014206043C019FFF79BFA641C072CF7D3D0
:103840001D48FFF795FA1D48FFF792FA1C48FFF74D
:103850008FFA1C48FFF78CFA1B48FFF789FA1648C5
:1038600070601430B06005E03068E96AC06A884270
:1038700000D83560F06A401CF0626864E86AB1699B
:10388000884200D9B06114214843C019291DFFF7AF
:1038900096FAFFF7ADFAF069002806D03068E96AB9
:1038A000C06A884201D2FFF7D3FA012009B0F0BD07
:1038B000A4470020E05C00206C5D0020805D0020BB
:1038C000945D0020A85D0020BC5D00200648C16911
:1038D000002904D0806B002803D00020704701200D
:1038E0007047022070470000A4470020014840694B
:1038F00070470000A4470020F8B5324F0026B86B8F
:10390000002808D0386A401C3862786A002800D045
:1039100001263046F8BD7D696D1C7D6115D1786842
:103920000068002801D072B6FEE77868B96879604F
:10393000B860B86A401CB86278680068002813D084
:103940007868C068C06840683863386B854211D3B6
:103950007868006800280AD07868C068C468606821
:10396000854211D2386305E00020C043ECE7002017
:10397000C043386338681421C06A48431249085864
:103980000128C2D90126C0E7201DFFF78BF9A06AE4
:10399000002803D020461830FFF784F9E06AB9699F
:1039A000884200D9B8611421484307494018211DB5
:1039B000FFF705FAE06A3968C96A8842C8D3012668
:1039C000C6E70000A4470020E05C002070B500219D
:1039D0000446002828D0154D2868844201D072B6CC
:1039E000FEE7206D002808D0401E2065E36CE26AE7
:1039F0009A4219D0002802D016E072B6FEE7201DC8
:103A0000FFF750F9E06C0721E062081AA061E06A54
:103A1000A969884200D9A861142148430449401883
:103A2000211DFFF7CCF90121084670BDA4470020F5
:103A3000E05C002070B504460020002C2AD0194D0F
:103A4000E16A2A68D26A914225D2A069002804DB83
:103A500028680721C06A081AA061E06A1422124E81
:103A6000504361698019814210D1201DFFF71AF976
:103A70002868C06AE062A969884200D9A861142157
:103A800048438019211DFFF79AF902E02868C06AAF
:103A9000E062012070BDE16C2A68D26A9142F8D3DD
:103AA00070BD0000A4470020E05C002070B5C06835
:103AB000C468002C0BD0204618300646FFF7F2F8F9
:103AC000104DA86B002804D031460F480EE072B6A6
:103AD000FEE7201DFFF7E6F8E06AA969884200D9F1
:103AE000A8611421484309494018211DFFF767F9CF
:103AF000E06A2968C96A884202D90120686270BDFB
:103B0000002070BDA4470020945D0020E05C0020F0
:103B1000F8B52E4D0027A86B002808D0FFF75CF9F8
:103B2000A86B401EA863A86B002802D046E072B6BE
:103B3000FEE72869002841D0254E306800282AD0A9
:103B4000F068C46820461830FFF7ACF8201DFFF776
:103B5000A9F8E06AA969884200D9A86114214843FC
:103B60001C494018211DFFF72AF9E06A2968C96A33
:103B7000884201D30120686230680028E0D1002C1F
:103B800009D068682946006800281BD04868C068CA
:103B9000C068406808632C6A002C09D00126FFF732
:103BA000ABFE002800D06E62641EF8D100202862AF
:103BB000686A002802D00127FFF74AF9FFF718F9D1
:103BC0003846F8BD0020C043E4E70000A4470020C9
:103BD000945D0020E05C002040BA7047C0BA704796
:103BE0000138FDD170470000F7B50325AD06286AFE
:103BF00082B016460C46400840002862286A02211E
:103C000008432862286A8007FCD466206860012780
:103C10002F61A86AC005FCD5992068602F61A86A49
:103C2000C005FCD5FF209130FFF7DAFFFF230133F9
:103C3000AB626846EF60352169602F61A96AC905EA
:103C4000FCD5AB62A969EF60C9B205226A602F6139
:103C5000AA6AD205FCD5AB62AA690902D2B21143A5
:103C60000180C80702D0032005B0F0BDAB626869CF
:103C7000FF210831884368616869C91E084368618B
:103C800002980002483068600820A860EE602F614A
:103C9000A86AC005FCD5FF200130A8620023F61CED
:103CA000B0080ED0B2081148006899006054060AA6
:103CB00009194E70060C000E8E705B1CC8709A427B
:103CC000F1D8FF200130A8626869FF2108318843DC
:103CD0006861686938436861286A800880002862E2
:103CE000286A38432862002005B0F0BD8000000C2F
:103CF000032080064169FF220832914341614269F5
:103D000001210A434261026A920892000262026A39
:103D10000A43026270470000002003218906096AF5
:103D2000490849000322920611621146096A0222DB
:103D3000114303229206116200BF03218906096A1A
:103D4000022211400229F8D0D10103229206916289
:103D50000321D1609F2151600121116100BF032126
:103D60008906896AFF22013211409142F7D103226C
:103D700092069162114688694969FF22083291438F
:103D8000032292065161114649690122114303221F
:103D9000920651611146096A89088900116211462B
:103DA000096A012211430322920611627047000042
:103DB0000000010200000000010203040138FDD1EF
:103DC00070470000F0B40324A406236A5B085B007C
:103DD0002362236A02252B432362236A9B07FCD4B8
:103DE000FF230133A3626569DE1DB5436561656923
:103DF0001E1D3543656100026B3060600820A060C5
:103E0000E26001262661A06AC005FCD5A3620023FA
:103E1000D21C90080ED095080F4800689A0088546C
:103E2000070A52185770070C000E97705B1CD07071
:103E30009D42F1D86069FF21083188436061606963
:103E400030436061206A800880002062206A30432D
:103E50002062F0BC002070478000000CF8B50646D8
:103E600001200025C004864201D90520F8BD0324A5
:103E7000A406206A400840002062206A022108430C
:103E80002062206A8007FCD4FF270137A76200F078
:103E9000BBF8002801D0032515E006206060012151
:103EA0002161A06AC005FCD5A762300220306060A5
:103EB0002161A06AC005FCD5A7620C4800F0C8F8D3
:103EC000002800D102256069FF2108318843606124
:103ED0006069012108436061206A800880002062D7
:103EE000206A084320622846F8BD0000E6960100DB
:103EF000F7B506460120C00482B01546864202D9B5
:103F0000052005B0F0BD03208006016A490849007C
:103F10000162016A022211430162016A8907FCD42D
:103F2000FF2101318162F2B28C1AA54200D8ACB2F5
:103F30000398009000F068F8002840D10621480658
:103F4000416001210161816AC905FCD5FF21013170
:103F50000320800681624169FF220832914341615A
:103F60004169042211434161310232314160C46030
:103F70000022002C16D9009887183B78F87819464B
:103F80007B7800061B021943BB781B0419430143CD
:103F90000802F978000A0906084319490860121D49
:103FA000A242E8D30121032080060161816AC9058C
:103FB000FCD5FF2101318162124800F049F8A54289
:103FC00009D00398361900192D1BFF2401340390E2
:103FD000A542ADD8ABE7032080064169FF22083235
:103FE000914341614169012211434161016A89089C
:103FF00089000162016A11430162002005B0F0BD31
:104000008000000C1A06000038B401250320800649
:104010006A46C560352141600561816AC905FCD5E4
:10402000FF24013484628169C560CBB205214160FF
:104030000561816AC905FCD5846280691902C0B234
:10404000014388B21180C00700D0012038BC7047FE
:10405000F8B400210125032292066B46D560352471
:1040600054601561946AE405FCD5FF270137976217
:104070009469D560E4B2052656601561966AF60526
:10408000FCD5976296692402F6B234431C80E3079C
:1040900022D0814202D9F8BC002070470322920648
:1040A0006B46D560352454601561491C946AE4055B
:1040B000FCD597629469D560E4B205265660156117
:1040C000966AF605FCD5976292692402D2B214432F
:1040D000A2B21C80D207DCD1F8BC012070470000DE
:1040E00000171300171000170E001709001704001F
:1040F00017000017180117140117150117190000F0
:104100000028000200000000032800020000000058
:10411000292A00020080800003280002000000001D
:10412000242A000200808000032800020000000012
:10413000252A000200808000032800020000000001
:10414000272A0002008080000328000200000000EF
:10415000262A0002008080000328000200000000E0
:10416000282A0002008080000328000200000000CE
:10417000232A00020080080003280002000000003B
:104180002A2A000200800800032800020000000024
:10419000502A00020080070031DD0001BFDC000171
:1041A000BDDC0001BBDC000100140000D9DD000112
:1041B000130C000015F000010314000095DE00014F
:1041C0007F240101F9230101AD23010161230101D4
:1041D000130C0000D9F00001150C0000B9F100012A
:1041E000170C0000F1EE0001000C000031EF00019F
:1041F000064700002727010103470000CD270101E2
:10420000084700006D2601010E470000B922010198
:104210000547000081290101FFFF00000DCF0001CB
:10422000130E000031E20001150E000041E1000113
:10423000170E0000B1E60001190E000089E600012A
:104240001842010105000000F7B586B00020029079
:104250005C48154604695C480E46824201D9054611
:1042600002E0002D00D10125002C08D0A18806987D
:10427000814204D1E088B04201D10120029053482C
:10428000039084460698010431430020002C1CD082
:104290000A0CA7888BB2974207D1E7889F4204D1C6
:1042A000002807D02168016007E020462468002C20
:1042B000EFD10AE0614622680A602168002902D035
:1042C0000020206001E061464860002C07D10221F7
:1042D000102000F095F8069981800446C6802801D8
:1042E000052100F077F807467D200E464643EFF3A0
:1042F0001085012080F31088684600F087F885F368
:10430000108800980490C0190501019927202D09F3
:104310008E1900010591864203D96D1C2D012D09CE
:10432000361AE660A5600398294F86460020844629
:1043300070460068002813D0A268E1680091C36845
:1043400081680193531A1B011B09BB420AD2914297
:1043500003D1019A0099914204D984460068E9E7A3
:104360007246546020606046002801D0046001E07D
:1043700071460C60134802990069002901D1A042DE
:1043800003D1C168806800F047F8EFF31084012082
:1043900080F3108802A800F039F884F3108803999C
:1043A00002980191291A090109090090B94204D221
:1043B000A84205D10198864202D8032000F032F8C5
:1043C00009B0F0BDC8010020FFFF7F02D801002026
:1043D000FFFFFF0730B50B460146002020220124D5
:1043E00009E00D46D5409D4205D31D469540491B29
:1043F0002546954040191546521E002DF1DC30BD72
:1044000003B40148019001BD2D7A010003B40148B5
:10441000019001BD5DB6020003B40148019001BDE9
:104420009DB6020003B40148019001BDAD780100C2
:1044300030B4C36882688868084D141A2401C968BA
:104440002409AC4203D2904204D18B4202D830BC42
:104450000120704730BC002070470000FFFFFF07BD
:104460000A0C838889B2934204D1C088884201D162
:10447000012070470020704770B405460068002294
:10448000002810D00B0C86888CB29E4207D1C688BB
:10449000A64204D10168002A07D0116006E0024656
:1044A00000680028EFD170BC7047296001680029BE
:1044B00003D00021016070BC70476A6070BC704717
:1044C000F0B5104F026886460025002A10D0C86853
:1044D0008C6893688446E01A00010009D668B842E7
:1044E00008D2A34201D1B44504D915461268ECE7BD
:1044F000704641600A60002D01D02960F0BD704611
:104500000160F0BDFFFFFF0770B584B004460E46A2
:10451000EFF31085012080F3108802A8FFF776FFE3
:1045200085F3108802980399024600900191A01A21
:10453000000107490009884204D2A24205D101982E
:10454000864202D8012004B070BD002004B070BDC6
:10455000FFFFFF0730B583B00446EFF3108501205D
:1045600080F310886846FFF751FF85F310880199A2
:1045700000986160206003B030BD00000028000298
:10458000000000000328000200000000002A000ACA
:10459000008020000328000200000000012A000221
:1045A000008002000328000200000000042A00022C
:1045B000008008000328000200000000A62A000274
:1045C000008001000328000200000000C92A000248
:1045D0000080010000280002000000000328000203
:1045E00000000000052A0020008004000229000AC3
:1045F000000002000328000200000000292B000A2E
:104600000080100003280002000000002A2B000296
:1046100000801000FFFF0000E9C90001A40D0000A8
:1046200055E90001A50D000089E900011A0D0000FF
:10463000A1EE0001150D0000E9E90001000D0000E8
:1046400015EA00011C0D0000D7EE0001A70D0000C7
:10465000F5ED0001A80D0000E3EE0001020C0000E2
:10466000C9EF0001000C0000A1EF0001010E0000E5
:10467000CDE400010F0E000089E80001110E0000DA
:10468000EDE800012C0E00006DE80001030E0000B3
:1046900025E600010A0E0000E1E70001300E0000EF
:1046A00061E800010C0E000015E90001000E000099
:1046B00039E40001090E000061E40001010F00006F
:1046C00029CC0001020F0000B1C80001030F000057
:1046D0000DCC0001040F0000F10701011446010197
:1046E00036470020010019000214000011DF00010C
:1046F000E846010101000000044801010300000038
:1047000001102EC78A0E7390E111C20860270000C5
:104710000028000000000000000000000000000071
:10472000000200000000032800000000000000005C
:10473000000000000000000A0000000001002EC779
:104740008A0E7390E111C20860270000000400C0C7
:10475000000201290000000000000000000000002D
:104760000000000A00801400032800000000000080
:104770000000000000000000000A0000000002002D
:104780002EC78A0E7390E111C20860270000001046
:1047900000C000020229000000000000000000002C
:1047A00000000000000A0080140003280000000040
:1047B00000000000000000000000000A00000000EF
:1047C00003002EC78A0E7390E111C2086027000013
:1047D000000A00C0000203280000000000000000E2
:1047E000000000000000000A0000000004002EC7C6
:1047F0008A0E7390E111C20860270000000200C019
:104800000002000004470000052901010A470000DA
:10481000ED270101074700001D270101A44B0101FD
:10482000704B010179A900014C4B0101344B01018E
:1048300029AD0001544B0101584A010151AB00015F
:10484000684B01019449010151A70001004B01018E
:10485000FC490101D9A60001C44A0101944A0101A1
:104860004DAA0001DC4B0101D0490101A19E0001CC
:10487000EC4B01017C4C0101699F0001AC4B010133
:10488000084B0101499B0001F44B01015C49010106
:104890007D9B00016C4C0101FC4B01015D98000106
:1048A000E44B0101384A01011DAB0001744C0101C8
:1048B000344C0101E9A80001644C0101C84A01011E
:1048C000E5AC00015C4B0101B44B010139AC0001C6
:1048D00001020304050607004040404040404040BC
:1048E00040414141414140404040404040404040C3
:1048F00040404040404040400502020202020202A5
:104900000202020202020202202020202020202097
:1049100020200202020202020290909090909010D9
:104920001010101010101010101010101010101087
:104930001010100202020202028888888888880803
:1049400008080808080808080808080808080808E7
:104950000808080202020240D84801016273736528
:1049600074203C6669656C643E203C76616C3E3A1E
:1049700020777269746520626F6F747365747469EF
:104980006E67206669656C64202863617265667570
:104990006C21290073686F772064657669636520F0
:1049A000696E666F202874656D702F7664642F665B
:1049B000616E2C2073616D6520617320424C45202F
:1049C000494E464F5F515545525920616C6C290044
:1049D000617070676574205B6A736F6E5D3A2073F7
:1049E000686F772061707020706172616D7320282C
:1049F0006C65642F70776D2900000000626C656C37
:104A00006F67205B6F6E7C6F66665D3A20424C4537
:104A10002074726166666963206C6F672028657612
:104A2000656E7473202B206672616D6520686578F1
:104A30002064756D7029000072657365743A207387
:104A4000797374656D207265736574202872656270
:104A50006F6F74290000000073686F7720467265DD
:104A60006552544F532072756E74696D6520696E7E
:104A7000666F2028757074696D652F7461736B7330
:104A80002F686561702F7461736B206C6973742972
:104A9000000000006C6564203C317C323E203C6F9D
:104AA0006E7C6F66667C746F67676C653E3A2063E8
:104AB0006F6E74726F6C20626F617264204C45443B
:104AC000000000006C656400756172747273743A62
:104AD0002072652D696E69742055534152543120FE
:104AE0002831313532303020384E31292C20666C57
:104AF0007573682072782071756575650000000017
:104B0000626C656C6F670000627364756D703A204B
:104B100073686F7720626F6F7473657474696E6702
:104B2000207265636F7264202B2063726320636858
:104B300065636B0073686F77206669726D77617269
:104B4000652076657273696F6E000000766572731A
:104B5000696F6E00737973696E666F007561727448
:104B6000696E666F00000000646576696E666F00AE
:104B700068656C70205B636D645D3A206C6973746A
:104B800020636F6D6D616E6473202F2073686F7783
:104B9000206F6E6520636F6D6D616E642773206892
:104BA000656C700068656C7000000000627364756D
:104BB0006D70000075617274696E666F3A2073687B
:104BC0006F77205553415254312070696E732F62B4
:104BD0006175642F666F726D61740000617070673B
:104BE0006574000072657365740000006170707315
:104BF0006574000062737365740000006170707307
:104C000077205B317C325D3A20737769746368206A
:104C1000626F6F742062616E6B202863726320760E
:104C20006572696669656429202B207265626F6F01
:104C300074000000666163746F72793A2072657364
:104C4000746F726520706172616D7320746F20647F
:104C5000656661756C747320616E64207265626F45
:104C60006F74000075617274727374006170707398
:104C700077000000666163746F7279006170707311
:104C80006574203C6C65647C70776D3E203C766179
:104C90006C3E207C20617070736574206A736F6E47
:104CA000207B226C6564223A3530307D00000000A4
:104CB00075736167653A20617070736574203C6C30
:104CC00065647C70776D3E203C76616C3E207C2074
:104CD000617070736574206A736F6E207B226C65DF
:104CE00064223A3530302C2270776D223A35307D8F
:104CF0000D0A000061707073773A2062616E6B2557
:104D00006C7520696D61676520637263206D6973DE
:104D10006D6174636820287265636F7264203078F7
:104D20002530386C582C2061637475616C203078A4
:104D30002530386C58290D0A000000002020202062
:104D400020202020206231616464727C62326164C0
:104D500064727C623173697A657C623273697A65E8
:104D60007C62316372637C62326372637C6231762F
:104D700065727C6232766572203C6865787C646519
:104D8000633E0D0A00000000A84D01010040002014
:104D90000C08000030950001BC5301010C480020B4
:104DA000C46F0000F02A0000A0060090D0030001AC
:104DB0001005A00000FF01D20001000651C2020050
:104DC000200001302B11D80D490868496813F008FC
:104DD000FB0498EFF78EFF0446C1888088FF22FF0E
:104DE000F79DFD2046FFF73AFCB3E705B0F0BD980C
:104DF000100707D8010020C804202930D70200007E
:104E00004B1847FBFD06460520307075800099B1B0
:104E100081301D3946E5F773FD3046F9F70EFF0E78
:104E200022294642200445FD074030112E0CD05364
:104E30004B052203212846FDF733FE121E40274B67
:104E400075002D05D0398F002902D000998979008D
:104E5000E000211176FAF74BF8044D2859F9F7FBD9
:104E6000FE002028518010060004002007771078EB
:104E700038B5049C0094014CA04738BD5143F84A12
:104E800026468F1839462036FD6D707D8031119190
:104E9000C97FA0370E912246397815320F92F14A18
:104EA000109203292BD0002873D0F17D0F980CF0BD
:104EB0000DF800286FD0688869460883F0B597B070
:104EC00008780C460F90002014900F984821484312
:104ED000FE4922464018064680361090F17F009128
:104EE000C56DA0301690014E100A27461292203749
:104EF000F74A1552146C2AD061783C2949D04329CD
:104F000047D0787D00287DD0F97D129800F0FCF91B
:104F1000002878D0698868468184687A297A0004F4
:104F200009020843E97908430690A97A08A8417262
:104F3000E97A8172297BC17229460D310E380E91B2
:104F400000F02FFAA878400733D5002132E0907E98
:104F5000012806D0507E401E0006000E507603D079
:104F600006143004DB480106141200F0D2F9169A38
:104F700001211170A978D448C9075C3690264823CE
:104F8000594308180022A0300270FF20F07752E049
:104F900001220270A878CC49C0074CD00098482361
:104FA00058434020101442E0E97C08A80173297D91
:104FB0004173697D8173A97DC108100D0174297E3B
:104FC0004174697E8174B189BC102281F189C181EB
:104FD000318A0182109940318A8F8283C98F01847E
:104FE000B188C183F18841840021C18442241472B4
:104FF000B848817808A8C17401E04DE11BE00226A1
:105000000675C821CC140C02D4E87A800705D5298E
:105010007B0E14300A7EF908A9087503A90F0C1439
:1050200012002801D11698067060783C2870D030A4
:10503000E1628A143D0A82A2884A82A2790A75E254
:10504000794A75207A8875E07EC875A08B0883E060
:105050008B4883208C8883608CC883214624310848
:10506000A800F0A4F9787A08A94871B87A8871A0E4
:105070008DC8140585206B0BC210050C90012018FB
:10508000103F75387D0875B87D8875A878C006C052
:1050900017401CC8758E486946028A0A87428A4AA8
:1050A00087827D08A90A77C27D4A77027E8A774285
:1050B0008B10A90A80828B4A80807F087104A90026
:1050C000A4380432F9000A14487C49401803907C43
:1050D00030129900F05DF90398F97D8030817003FA
:1050E000990922A0310A700121C170039800218121
:1050F00066E18B490041660521C16601671599602B
:1051000030C97E002904D072498161012102E02A60
:10511000BA4809816181750099818224400DF6F8B1
:10512000022802D2012100F003F912201B05F90622
:10513000280CD20A215F4A41438918FF3181314945
:105140007F890703D5FA7D7C23FCF8961005FFF8CC
:105150001699E035C41A01AE1818092000F0FBF8C2
:1051600021460F31059100284ED020233E220021F8
:1051700056241C06F6F806460A96031714986C1E69
:10518000D03A04200EE03C2070700120307100986D
:1051900070801620052CD0B01D5A2407F2F8F87D37
:1051A0007071AC201306D52146304609310C300011
:1051B000F0E7F803E030460A12DD2025C81006307B
:1051C000461230053032DA1A12121A1406D0F8E0FC
:1051D0008B309A16709A2813B083B87AB07730461D
:1051E00000F0BFF83AE0287B7071DC2007B01D00AA
:1051F000F0C2F8163006B4F83DE0149E1A2EC23004
:1052000008A7F801210646019E120D9E3004707019
:105210003198200BF87D820709D57171B01D6A3075
:1052200004A5F80AB6400B30461DE0C007C00F7059
:1052300071B2129978100BB081208CF081608C30A3
:105240008278227462300483F8066012166030247B
:1052500077F81421017000994180B97D017100F047
:1052600075F81598807E022826D160781499084335
:1052700022D0082C120B2C100461F8122C1C0C618B
:10528000784170297881700FE04064041C06C006E4
:1052900000200A6E0512390412400C1D88031C08F8
:1052A00020B1A201000411A0051007998180397E68
:1052B00081563C064AF80020171805100640BA70BF
:1052C00047C004600D03B40148019001BD919B02E9
:1052D000000C83E1980C837D9F0C700449FA010C4B
:1052E0008309D30C836D5B24933D99488290488356
:1052F00055073083D59C3083397B181027796D0191
:1053000000002101804180818070470A7802704B43
:105310007843708A788270CA78C2700B7903714AB8
:105320007942711A20046802600E0F3470474006FB
:105330003414497B41700570F1F7F3FC2068F1F7F4
:10534000A4FB256003141B2400761C098002408006
:10535000C10240062B066419F8B54E784821F0B218
:1053600048432349214D41180C46AA7EA03400270A
:10537000282C22EDC3020010B5074CE06900040898
:10538000D5FFF7F3FF05480078002802D10120C0BF
:10539000032062100006115012C6580F4EF4010689
:1053A00007CD7007100671B800010D040006550105
:0C53B0002A0101000112AA01E15C0000CA
:020000040102F7
:10400000D0B7002069410201714102016D710201C6
:1040100000000000000000000000000000000000A0
:1040200000000000000000000000000031750201E7
:104030000000000000000000274102013575020168
:104040007B4102017B4102017B4102017B41020174
:104050007B4102017B4102017B4102017B41020164
:104060007B4102017B4102017B4102017B41020154
:104070007B4102017B4102017B4102017B41020144
:104080007B4102017B4102017B4102017B41020134
:104090007B4102017B4102017B4102017B41020124
:1040A0007B4102017B4102017B4102017B41020114
:1040B0003D7702017B4102017B4102017B4102010C
:1040C0000348854601F076F80048004735BA0201FA
:1040D000D0B7002040BA7047C0BA70470138FDD150
:1040E0007047000040BA7047C0BA704770467047CA
:1040F000084B19680868203080F30988022080F393
:104100001488BFF36F8F3FBCAE4608BC04BC62B6D8
:1041100018470000A4470020EFF3108072B67047E4
:1041200080F310887047EFF309800E4B1A6820382F
:104130001060F0C044464D4656465F46F0C008B594
:1041400072B60BF031F862B60CBC1168086810301A
:10415000F0C8A046A946B246BB4680F3098820387D
:10416000F0C81847A4470020044880470448004787
:10417000FEE7FEE7FEE7FEE7FEE7FEE78D750201DC
:10418000C140020130B50B46014600202022012427
:1041900009E00D46D5409D4205D31D469540491B7B
:1041A0002546954040191546521E002DF1DC30BDC4
:1041B00070B500242546002801DA01244042002978
:1041C00001DA01254942FFF7DDFFAC4200D0404251
:1041D000002C00D0494270BDF0B51FB40646002047
:1041E00082B005464024019100901BE001992246CF
:1041F0000F46304600F02DFE049A059B801A994127
:1042000010D310461946224600F013FE361A8F418D
:104210000197224601200021009F00F00AFE381875
:104220004D4100902046641E0028DFDC019B009871
:104230002946324607B0F0BD01464139192900D858
:10424000203070470549064A08685043054A8018DF
:10425000086040087047014908607047FC4700202B
:104260006D4EC6413930000003460B439B0703D017
:1042700009E008C9121F08C0042AFAD203E00B782B
:104280000370401C491C521EF9D27047D2B201E0A3
:104290000270401C491EFBD270470022F6E710B5A1
:1042A00013460A4604461946FFF7F0FF204610BDA4
:1042B000421C0178401C0029FBD1801A704710B5C0
:1042C000002200E0521C835C8C5CA34201D1002BD5
:1042D000F8D1D8B2E1B2401A10BDC9B203E00378F8
:1042E0008B4203D0401C521EF9D20020704730B5DB
:1042F00004460020034600E05B1C934203D2E05CCE
:10430000CD5C401BF8D030BD03460A780270401CDB
:10431000491C002AF9D11846704730B505460020DF
:10432000034600E05B1C934205D2EC5CC85C201A9B
:1043300001D1002CF6D130BD0FB400B58DB009907D
:104340000B9010A900200091C0430A9000200C900F
:1043500006480690064807906A4609A80F9900F09B
:10436000B1FD0DB008BC04B018470000E54E0201D5
:10437000054F0201FFB5087889B01546FF2805D022
:10438000491C2D2804D00022002407E000240BE063
:104390000122F9E70A235C430419491C0878FF2825
:1043A000F8D1002A00D06442002004902A78014607
:1043B0002D2A01D02B2A0FD16D1C2D2A02D00022CC
:1043C000049209E00122FBE700260A2233466D1C15
:1043D00000F0F2FC381871412F78FF2FF4D10C9ABD
:1043E000A218069202460A4304D0FF23069A91338C
:1043F000DA4205DA002109980A4606C00DB0F0BD80
:104400000024B74AB54D2646079200F011FC0290F1
:1044100006980391002801DA474200E00746390573
:104420000020AF4A001C51410191009012E0F807B2
:1044300007D022462B463046079900F0D9FA0646A7
:10444000079122462B461046194600F0D1FA044641
:104450000D467F10002FEAD10698019B0028009A94
:104460000399029806DA00F02BFB3246079B00F016
:1044700027FB05E000F0BCFA3246079B00F0B8FAD3
:10448000049A002A02D00122D2075140099A03C29D
:10449000B4E7FFB591B0002009900025ED432E2030
:1044A0009E685C681F460190B9696D1C1298884728
:1044B0000090396A88470028F6D10098401C0AD03D
:1044C0000D20C0018443002E12DD00982B2809D056
:1044D0002D280DD103E00020C04315B0F0BD012010
:1044E00080020443B9696D1C12988847761E0090BB
:1044F00003A9600501D52D2000E02B206A4610732A
:10450000491C0CA80F9102900AE0B9696D1C129821
:10451000884700900120400204431398761E0560EE
:10452000002E02DD00983028EFD0019900988842D3
:1045300046D18020044308E00998401E09900120DC
:10454000400204431399681C0860B9696D1C761E0B
:104550001298884700903028EED031E001998842C7
:1045600005D1200603D480200443761E1EE0009867
:1045700003F0F2FA002826D001204002044307A9E4
:104580000F980331761E88420BD200980F9930386D
:1045900008700F98401C0F90200607D50998401E00
:1045A00003E0200602D40998401C0990A00502D51A
:1045B0001399681C0860B9696D1C129888470090AF
:1045C000002ECBDC59E0002E57DD0098652801D085
:1045D000452852D1A00550D5032000028443B96973
:1045E0006D1C761E129888470090002E0CDD2B283B
:1045F00004D02D2808D1FF2001300443B9696D1C77
:1046000012988847761E0090E00501D52D2100E024
:104610002B21029801700298401C0290019025E025
:104620000120400204430EA902980131761E8842FF
:104630000ED20098029930380006000E087003D19F
:104640000299019881420AD90298401C029006E022
:10465000E00501D5234801E0224840420990B969AC
:104660006D1C12988847009013980560002E04DD99
:10467000009803F071FA0028D2D1F969129888479E
:104680000F99FF200870029903AA087000200A9071
:104690000B900CA90AA8099BFFF76CFEA00502D499
:1046A0000120C04319E72420044209D0E00713D1B8
:1046B00038680B9A0A99031D3B60006806C00BE03E
:1046C0000B990A9800F05CFB0146E00704D13868BA
:1046D000021D3A60006801602846FEE600001440B2
:1046E0000000F03FF1D8FFFFF7B582B00F4600267B
:1046F000029C03F01DF90090006801902578641C6D
:10470000002D05D000F0CAFB0068405DC007F5D160
:104710002B2D02D02D2D1CD0641E0098002101608D
:1047200039462046049A00F0FFFB0146002F04D0D2
:104730003868A04201D102983860009800680228C9
:104740000BD00098019A0260700506D5484205B06A
:10475000F0BD012080020643DFE70846F7E7F8B521
:1047600002464A40D40F42004B0052085B089A426E
:1047700002D20246084611464A0023D0C30D4A0021
:10478000DDB2120EAD1A202D35DA49020126490A92
:10479000F6058A19002C00D0524220214F1B1146E9
:1047A000B9402A411018C20D9A4221D0002C17D0CE
:1047B000012D08DCDA05801AD20F8019D207DBB28E
:1047C00000F060FCF8BDDA05801A012340001B06EA
:1047D000C01880185A428018CA0F1043490007E0D9
:1047E0004908C2071143DA05801A80194008801869
:1047F00000F040FCF8BD61000122511A001BF7E7F0
:104800000122D2075140AAE70122D2075040A6E771
:10481000024670B54A40D30FDB0740002DD04A0056
:104820002AD0010E140E000212020919400A520A7F
:104830008418E50104465443000A120A2E0450432A
:10484000A4194219200CC543AA18120C0125AD0366
:10485000521C521912047F39240400D0521C1043F8
:1048600001D44000491EC2B20C06C0092018401CE9
:104870004008802A02D003E0002070BD40084000BC
:10488000002900DA0020184370BD0000F0B507468B
:104890000846584087B0C00F049048000E465900A3
:1048A00040084908BC1A884105D2384631461E46A0
:1048B00017460B4602465800400810434CD0300DB6
:1048C000039040055900400D490D0590401A029093
:1048D000402872DA18030121000B090508430190F2
:1048E00004980092002805D0019952420020884186
:1048F00000920190029840210A1A0199009800F054
:1049000098FA05460C466B4607CB00F0B3FAC0197F
:104910007141039A0E0D0023D71756401A467A406C
:10492000164344D0049A002A2DD0029A012A039AF1
:1049300015DC1205C01A914101263605001C714193
:10494000D20F059ED2070093019202962A46234673
:1049500000F0DEFB07B0F0BD38463146FAE7160539
:10496000224A0F46B218C01AB74101210905001C9E
:104970004F4100187F41114618187941E20F10434A
:104980006D19644113E0E2076D0815436408C2071E
:104990001443039A01261205C01A91413605001CE2
:1049A0007141CE07400830434908C01851412A469A
:1049B000234600F0A0FBCDE7FFE70498012240006A
:1049C000C117121A00238B4104983146C417381AB4
:1049D000A141EEE730B40124E407634030BC55E761
:1049E00030B40124E407614030BC4FE70000E0FF31
:1049F000F0B51FB488B00B99099800244840099974
:104A0000C00F490049080991C0070B99009049005F
:104A100049080B9109990898A64608431CD00B99A0
:104A20000A98084318D0099801244000420D480014
:104A3000410D099824050003000B204309900B98B1
:104A40000003000B20430B9050181C494018002213
:104A500001901446104605E0002001460DB0F0BD5F
:104A6000032801DA034600E003239C46C11A0AAE7C
:104A70000AE05F0008ADED5B4F00F75B7D43002768
:104A8000AA187C41491C5B1E6145F2DD410004AB64
:104A90005A522104120C0A43240C401C0828DFDB64
:104AA000019802900099704601910090059B049A2C
:104AB0000799069800F02CFBD0E700000DFCFFFFE3
:104AC000F0B50C465C4085B0E40FE40703944C005D
:104AD000002664085900944649080246029622437B
:104AE00021D062460A431ED06200570D4A000E03D1
:104AF0002303550D012402462C492405781B1B0B6A
:104B0000360B401823432643614600901C46501A3A
:104B1000B44103D30098401C009002E09218009822
:104B20005B41002803DA0020014605B0F0BD0020FB
:104B3000012109050746864611E064461D46141BFF
:104B4000B54106D36546521BB341744607430C4337
:104B5000A646CD0740084908284392185B41054600
:104B60000D43EAD11046184313D060461946504011
:104B70007140084306D06046101AB34106D20122A4
:104B8000002306E000220123DB0702E00122D243DA
:104B90005310009874460105381C6141029C039D26
:104BA0000019694100F0A7FABFE70000FD0300000B
:104BB00070B54B005B0803430BD04B005C0D002627
:104BC00033466542B341D417AD1AA34102DB00203E
:104BD000014670BD12053018514170BD10B500225C
:104BE0009623114600F04EFA10BD00000EB5C21714
:104BF000C10F5040CA0740180021054B0293019293
:104C000000910A460B4600F083FA03B000BD000095
:104C1000330400000EB505490291002100910A46B7
:104C20000B46019100F074FA03B000BD330400009C
:104C30000EB5054A0292002200921346019200F03E
:104C400067FA03B000BD000033040000C20F41004A
:104C500040020123400ADB05D207090EC0187F2954
:104C600001DA00207047962903DC9623591AC840C0
:104C700001E096398840002AF4D040427047000095
:104C800070B5CD0F4A0009030123090B1B05194319
:104C90000B4BED070024520D9A4201DA002070BD43
:104CA000074B34339A4203DC9A1A00F0D2F802E040
:104CB0000449511888402C43F1D0404270BD000097
:104CC000FF030000CDFBFFFF4A0009030123090B8E
:104CD0001B0519430A4B10B5520D9A4202DA002007
:104CE000014610BD064B34339A4203DC9A1A00F099
:104CF000B0F810BD034BD21800F09BF810BD0000B7
:104D0000FF030000CDFBFFFFC20FD20740004008A9
:104D10000BD0C10D0723DB01C91840020905400A69
:104D20001143C208400711437047002001467047F5
:104D300010B5002904DB0124E40740428C412146E0
:104D4000002B04DB1C460123DB075242A3418B42AC
:104D500000D1824210BD000010B5002904DB0124FF
:104D6000E40740428C412146002B04DB1C46012312
:104D7000DB075242A341994200D1904210BD00008E
:104D8000CB0FDB07490010B5490802460A4307D09C
:104D90000A0D07240903E401090B121B002A01DC98
:104DA000002010BDC900440F0C43C100E018D2051B
:104DB000801800F05FF910BDF0B51FB486B0002078
:104DC0000090019002900698069980B2049007988E
:104DD000090C02040014114307900027089D09984C
:104DE00006913E463C4603900398A9B20204000C8B
:104DF000039004982D0C154348430021224600F0EF
:104E000018F8C719714110340E46402CECDB3846B7
:104E1000029A00F00EF8009A019B80180090594108
:104E200002980191103002904028CCDB00980BB022
:104E3000F0BD10B5202A04DB0146203A9140002045
:104E400010BD914020239C1A0346E3401943904033
:104E500010BD10B5202A04DB0846203AD0400021BE
:104E600010BD0B46D340D0402024A21A91400843E5
:104E7000194610BD10B5202A06DBCB170846203A8C
:104E80001041C1170B4306E00B461341D0402024CC
:104E9000A21A91400843194610BD0000004870470F
:104EA000840A030110B50446FFF7F8FF0068005DAF
:104EB000C007C00F10BD00000268137851180160D0
:104EC0001846704710B5D160044951610449116218
:104ED00000211161114600F08FF910BDB94E020199
:104EE000A54E02014268002A08D001680B78491CCF
:104EF000002B03D0521E06C0184670470121C16026
:104F0000881E70474268002A0BD0C3680168002BD6
:104F100007D183688B4204D0491E521C06C0002072
:104F200070470020C0437047F7B582B0029C00274D
:104F30002078641C15460197302802D0002D15D02A
:104F400015E020780127641C782804D0582802D066
:104F5000002D09D00BE0002D01D0102D07D1002726
:104F600010252078641C02E0082500E00A250026B0
:104F7000009610E00099012769430818020C2946A1
:104F800080B2714300908E183804864201D301200C
:104F900001902078641C294600F01EF90028E9DA07
:104FA0000398002805D0002F01D0641E00E0029C69
:104FB00004600198002806D002F0BAFC02210160CA
:104FC000C81E05B0F0BD009930040843F9E70000A1
:104FD0000FB400B589B00CA900910B990023CB60E8
:104FE000204B214A06930792042201921F4A029203
:104FF0001F4A089202466B460020FFF74AFA09B0A2
:1050000008BC04B0184770B586B006460020C043FF
:105010000190002015460C46009102910490324602
:10502000694604A8FFF7D4FF024604982118002D12
:1050300005D0002801D0084600E0204628600498EA
:1050400000280DD0002A02DD0098884208D0081BF5
:105050000190009432466946029404A8FFF7B8FF15
:1050600006B070BDE54E0201054F0201FFFFFF7F54
:10507000A54E0201002904DA401C490001D1400874
:105080004000704770B40024050C05D110240004C2
:1050900002D1002921D01124050E01D100020834CB
:1050A000050F01D10001241D850F01D18000A41C32
:1050B000002801DB4000641C002908D020252E1B9D
:1050C0000D46F540A14000D00121294308430106C7
:1050D0001B1B000ADB1D02D5002070BC7047DB05DE
:1050E000181880180029F8DA401C4900F5D170BC66
:1050F00040084000704710B5002B08DA0024401C1F
:10510000614192185B411A4301D14008400010BD33
:10511000F0B51FB482B005460C0003D0084602F07B
:10512000EFFB02E002F0ECFB20300246009021464B
:105130002846FFF77EFE049B059A04460F46184357
:105140001143084314D0184610431BD00098402147
:105150000A1A18460599FFF77CFE05460E46009A86
:1051600005990498FFF765FE084305D0012004E087
:105170002046394607B0F0BD0020C11705430E4355
:105180002C43374300990E986305401A7905E40AC9
:1051900000220C43FD0A0A3002D500200146E9E74F
:1051A0000105101969410C9C0D9D00196941FFF71B
:1051B000A2FFDFE7064C0125064E05E0E36807CCB9
:1051C0002B430C3C98471034B442F7D3FEF77CFFD6
:1051D000B40E0301D40E03013A2800D23038202344
:1051E00002469A43412A01D310463738884201D3F8
:1051F0000020C04370470000F3B58DB000200A9036
:1052000001200B90002608460C300C46099062697C
:10521000012109989047051E2ED0252D2DD0216AF9
:105220008847002818D06269012109989047216AAF
:1052300088470028F7D1411E62690998904700E02D
:10524000761CA1690D988847216A88470028F7D104
:10525000E1690D988847DAE7A1690D988847074604
:10526000A84201D1761CD2E7E1690D9888477F1CDE
:1052700002D10A98002877D049E1002762693D46AB
:105280003946099890472A280CD16269012109986A
:105290009047012506E00A214F433F18303FEBD4E9
:1052A0001020054362690121099890470146303971
:1052B0000A2903D29B498F42DEDCECE7E90600D4E1
:1052C000994F6C280AD04C2810D0682824D06A281E
:1052D0002ED074280CD07A280AD00DE06269012102
:1052E000099890476C2823D004211CE02020054316
:1052F0006269012109989047A760656065284FD0D1
:1053000026DC582839D01ADC452849D012DC25285B
:1053100034D04128B0D143E0626901210998904717
:10532000682802D008210D43E6E70120C002DEE72D
:105330000220DCE7462833D047282CD130E05B2818
:1053400070D061282CD063286CD0642823D161E010
:105350006F284FD009DC662822D0672820D0692822
:1053600026D06E2817D12EE0CDE070284DD07328BE
:105370006FD075284ED078280DD154E0A1690D98D2
:1053800088470546252800D16CE7E1690D988847D4
:105390006D1C00D16DE7BAE00A224CE00A2252E00F
:1053A000012023466A46C0430D99FFF772F8A3E037
:1053B0002846402108436060A807234601D5002203
:1053C00039E000223FE0E80700D020E72068011D17
:1053D00021600068290501D5067018E7290701D565
:1053E000068014E7A90703D5F117066041600EE7B0
:1053F00006600CE72846402108436060A807234662
:1054000001D5082217E008221DE048492846084037
:10541000606016E02846402108436060A8072346E4
:10542000BCD5B9E715E02846402108436060A807CD
:1054300007D5234610220120C0430D99C046C0461F
:105440005AE0234610220120C0430D99C046C046B1
:1054500052E000210C910B460091632802D05B289A
:1054600007D043E0E80601D40120A06001200090AD
:105470003CE062690121099890475E2805D101202E
:105480000C9001466269099890472169002906D16C
:105490000B4601AA8F00491CD3510829FADB0028CA
:1054A00035D0216900290ED1C117C90E09184A113A
:1054B000930001AA9A1849094901411A0120136869
:1054C00088400343136062690121099890475D2871
:1054D000E5D10C98002808D0002001AB81005A5873
:1054E000401CD2435A500828F8DB01AB0120224669
:1054F000C0430D99C046C04600280ADA401C06D1B8
:105500000B98002803D00020C0430FB0F0BD0A98CC
:10551000FBE7E90702D10A99491C0A9136180020D5
:105520000B9074E6CCCCCC0CFFFFFF7FF1F7FFFFB4
:1055300070B58D180478401CA207920F01D1027833
:10554000401C231106D10378401C03E006780E703E
:10555000401C491C521EF9D1002B15D002780C2694
:105560008A1A3440401C0C2C03D0A401121B9B1C33
:1055700008E004782402121B401CF8E714780C7031
:10558000491C521C5B1EF9D5A942D3D3002070BD23
:1055900003B40148019001BD232A000003B401486F
:1055A000019001BD397B010003B40148019001BDA8
:1055B000B17B010003B40148019001BDBD80010031
:1055C00003B40148019001BD6D56000003B40148C9
:1055D000019001BD6560000003B40148019001BD68
:1055E000A1B3020003B40148019001BDAF7F0000E8
:1055F00003B40148019001BD1979010003B40148C9
:10560000019001BDB551000003B40148019001BDF6
:105610002D7A010003B40148019001BDD37E000042
:1056200003B40148019001BDD97C010003B40148D5
:10563000019001BD697E000003B40148019001BDE5
:10564000C37F000003B40148019001BDB57C010097
:1056500003B40148019001BD5DB6020003B40148E6
:10566000019001BD9D7B010003B40148019001BD83
:10567000D97B010003B40148019001BD7D7F010089
:1056800003B40148019001BDAD78010003B40148A5
:10569000019001BDE954000003B40148019001BD2F
:1056A0009957000003B40148019001BDED57000077
:1056B00003B40148019001BD1D7C000003B4014802
:1056C000019001BD617D010003B40148019001BD5D
:1056D000957D010003B40148019001BDDD7D01000D
:1056E00003B40148019001BD0D2A000003B4014834
:1056F000019001BDAB52000003B40148019001BD0F
:10570000E579010003B40148019001BDFD7A010073
:1057100003B40148019001BDE1AA020003B40148AD
:10572000019001BDF58F000003B40148019001BD57
:105730006DB1020003B40148019001BDE1FE00001B
:1057400003B40148019001BD250E010003B40148D6
:10575000019001BDB143000003B40148019001BDB7
:1057600085AC020003B40148019001BDA1AC020068
:1057700003B40148019001BD25B0020003B4014803
:10578000019001BDB5B2020003B40148019001BD12
:10579000D1B2020003B40148019001BD8529000087
:1057A000C943416070470268702392B29A430A432A
:1057B0000260704770B5044601F0A8FF002818D0B9
:1057C0008069002815D0FFF709FA05462046FFF743
:1057D00005FA2946FFF718F8FFF796FA064A074B2D
:1057E000FFF76EF90022064BFFF750F8FFF7C8FAF3
:1057F00070BD044DEAE700001F85EB51B81E014063
:105800000000394000803B4470B50D460646002438
:1058100001F07CFF002816D0C169002913D0026A6C
:10582000002A10D08BB290B289B292B2102D0CD057
:10583000202D0AD0302D17D0402D15D0502D13D04B
:10584000602D11D022E0002070BD891AB01AAF225D
:1058500092005043FEF7ACFC044696340FD47D20F2
:10586000C000844211DC11E0191AAF22301A120173
:105870005043FEF79DFC4B21C900441801D500247C
:1058800004E0E1200001844200DD0446204670BDB2
:1058900070B5104CA0421BD185140121284601F09F
:1058A000E7FD0021284601F0E3FD0121284601F033
:1058B000D3FD094860610020206060601F21A16065
:1058C00006492161A06160622062A0620448E06133
:1058D00070BD000000080240080A02000000FC0F32
:1058E0002E6D00000029016802D00122114301E061
:1058F000490849000160704704220029816902D0EB
:105900001143816170479143816108480649C16232
:105910000749016307494163074981630749C16337
:1059200008490748086070472200780000080240D4
:10593000E700E1009F00BF04190C051670206E28D7
:105940006E2B00004008024002220029016801D0AD
:10595000114300E0914301607047C06880B2704716
:105960000246526800200A4200D001207047000021
:10597000044A9068C90640094001C90E014391607C
:10598000704700000008024070B5054649480C46C3
:105990004EC88CB003960293019200914EC80796B0
:1059A0000693059204914268016880680992089103
:1059B0000A90414A00996846914217D1282104F083
:1059C000BFF80A99884211D1022D1ADB00206468C1
:1059D00002460B900BA92046FEF786FE05460B9863
:1059E000A04209D00078002806D101E033A004E0ED
:1059F000012D0AD0022D08D03EA004F09FF90CB072
:105A000070BD0198012809D001250198A84207D14D
:105A1000294647A004F02CF90CB070BD0225F4E72C
:105A2000012D6C4614D01834012D13D0474822683C
:105A3000824206D16068002803D00721890388428A
:105A40000AD9294642A0636804F012F90CB070BD6F
:105A50000834E9E74C48EAE74CA004F06FF96168C4
:105A6000206804F06DF8A268824206D003462946F9
:105A7000544804F0FDF854A0BFE729465FA06368CE
:105A8000E26804F0F5F86846019503F079FC002817
:105A900001D06AA0B1E76EA004F050F9C82009F067
:105AA00079FABFF34F8F72497048C860BFF34F8FC8
:105AB000FEE700000040000111C011CA6170707360
:105AC000773A20626F6F7473657474696E672072C1
:105AD00065636F726420696E76616C69642C2072F4
:105AE000656675736520746F207377697463680DDC
:105AF0000A00000075736167653A20617070737702
:105B0000205B317C325D20286E6F20617267203D02
:105B10002073776974636820746F20746865206FE0
:105B2000746865722062616E6B290D0A00000000C6
:105B300061707073773A20616C7265616479206F6F
:105B40006E20415050256C750D0A00000040020186
:105B500061707073773A2062616E6B256C7520728C
:105B600065636F726420696E76616C696420286178
:105B70006464723D30782530386C582073697A65DA
:105B80003D256C75290D0A0000800001617070735D
:105B9000773A20766572696679696E6720746172FA
:105BA00067657420696D616765206372632028668C
:105BB0006577207365636F6E6473292E2E2E0D0A30
:105BC00000000000200E0301202020202020207251
:105BD000756E20424C45204F544120746F207772DF
:105BE00069746520612076616C696420696D616704
:105BF000652066697273740D0A000000617070732D
:105C0000773A2062616E6B256C7520696D616765FE
:105C1000206F6B20287665722030782530386C58DC
:105C20002C20256C752042292C20737769746368B9
:105C3000696E672E2E2E0D0A0000000061707073D1
:105C4000773A20666C617368206661696C0D0A00A2
:105C500061707073773A20646F6E652C2072657383
:105C6000657474696E672E2E2E0D0A000400FA0505
:105C700000ED00E010B50B488CB01EC803940293F1
:105C8000019200911EC80794069305920491426800
:105C9000016880680A9009920891684603F09EFBAB
:105CA0000CB010BD00400001F0B58DB00E460328C9
:105CB00007DA54A004F042F85AA004F03FF85F4815
:105CC0000FE00024B76822460BA938460B94FEF774
:105CD0000BFD05460B98B84202D00078002804D08E
:105CE00057A004F02BF80DB0F0BD5A4B87CB0397AB
:105CF00002920191009087CB07970692059104903C
:105D00009A68596818680A920991534A009908904C
:105D10006846914205D1282103F012FF0A99884272
:105D20000DD0009401940294039404940594069475
:105D300007940894099449A00A9403F0FFFF55A121
:105D40007068FEF7BCFA002804D0706801786229F8
:105D500008D02BE0012D03D0022D01D04FA0C0E7C9
:105D600001953AE04178312902D0322902D01DE074
:105D700002AC00E006AC51A1801CFEF7A0FA00289E
:105D800016D070684FA1801CFEF799FA002819D030
:105D900070684EA1801CFEF792FA00281AD0706835
:105DA0004BA1801CFEF78BFA002815D049A098E77C
:105DB0004E48854204D04E48854201D04DA090E720
:105DC00025600AE007208003854201D958A088E7B2
:105DD000656002E0A56000E0E5602A465DA07168AC
:105DE00003F046FF684603F0CBFA002801D062A01A
:105DF00077E766A003F0A2FF684603F0EFFA0DB064
:105E0000F0BD000075736167653A20627373657455
:105E1000203C6669656C643E203C76616C3E0D0AF0
:105E20000000000020206669656C643A206163749C
:105E3000697665203C317C323E0D0A00680E030114
:105E400062737365743A206261642076616C756573
:105E50000D0A00000040000111C011CA6273736591
:105E6000743A206578697374696E67207265636F30
:105E7000726420696E76616C69642C20726562754B
:105E8000696C642066726F6D2073637261746368FD
:105E90000D0A0000616374697665000062737365C2
:105EA000743A20616374697665206D75737420623D
:105EB000652031206F7220320D0A00006164647227
:105EC0000000000073697A650000000063726300DF
:105ED0007665720062737365743A20756E6B6E6FCF
:105EE000776E206669656C640D0A00000080000111
:105EF0000040020162737365743A20616464722029
:105F00006D7573742062652043414949435F415078
:105F100050315F42415345206F722043414949430C
:105F20005F415050325F424153450D0A000000006E
:105F300062737365743A2073697A65206578636566
:105F4000656473207468652062616E6B2073697A82
:105F5000650D0A0062737365743A202573203D2035
:105F600030782530386C582C2077726974696E67E8
:105F70002E2E2E0D0A00000062737365743A20669F
:105F80006C617368206661696C0D0A0062737365E9
:105F9000743A206F6B20287665726966696564299A
:105FA0000D0A000000B583B0002103200B4601223A
:105FB00001910090920203A1034809F061FC03B033
:105FC00000BD0000434C4900D163020110B5022816
:105FD00005DB48680DA1FEF772F9002805D00D48D1
:105FE0000078002804D00CA103E006F0C3FF10BD28
:105FF0000BA110A003F03CFE124C13A0218903F06A
:1060000037FE1CA0E16803F033FE10BD6A736F6EAB
:10601000000000008847002076616C696400000081
:1060200064656661756C7420286E6F742073617688
:1060300065642900706172616D733A2025730D0AE1
:1060400000000000AC5C002020206C6564203D2036
:1060500025752020286C65643120626C696E6B2088
:1060600068616C6620706572696F642C206D73299D
:106070000D0A0000202070776D203D20256C7520D2
:10608000202870776D20647574792C202525290DC2
:106090000A000000F3B595B015980D46032807DAFD
:1060A0006F4803F04BFE6FA003F048FE79A023E099
:1060B0007FA16868FEF703F9002810D00020AE68C1
:1060C0000246009069463046FEF70EFB04460098F3
:1060D000B04202D0007800287BD077A00CE00024EA
:1060E0000226B00014902858FEF7E2F80746E0199F
:1060F000801C502804D975A003F020FE17B0F0BD15
:10610000002C03D0202069460855641C14983A4698
:10611000295868460019FEF7A7F81598E419761C67
:106120008642DEDB002069460855451E6E462C4639
:1061300005F02EFB304603F059FC060023D003F097
:106140003AFC00281FD069A1304603F0FDFB07464A
:1061500003F028FC002800D07D6965A1304603F0DB
:10616000F3FB074603F01EFC002800D07C69002DDD
:1061700013DA002C22DA5FA003F0E0FD304603F0D2
:10618000B9FB17B0F0BD65A003F0D8FD002EF8D024
:10619000304603F0AFFB17B0F0BD294666483239F0
:1061A000814209D3654A322165A003F061FD304682
:1061B00003F0A0FB17B0F0BD002C0BDB642C09DD55
:1061C000642164A003F054FD304603F093FB17B044
:1061D000F0BD14E0304603F08DFB002D01DB62487A
:1061E0000581002C01DB6048C46006F017FF002821
:1061F00001D05EA080E706F0BDFE17B0F0BD3BA168
:106200006868FEF75CF8002807D039A16868FEF7D7
:1062100056F800280DD05CA06EE72046464932387B
:10622000884203D3454A322145A015E04E480481F7
:1062300009E0642C05D9642146A003F019FD17B0CC
:10624000F0BD4948C46006F0E9FE002801D055A021
:1062500052E7224659A0696803F00AFD17B0F0BD65
:10626000DC0D030120206C6564203D206C656431E9
:1062700020626C696E6B2068616C66207065726963
:106280006F642035302E2E3130303030206D730D5C
:106290000A000000202070776D203D2070776D206F
:1062A0006475747920302E2E31303020250D0A008F
:1062B0006A736F6E000000006170707365743A203D
:1062C0006261642076616C75650D0A00617070739F
:1062D0006574206A736F6E3A206C696E6520746F06
:1062E0006F206C6F6E670D0A000000006C65640023
:1062F00070776D00617070736574206A736F6E3AA9
:10630000206E6F206B6E6F776E206B657920286C26
:1063100065642C2070776D290D0A00006170707320
:106320006574206A736F6E3A2070617273652066BF
:1063300061696C0D0A000000DF26000010270000D4
:106340006C65642072616E67652025752E2E25753B
:106350000D0A000070776D2072616E676520302E27
:106360002E25750D0A000000AC5C00206170707372
:106370006574206A736F6E3A20666C61736820667C
:1063800061696C0D0A000000756E6B6E6F776E2090
:10639000706172616D20286C65642C2070776D29A6
:1063A0000D0A00006170707365743A20666C617349
:1063B00068206661696C0D0A000000002573203DAD
:1063C00020256C752C2073617665640D0A00000031
:1063D000002498B0F4A725461594661E38461294FA
:1063E000FDF766FF81B2384603F0C2F90027FF438C
:1063F0003946684603F01CF90028F7D015980028A4
:1064000005D000211591694609788142EED0129895
:1064100001281FD0022826D0684600781B287DD08E
:1064200009287CD00D287BD00A287AD0082879D07A
:106430007F2877D0014620395F29D7D23F2C72D2EE
:10644000E5490855641CA4B20121684603F090F99F
:106450002546CBE7684600785B2802D000201290E2
:10646000C4E70220FBE7002012906846007841282C
:1064700016D04228BAD1002EB8DB761E57D4D748A2
:106480004078801BC01DC117490F0918C908C900F1
:10649000401A8101D24809184038FDF735FF49E01C
:1064A000CE48711C02789142A0DA4078761C801B9D
:1064B000C01DC117490F0918C908C900401A810138
:1064C000C74809184038FDF71FFFC3480290FDF781
:1064D000EFFE87B2C3A42046FDF7EAFE81B2204654
:1064E00003F046F90024002D0BD9C1A00190FDF75F
:1064F000DFFE81B2019803F03BF9641CA4B2AC4208
:10650000F3D3B8A42046FDF7D3FE81B2204603F0B2
:106510002FF9002F34D03946029805E036E038E0F4
:10652000E2E0E3E029E136E103F022F928E0AA49BC
:1065300000200870A8480290FDF7BAFE87B2A9A40F
:106540002046FDF7B5FE81B2204603F011F9002484
:10655000002D0BD9A6A00190FDF7AAFE81B20198EB
:1065600003F006F9641CA4B2AC42F3D39DA4204608
:10657000FDF79EFE81B2204603F0FAF8002FCAD143
:106580003D469548FDF794FE84B22FE70120129016
:106590002CE703F0CBF8904800252F46019003F03C
:1065A000FEFA1390224620210198FDF796FE00285E
:1065B00060D1019908551399149000295AD914985B
:1065C00003F0F0FA224616900199FDF7A6FE002886
:1065D00019D1002F0AD102A81699FDF795FE02A83D
:1065E000FDF766FE85B20DE06D1EADB2A54206D97F
:1065F0002A4602A81699FDF790FE0028F4D1002043
:1066000002A948557F1C14981399401C1490884285
:10661000D5D3002F64D0012F1AD0A5422BD902AFB9
:106620003F2C5DD2AC425BD23819012103F0A0F8B7
:106630000198395D0155641CA4B2F1E738190121B4
:1066400003F096F80198395D0155641CA4B200E08E
:1066500002AF3F2C44D2AC42F0D301982021015527
:10666000641C63A5A4B22846FDF722FE81B2284629
:1066700003F07EF834E05FA52846FDF719FE81B2ED
:10668000284603F075F81398002500281CD92846E1
:1066900003F088FA074622460199FDF73EFE0028DE
:1066A0000ED13846FDF704FE81B2384603F060F89B
:1066B00051A73846FDF7FCFD81B2384603F058F883
:1066C00013986D1C8542E2D34AA52846FDF7F0FDDC
:1066D00081B2284603F04CF82146019803F0DEFA17
:1066E000254603F033F881E60A2000E00D201590DE
:1066F00003F01CF83FA52846FDF7DAFD81B22846D5
:1067000003F036F83449002008550D462878002853
:106710001FD0324C207800280AD06078C01D400776
:10672000C10D2F4808182946FDF7C9FD002810D0D3
:10673000607881012A4808182946FDF7E5FD607850
:10674000401C4007400F60702078082801D2401C90
:106750002070002003F0ECFA1F4803F02FFA1CA46D
:106760002046FDF7A5FD81B2204603F001F802F0B6
:10677000EDFF002425463E4638E6002CB3D0641ECB
:106780001EA5A4B22846FDF793FD81B2284602F06B
:10679000EFFF25462AE61AA73846FDF789FD81B2A4
:1067A000384602F0E5FF21E60D0A434C49207265A8
:1067B0006164792E2054797065202768656C702794
:1067C00020666F7220636F6D6D616E64732E0D0AAB
:1067D00063616969632D3E00C0500020444700207A
:1067E000005100200D63616969632D3E00000000C7
:1067F000200000000D0A00002020000008200800F2
:106800000700000010B50C46022812DB0EA16068DC
:10681000FDF755FD002809D00CA16068FDF74FFD7C
:10682000002804D00AA003F089FA10BD012001F06D
:106830006BFF01F063FF002801D003A100E003A17A
:106840000AA003F015FA10BD6F6E00006F666600B7
:1068500075736167653A20626C656C6F67205B6F6A
:106860006E7C6F66665D0D0A00000000626C65203C
:106870006C6F673A2025730D0A000000F8B502F02E
:10688000CFF9074602F0C8F90546254A25A128A0F8
:1068900003F0EEF902F0F2F901462CA003F0E8F95A
:1068A0002F48874203D12FA003F048FA15E000F0EB
:1068B0002DFF044602F014FA06460A213846FDF779
:1068C00077FC0A460146002C01D0A06900E00020B8
:1068D000009033462BA003F0CBF902F01DFA0146DD
:1068E00032A003F0C5F93548854203D134A003F046
:1068F00025FA03E029463AA003F0BAF909F08CF82A
:106900007D21C900FDF73EFC014639A003F0B0F936
:1069100008F07CFC01463AA003F0AAF9F8BD00009B
:106920001100010056312E30302E313700000000AA
:106930006669726D776172653A2025732028307818
:106940002530386C58290D0A00000000637572204C
:1069500062616E6B3A2041505025750D0A000000AF
:10696000FF7F0000636869702074656D703A204194
:10697000444320726561642074696D656F75740DA0
:106980000A000000636869702074656D703A202504
:10699000642E2564204320286164633D257520749E
:1069A00072696D3D256C75290D0A00007664643AA4
:1069B000202575206D560D0A00000000FFFF000025
:1069C00066616E2072706D3A206E2F6120286E6FA6
:1069D00020746163686F6D65746572290D0A00002B
:1069E00066616E2072706D3A2025750D0A000000F8
:1069F000757074696D653A20256C7520730D0A00F9
:106A00006672656520686561703A20257520420DC3
:106A10000A00000002F0C6FA00280DD007A003F01B
:106A20008DF9C82008F0B6FABFF34F8F114910480E
:106A3000C860BFF34F8FFEE70FA0F0E76661637495
:106A40006F72793A20666C61736820777269746539
:106A5000206661696C65642C207265736574746965
:106A60006E6720616E797761792E2E2E0D0A0000F7
:106A70000400FA0500ED00E0666163746F7279202E
:106A800064656661756C747320726573746F72658A
:106A9000642C20726573657474696E672E2E2E0DDA
:106AA0000A00000070B5194D0E46022819DB0024BB
:106AB0000C20604329587068FDF701FC002807D0BE
:106AC000641C0F2CF4D312A0716803F0D1F870BDD0
:106AD0000C20444360194268295916A003F0C8F8F5
:106AE00070BD17A003F02AF9002420460C2148436A
:106AF00041194A6829580FA003F0BAF8641C0F2CFA
:106B0000F3D312A003F01AF970BD00004809030185
:106B1000756E6B6E6F776E20636F6D6D616E643A2C
:106B20002025732028747279202768656C702729C6
:106B30000D0A00002020252D38732025730D0A0032
:106B4000636F6D6D616E64733A0D0A006B657973E6
:106B50003A20544142203D20636F6D706C6574652E
:106B60002C2055502F444F574E203D206869737498
:106B70006F72790D0A00000070B50C46032823DB04
:106B800060680178312902D0322906D01CE04078B3
:106B9000002819D1184E012504E04078002813D1AF
:106BA000164E402516A1A068FDF789FB00280FD0DE
:106BB00014A1A068FDF783FB00280ED012A1A068E5
:106BC000FDF77DFB00280DD011A003F0B7F870BDD4
:106BD0002946304600F050FB08E02946304600F0D8
:106BE00047FB03E02946304600F018FB11A0A268DD
:106BF000616803F03DF870BD000C014000080140E1
:106C00006F6E00006F666600746F67676C650000EA
:106C100075736167653A206C6564203C317C323E57
:106C2000203C6F6E7C6F66667C746F67676C653E38
:106C30000D0A00006C656420257320257320646FA5
:106C40006E650D0A0000000006A003F077F8C8206A
:106C500008F0A0F9BFF34F8F07490648C860BFF39B
:106C60004F8FFEE7726573657474696E672E2E2E02
:106C70000D0A00000400FA0500ED00E010B508F070
:106C8000CBFE7D210446C900FDF77CFA0246214671
:106C900010A002F0EDFF08F0AFF8014614A002F0DA
:106CA000E7FF08F0B9FA044608F0B0FA02460521F9
:106CB0002346090311A002F0DBFF1DA003F03EF8FC
:106CC000274900200870084608F084F9244803F09A
:106CD00035F810BD757074696D653A20256C7520A6
:106CE0007469636B732028256C752073290D0A0065
:106CF0007461736B733A2025750D0A0068656170C5
:106D00003A20746F74616C20257520422C206672C5
:106D1000656520257520422C206D696E206576659D
:106D200072206672656520257520420D0A000000FC
:106D30006E616D6520202020202020202020202032
:106D400020737461746520207072696F20207374E1
:106D500061636B28772920206E756D0D0A00000095
:106D6000E04E002010B506A002F0E8FFE121490244
:106D70000BA002F07DFF16A002F0E0FF10BD0000A6
:106D80007573617274313A2054583D504236205226
:106D9000583D5042372028414634290D0A00000052
:106DA000626175643A20256C752C2038206461740A
:106DB0006120626974732C206E6F20706172697437
:106DC000792C20312073746F70206269740D0A0071
:106DD000666C6F7720636F6E74726F6C3A206E6FA3
:106DE0006E653B2074783A20444D41204348312061
:106DF00028706F6C6C6564293B2072783A20525879
:106E0000444E45206972712071756575650D0A00E3
:106E100010B5E1246402204602F050FC214602A095
:106E200002F026FF10BD0000757361727420726558
:106E30007365743A20256C7520384E312C20727899
:106E400020717565756520666C75736865640D0ADB
:106E50000000000010B506A108A002F009FF0DA077
:106E600002F06CFF1948016819A002F001FF10BD83
:106E700056312E30302E3137000000006669726DB9
:106E8000776172652076657273696F6E3A2025733B
:106E90000D0A00006D636D2D6464632D626C653AAC
:106EA00020424C4528726474737329202B2046724B
:106EB000656552544F53202B205541525428444D60
:106EC0004129202B20434C490D0A0000004000209E
:106ED00053797374656D436F7265436C6F636B2098
:106EE0003D20256C7520487A0D0A000048607047E7
:106EF00001681A4A1140016000210160416081600F
:106F0000C160174A1749904204D148680F221043C4
:106F100048607047144A904204D14868F0221043F8
:106F200048607047114A904205D148680F2212020A
:106F30001043486070470E4A904205D148680F22BE
:106F400012031043486070470A4A9042FBD14868D8
:106F50000F2212041043486070470000FEFF00003B
:106F600008000240000002401C00024030000240C5
:106F700044000240580002400029016802D001226A
:106F8000114301E0014A114001607047FEFF00001B
:106F9000024609680020114200D00120704700001D
:106FA00030B403680D4A0C6A13408A684D69224365
:106FB0000C692C4322438C692243CC6922434C6ADE
:106FC00022438C6A22431A430260CA6842600A68FC
:106FD00082604968C16030BC704700000F80FFFFCD
:106FE000002B01D010617047002010617047000035
:106FF000014948617047000000040140054B002230
:1070000019685B690140034202D0002900D00122C7
:10701000104670470004014010B483791949026892
:10702000002B28D00B6893430B604A6803689A438F
:107030004A600279521813680468234313608A680F
:1070400003689A438A60CA6803689A43CA604279AF
:10705000102A06D051180A68006802430A6010BC62
:1070600070478A6803681A438A60CA6800680243E6
:10707000CA6010BC704700794018016891430160F4
:1070800010BC7047000401400B680022002B56D052
:10709000F0B401240B68944023424AD04B68022B81
:1070A00001D0122B16D113070AD5456A5307DB0E00
:1070B0000F269E40B5434E699E402E43466209E02E
:1070C000056A5307DB0E0F269E40B5434E699E406E
:1070D0002E4306624B68012B05D0112B03D0022BE7
:1070E00001D0122B06D14568DB06DB0FA543934088
:1070F0002B4343600568530003279F400E79BD432F
:10710000B607B60F9E402E430660C5688E68BD4325
:107110009E402E43C66085680126A543CC689440F6
:107120002C438460C46A9E400D69B4439D4025434E
:10713000C5620B68521CD340ABD1F0BC704770479E
:1071400005490160002242600F21826041610121F6
:107150000261C16070470000FF3F0000816270471C
:107160008161704742694A404261704782B0EFF3E3
:107170000884FCF7BBFF400701D5EFF309840AA0A0
:1071800000F084FBE06800900CA0A36862682168AE
:1071900000F07CFBE069009014A0A369626921699A
:1071A00000F074FBFEE700000A2A2A2A20486172D8
:1071B000644661756C74202A2A2A0A005230202005
:1071C0003D2530386C5820523120203D2530386C18
:1071D0005820523220203D2530386C582052332020
:1071E000203D2530386C580A000000005231322012
:1071F0003D2530386C58204C5220203D2530386CCD
:107200005820504320203D2530386C58207850536A
:10721000523D2530386C580A0000000010B5FFF7C9
:10722000A1FF10BD30B505460E4887B00C4685421B
:1072300002D10121042004E00B48854210D1012134
:10724000082000F021F90948844209D86846FFF770
:1072500077FF01200190694600942846FFF714FF4C
:1072600007B030BD00080140000C0140FF3F0000A6
:1072700010B5FFF773FF10BD10B5FFF771FF10BD1C
:1072800010B400214156FF23CAB29207D40E4278AF
:10729000A3409207120EA24000290BDA0907090F3A
:1072A00008398C081049A4006118CC699C43144328
:1072B000CC6107E08C080D49A40061180C689C4360
:1072C00014430C60827801210078002A04D0C006A3
:1072D000C00E8140064803E0C006C00E814005484C
:1072E000016010BC7047000000ED00E000E400E029
:1072F00000E100E080E100E0F7B5FFB004460025C2
:10730000A5B00520EFF31087FF210090453102A8BA
:10731000FCF7C3FFEFF31086FF21453153A8FCF7BC
:10732000BCFF53A8013001909822224953A8FCF7D2
:107330009BFF012080F310880198804786F3108816
:1073400001221D49120303265300360388420AD145
:1073500094421AD09C4201D1151116E0B44210D1CA
:1073600001256D0211E0154988420AD1944201D1EC
:1073700015460AE09C4201D11D4606E03546AC4266
:1073800003D000987FB028B0F0BD06ACFF220134D6
:1073900041320B4902A8FCF767FF012080F31088F7
:1073A0002846A69AA599A04787F310887FB028B0F1
:1073B000F0BD000044FE0201C440130085601300CC
:1073C00004FD020110B5EFF31084012181F3108850
:1073D000FF210906401803490968884784F310888B
:1073E00010BD00000440002010B5084806490160A7
:1073F0000749416007498160C92292000649074850
:10740000FCF732FF10BD0000E148002004400020DE
:107410007549002049480020E8FE0201404800204C
:1074200010B5EFF31084012383F31088FF231B06AC
:10743000C018034B5B68984784F3108810BD0000A8
:1074400004400020034AD16A102399430143D162CA
:107450007047000000100240044A0029516901D021
:10746000014300E081435161704700000010024079
:10747000044A0029916A01D0014300E081439162EE
:107480007047000000100240044A0029916901D0B1
:10749000014300E081439161704700000010024009
:1074A0000122054912060128086802D090430860AD
:1074B00070471043FBE700000010024030B4164A4A
:1074C000516804231940154B01D0042901D00360F1
:1074D00001E0134901605168124B8906890F5B5C1A
:1074E0000168D940416053680F4C5B055B0FE35C5A
:1074F0000D46DD40856053689B045B0FE35CD9401B
:10750000C160D16AC90601D5084901E07D21C903DE
:10751000016130BC70470000001002400090D003B1
:107520000048E801DCFE0201E0FE020100093D0026
:107530007047000010B5FCF7EFFD044608F072FA42
:10754000002803D001200349000748602046FCF7CB
:10755000E7FD10BD00ED00E010B50A4C2069411CAC
:1075600001D000280AD10120064934220003FFF788
:10757000C3FE2069411C03D0002801D0024810BD81
:10758000002010BD0C48002035480020F0B5564CB6
:1075900085B0E06921040843E0618120534D000675
:1075A000286353486861534828625348032201689E
:1075B000920391430160514934228014FFF79CFEED
:1075C0004E4B4F4E18694F4F411C29D0002827D0F1
:1075D000A9691A7849094901D206D20E0A43AA615B
:1075E0002168EA139143216021687F2212029143AE
:1075F0000002084320606068304360606068B84300
:1076000060606068211508436060206A3E49084058
:107610002062206AD96809020843206205B0F0BDE3
:1076200061682046314361606168B94361606168A7
:107630000127BF0239436160002104917D21C90007
:107640000391002100917F214024002502950191A2
:10765000026861028A4302600E11234908687F2292
:1076600012029043220202430A600520FCF736FD15
:107670000120FCF733FD1C48406B800704D42846EA
:1076800003996D1C8842F3D91748C06B80B2B04291
:1076900001D9811B00E0311AB94202D2E2B28FB2A5
:1076A0000292B04201D3019400E00094019A009844
:1076B0008018C005000EA04203D004460498814201
:1076C000CBD8094801687F2212029143029A120224
:1076D0000A4302604168490849004160416849071E
:1076E000FCD405B0F0BD0000001002400070004066
:1076F0000F08000018000200001001400C48002094
:107700000000010000070000FF00F8FF10B50A4C60
:107710002069411C01D000280AD1012006493422E9
:107720000003FFF7E9FD2069411C03D0002801D0C8
:10773000014810BD002010BD0C48002010B501F01C
:1077400093FF10BD10B40B06CC065B0FE40E0121B5
:10775000A140012B07D0022B07D01430002A026869
:1077600005D00A4304E00C30F8E71030F6E78A430E
:10777000026010BC704700000029818903D00122FB
:107780005203114301E0024A114081817047000019
:10779000FFDF0000002A828A01D00A4300E08A430A
:1077A000828270470246128800200A4200D00120DF
:1077B000704770B40A06530FCE060125F60E2A460E
:1077C0000024B240012B0FD0022B10D0838A13402B
:1077D000090A00888D402840002B02D0002800D0E4
:1077E0000124204670BC704783891340F0E7038A68
:1077F000EDE7000070B50446008A86B00D461B49CF
:107800000840E98801432182A08919492A89084052
:10781000A98811436A8902431143A181A08A1549AD
:107820000840A9890143A1826846FFF747FE124834
:10783000844201D1039800E0029829681922890046
:107840005043FCF79FFC06466421FCF79BFC0501B6
:10785000280964214843301A00013230FCF792FCB9
:107860000007000F2843208106B070BDFFCF000045
:10787000F3E90000FFFC0000003801408088C005EB
:10788000C00D7047C905C90D818070470FB410B590
:1078900003A9044B044A029800F066F910BC08BC26
:1078A00004B0184731A20201C40100200FB410B582
:1078B00004A9074B02AA039800F056F9044602A94E
:1078C000002000F0F8FC204610BC08BC04B01847AB
:1078D000B78202017CB51546024600201C460029ED
:1078E0000BD0491E00920191044B6A46214628465E
:1078F00000F03AF9009A002111707CBDA1820201CA
:107900002021020C01D010211046020A01D010469D
:107910000839020901D01046091F820801D010461B
:10792000891E420801D0881E7047081A704700005F
:10793000004870470848002030B5002805D0164C94
:10794000021F20680023014605E0084630BD904232
:1079500003D8034640680028F9D1002B00D05968AD
:10796000002B0AD01C68D51AA54204D11268A418AD
:107970001A461C6002E05A6000E02260002807D02E
:107980001468851AA54203D105686419146040681B
:107990005060184630BD000000480020F1B50E4C84
:1079A0000F480C4E001B0D4FC508ED00002211467C
:1079B000009803F005FF002803D13068002801D0AB
:1079C0000020F8BD3C600020256060600120306030
:1079D000ECE7000004480020D4AD0020004800205F
:1079E000D0AF0020F0B51FB486B00998089A030DF7
:1079F0000021024314D05148514A1818504305142D
:107A00001198012810981AD0281A401C00264D4FB2
:107A10004D49009601910490002812DA444211E089
:107A20001198012449A3012801D11098C143069857
:107A3000119A84600360C26041600BB0F0BD4042A7
:107A4000E4E70446210500203F4A001C5141039110
:107A5000029012E0E00707D032463B4601990098B9
:107A6000FCF7C6FF0191009032463B46104619468E
:107A7000FCF7BEFF06460F466410002CEAD10498BE
:107A8000039B0028029A0999089806DAFCF7B0FFD0
:107A9000019B009AFCF7ACFF05E0FDF711F8019B94
:107AA000009AFDF70DF804460E460022284BFDF71C
:107AB00053F903D80020C043014607E00022254BBC
:107AC00020463146FCF7E2FEFDF7FEF8102409E0FF
:107AD000002C0ADB0A220023FCF77EFB079B3032D6
:107AE0001A55641E02460A43F2D11122641C079BF8
:107AF000121B1C19119B012B03D0012308430ED12B
:107B00000AE0084304D0112010900020119077E77C
:107B10001098151A6D1E0BE01098824202DD0023AA
:107B20006D1C03E0824201DA00236D1E002BEED0B3
:107B3000069811998260C16030C07EE701FCFFFFAA
:107B4000104D0000000014400000F03F3000000025
:107B50000000F0430000E03F30380A2801D2012045
:107B60007047002070470000FFB597B0064600251B
:107B700018E2252877D100242746FD49049400E027
:107B80000443761C32780120203A90400842F7D115
:107B900030782A280ED0022230780146303909295F
:107BA00016D804990A235943303940181443761CD7
:107BB0000490F1E7189802C804911890002904DA9B
:107BC0000120400304434842049002200443761CF1
:107BD00030782E2814D1042004437078761C2A288B
:107BE00009D11898761C80C8189009E00A214F43E3
:107BF000303FC719761C3078014630390929F5D94C
:107C000030786C2810D006DC4C281AD068280ED0AA
:107C10006A2817D104E0742813D07A2812D110E012
:107C20000120400504430CE00121090501E0032186
:107C300009050C437178814203D101200005241805
:107C4000761C761C3078119066280BD013DC5828EF
:107C50007DD009DC00287BD04528F6D04628F4D01A
:107C600047281AD1A5E118E0632835D0642870D0E0
:107C7000652812D19DE170286CD008DC6728F1D00E
:107C800069287BD06E280DD06F2806D1BAE0732802
:107C90002ED0752871D0782859D01A9A1999904702
:107CA0006D1C7EE16002400F022809D003280DD030
:107CB0000428189801680DD00D60001D189070E11F
:107CC0001898EA1701680D604A60F6E7189801688D
:107CD0000D80F2E70D70F0E718986A46017811728E
:107CE000001D18900020507202A80090012005E0AD
:107CF000189802C8189000200091C04361070DD564
:107D0000002101E00199491C0191B94212DA814236
:107D1000F8DB009A515C0029F4D10BE0002101E06E
:107D20000199491C01918142FADB019A0099895C11
:107D30000029F5D1019904981A9B471A2146384623
:107D4000199A00F097FA0199401945180BE04FE095
:107D50002CE113E04EE0009800990078491C009156
:107D60001A9A199990470198401E0190401CF2D12F
:107D7000214638461A9B199A10E137E00A20002163
:107D8000009001916002410F022907D0189A01CAA0
:107D90001892C2179446032908D00AE01898C01D0B
:107DA000C108C90005C91891944607E000B2C2177E
:107DB0009446042902D140B2C1178C460022614684
:107DC000944506DA0A460021404291418C462D2115
:107DD00002E0210504D52B216A461173012103E03D
:107DE000E10701D02021F7E7029155E00A200AE0DF
:107DF000102008E01020009000210420044301918D
:107E0000082703E008200021019100906002410F43
:107E1000022907D0189A01CA189200229446032911
:107E200008D008E01898C01DC108C90005C91891FC
:107E3000944603E080B2042900D1C0B2002102912F
:107E4000210729D51199702906D0009A1021019B8C
:107E50004A401A4305D00EE040216A4611730121C1
:107E600008E06146014306D030216A46117311993A
:107E7000517302210291009A0821019B4A401A4342
:107E80000AD16146014301D1610705D530216A4617
:107E9000117301217F1E02911199582904D035A137
:107EA0000E910DA90D910DE037A1F9E76146019BF7
:107EB000009AFCF791F90E9B8C469B5C0D9A521E22
:107EC0000D92137061460143F0D10D9805A9081A6F
:107ED00020300190600703D501200004844300E0B6
:107EE00001270198874201DD381A00E0002001993E
:107EF00000904118029809180498401A0490E00371
:107F000006D421461A9B199A049800F0B3F9451932
:107F1000002706E003A81A9AC05D199990476D1CC6
:107F20007F1C02988742F5DBE0030CD521461A9BA3
:107F3000199A049800F09EF9451904E01A9A302025
:107F4000199990476D1C0099481E00900029F5DC96
:107F500008E00D980D990078491C0D911A9A19990D
:107F600090476D1C0199481E01900029F1DC63E1E6
:107F700009280100303132333435363738396162FF
:107F800063646566000000003031323334353637C3
:107F900038394142434445460000000000F05AF998
:107FA0004519761C3078002800D0E2E528461BB041
:107FB000F0BD600700D406271898C01DC108C9008D
:107FC00048680A680831C30FDB071891190001D00F
:107FD0009CA108E0210501D59BA104E0E10701D0A7
:107FE0009AA100E09AA1430011985B0810916528BE
:107FF0000CD006DC452809D046281DD0472841D1A1
:1080000041E0662818D067283CD13CE00021112FC0
